:020000040002F8
:10600000F8B40020DD630200E5630200A18802000D
:10601000E9630200EB630200ED6302000000000090
:10602000000000000000000000000000EF6302001C
:10603000F163020000000000F3630200F563020058
:106040001DA20200F7630200F763020055B50200CB
:1060500069B50200F7630200F763020031B1020084
:10606000F7630200F7630200F7630200F7630200C0
:10607000F7630200F7630200F7630200F7630200B0
:10608000D5C70200A5AC0200F7630200F763020067
:10609000F7630200F7630200E1B50200F763020054
:1060A000F7630200F7630200F7630200F763020080
:1060B000DDA20200F7630200000000000000000003
:1060C000F7630200F7630200F76302007DB5020088
:1060D000BDAC0200F7630200F7630200000000009D
:1060E00000000000000000000000000000000000B0
:1060F00000000000000000000000000000000000A0
:10610000000000000000000000000000000000008F
:10611000000000000000000000000000000000007F
:10612000000000000000000000000000000000006F
:10613000000000000000000000000000000000005F
:10614000000000000000000000000000000000004F
:10615000000000000000000000000000000000003F
:10616000000000000000000000000000000000002F
:10617000000000000000000000000000000000001F
:10618000000000000000000000000000000000000F
:1061900000000000000000000000000000000000FF
:1061A00000000000000000000000000000000000EF
:1061B00000000000000000000000000000000000DF
:1061C00000000000000000000000000000000000CF
:1061D00000000000000000000000000000000000BF
:1061E00000000000000000000000000000000000AF
:1061F000000000000000000000000000000000009F
:10620000DFF80CD000F0F4FC0048004785CF030015
:10621000F8B4002000B583B002900091019244F2DE
:10622000010071466A460AF08BF803B000BD000019
:1062300030B450E8012F93B2C48923448489A34227
:1062400028BF1B1B0489A34202BFBFF32F8F00206E
:1062500007E0C3EA020340E80134002CE9D14FF023
:1062600001000A6030BC704750E8012FC2EA0242C8
:1062700040E801210029F7D1704730B450E8022FDF
:106280001FFAA2F3C488A34202BFBFF32F8F0020DE
:106290000DE0C48923448489A34228BF1B1BC2EAA2
:1062A000034340E80234002CE8D14FF001000A60BB
:1062B00030BC704750E8022FC2EA224240E8022177
:1062C0000029F7D17047034653E8022FD988B2EB73
:1062D000324F4FF0000017BF92B241EA014142EA4B
:1062E000014104E05A68B2EB324F08BF012043E895
:1062F0000212002AE8D1704730B4044654E8000F77
:106300000D4644E80053002BF8D1156030BC7047AF
:1063100030B4044654E8000F40EA010544E8005355
:10632000002BF7D1156030BC704730B4044654E8F8
:10633000000F00EA010544E80053002BF7D1156077
:1063400030BC704730B4044654E8000F80EA0105C1
:1063500044E80053002BF7D1156030BC704730B4CF
:10636000044654E8000F00EB010544E80053002BFD
:10637000F7D1156030BC704730B4044654E8000FC4
:10638000A0EB010544E80053002BF7D1156030BCA9
:10639000704770B404464FF0000054E8006F0D6879
:1063A000AE4207BF44E80023012044E800630E60CA
:1063B000002B1CBF0020F0E770BC704730B40446CF
:1063C00054E8000F88422CBF451A054644E80053A4
:1063D000002BF5D1156030BC70470000064880479F
:1063E00006480047FEE7FEE7FEE7FEE7FEE7FEE7BA
:1063F000FEE7FEE7FEE7FEE799C202000162020047
:106400002DE9F05F0546002092469B4688460646E9
:10641000814640241BE0284641464746224600F07C
:10642000C8FA53465A46C01A914110D3114618462D
:10643000224600F0AFFA2D1A67EB01084F462246BC
:106440000120002100F0A6FA17EB00094E41201EA2
:10645000A4F10104DFDC484631462A464346BDE844
:10646000F09F40EA01039B0703D009E008C9121F0F
:1064700008C0042AFAD203E011F8013B00F8013BFE
:10648000521EF9D27047D2B201E000F8012B491E2A
:10649000FBD270470022F6E710B513460A460446C1
:1064A0001946FFF7F0FF204610BD421C10F8011BF3
:1064B0000029FBD1801A704710B5002200E0521C61
:1064C000835C8C5CA34201D1002BF8D1D8B2E1B23D
:1064D000401A10BD30B504460020034600E05B1CA6
:1064E000934203D2E05CCD5C401BF8D030BD2DE977
:1064F000FE4F804681EA0300C00F0C46009021F059
:10650000004123F00045B8EB0200A94105D2404606
:10651000214690461C460B46024623F0004010439D
:1065200047D0270DC7F30A00C3F30A510290401A5F
:10653000019040286BDAC3F3130040F4801B0098ED
:10654000924620B10023D2EB030A63EB0B0B0198B8
:106550005946C0F14002504600F01CFA06460D466E
:1065600050465946019A00F034FA10EB0800614198
:10657000002487EA115284EAE7731A4340D0009A54
:1065800062B3019A012A4FEA075215DC001B61EB46
:1065900002014FF0004202EA0752CDE90042001C1E
:1065A00041F5801132462B4600F06BFA03B0BDE88E
:1065B000F08F40462146F9E7001B61EB0201001C09
:1065C00041F5801300185B412018A2F5001747EB36
:1065D000030140EAD570B6196D4111E06D084FEA2C
:1065E000360645EAC0754FEA0752001B61EB02010F
:1065F000001C41F5801149084FEA30000019514153
:1066000032462B4603B0BDE8F04F00F02BBA00989D
:10661000012240000023D0EB020263EBE0730098FC
:1066200021464FEAE074B8EB000061EB0401E9E7B2
:1066300083F000435BE781F0004158E72DE9FE4F0E
:1066400081EA030404F0004421F0004100944FF07B
:10665000000B23F0004350EA01045ED052EA030429
:106660005BD0C3F30A54C1F30A552C44A4F2F334AB
:106670000194A0FB0254C1F3130141F48011C3F350
:10668000130343F4801301FB024400FB034E840A0E
:10669000970A44EA815447EA8357A4FB07680295A6
:1066A0008D0A05FB07854FEA932C04FB0C54270544
:1066B000029D4FEA065847EA1637B5EB08056EEB20
:1066C000070C870E920E47EA811742EA8312A7FB56
:1066D0000201B6EB0B0164EB00042B0D43EA0C3313
:1066E0005E1844EB1C50DA465146E7FB0201C5F345
:1066F00013044FEA0B3343EA14534FEA0432019C6C
:1067000043EA0603A4F10C040294009CCDE900B412
:1067100000F0B7F903B0BDE8F08F00200146F9E7BB
:106720002DE9F04D81EA030404F0004B21F000450F
:1067300014464FF0000A23F0004150EA050220D031
:1067400054EA01021DD0C5F30A570246C5F31303EC
:10675000C1F31300C1F30A5640F4801543F48013CB
:10676000A7EB0608101BD64608F2FD3873EB0500B0
:1067700002D308F1010801E092185B41B8F1000F63
:1067800003DA00200146BDE8F08D00204FF48011AF
:10679000064684460EE0171B73EB050705D3121B54
:1067A00063EB050306434CEA010C49084FEA30004D
:1067B00092185B4150EA0107EDD152EA030012D072
:1067C00082EA040083EA0501084305D0101BAB41AF
:1067D00006D20122002306E000224FF0004302E02F
:1067E0006FF0010253101AEB06004CEB085110EB4E
:1067F0000A0041EB0B01BDE8F04D00F033B90EB5D6
:10680000C10F80EAE0700844CA07002140F2334318
:106810008DE80E000A460B4600F033F903B000BDC8
:106820000EB540F2334102910021CDE900110A4634
:106830000B4600F026F903B000BD70B5C1F30A5253
:1068400001F000450024C1F3130140F2FF3341F48D
:1068500080119A4201DA002070BD40F233439A421F
:10686000A2F2334203DC524200F0A3F800E0904071
:106870002C43F1D0404270BDC1F30A5210B5C1F3B0
:10688000130140F2FF3341F480119A4201DA0020F3
:1068900010BD40F233439A42A2F2334203DC52422B
:1068A00000F087F810BD904010BD00F0004230F0BD
:1068B00000400AD0C10D01F56071C0F3160042EA34
:1068C0000151C2084007114370470020014670473C
:1068D00030B5041E71F1000404DB4FF00044404267
:1068E00064EB0101141E73F1000405DB1C464FF03C
:1068F0000043524263EB04038B4208BF824230BD27
:1069000030B5041E71F1000404DB4FF00044404236
:1069100064EB0101141E73F1000405DB1C464FF00B
:106920000043524263EB0403994208BF904230BDDA
:1069300001F0004330B421F0004150EA010206D0DA
:106940000A0DA2F56072C1F31301002A02DC30BC0B
:1069500000207047440F44EAC104C100E01830BC75
:1069600000EBC25000F047B830B50B46014600209E
:106970002022012409E021FA02F59D4205D303FA01
:1069800002F5491B04FA02F52844151EA2F1010282
:10699000F1DC30BD202A04DB203A00FA02F10020AD
:1069A00070479140C2F1200320FA03F3194390404D
:1069B0007047202A04DB203A21FA02F000217047B8
:1069C00021FA02F3D040C2F1200291400843194657
:1069D0007047202A06DBCB17203A41FA02F043EA3F
:1069E000E07306E041FA02F3D040C2F12002914088
:1069F0000843194670470029A8BF7047401C49004A
:106A000008BF20F00100704710B4B0FA80FC00FA13
:106A10000CF050EA010404BF10BC704749B1CCF13E
:106A2000200421FA04F411FA0CF118BF01212143CA
:106A30000843A3EB0C01CB1D4FEA00614FEA102085
:106A400042BF002010BC704700EBC3501044002927
:106A5000A4BF10BC7047401C490008BF20F00100D3
:106A600010BC704710B5141E73F1000408DA401C06
:106A700041F1000192185B411A4301D120F001005D
:106A800010BD2DE9F04D92469B4611B1B1FA81F24D
:106A900002E0B0FA80F220329046FFF77BFF044616
:106AA0000F4640EA0A0041EA0B0153465A460843A2
:106AB00013D0114653EA010019D0C8F140025046E4
:106AC000FFF777FF05460E46504659464246FFF708
:106AD00061FF084305D0012004E020463946BDE8A7
:106AE000F08D0020054346EAE0762C4337430A98B0
:106AF0006305E40AA0EB08000022FD0A44EA4754BB
:106B00000A3002D500200146E9E701051019694164
:106B1000DDE9084500196941BDE8F04DA2E72DE91E
:106B2000F04D00231A461B1A8A4103DB0020014660
:106B3000BDE8F08DC1F30A52C1F3130141F4801591
:106B40004FF0000BD10702D100186D41521E0027F3
:106B5000044640F2FF11384601EB620A3E46804689
:106B6000024600204FF48011FFF723FFC219714144
:106B7000BB1846EB0100B4EB030C75EB000C04D31F
:106B8000E41A65EB000517460E46241908F10100CA
:106B90006D4180463428E3DDF91946EB0600091BF8
:106BA000A84103D24FF0FF32134601E00022134602
:106BB0001BEB070046EB0A51BDE8F04DFFF752BF53
:106BC000C1F30A52C1F3130140F2FF3341F48011C3
:106BD0009A4202DA00200146704740F233439A425B
:106BE000A2F2334202DC5242FFF7E3BEFFF7D2BE0D
:106BF000064C074D06E0E06840F0010394E807000A
:106C000098471034AC42F6D3FFF7FEFA0C7104003B
:106C10002C71040070B58C1810F8015B15F0070397
:106C200001D110F8013B2A1106D110F8012B03E025
:106C300010F8016B01F8016B5B1EF9D12B0705D42D
:106C40000023521E0DD401F8013BFAE710F8013B76
:106C5000CB1A921C03E013F8015B01F8015B521E92
:106C6000F9D5A142D8D3002070BD10B519F0E4FFCA
:106C700010BD10B500F002F810BD0000F8B50027F7
:106C80001D480068009003208DF802006C461B4EE2
:106C900004B91B4C3146204619F0E2FE0DB14FF00D
:106CA000FF37002419E0174850F83400FF2813D0AC
:106CB000144800EBC4004068FF280DD0114A02EBD5
:106CC000C402526802EBC2020F4BD1180D4A02EB0C
:106CD000C402107919F02CFE641C082CE3DB0B486D
:106CE000006840B10948008881B2094819F0C0FD28
:106CF0000DB14FF0FF37F8BD146A040051EB0200EC
:106D0000106A040020410020AC790020604100207E
:106D1000F479002070B505460E4600242CE0184892
:106D200050F83400A84226D1154800EBC400406852
:106D3000B04220D1124901EBC401087919F064FE78
:106D400000200F4901EBC401496801EBC1010D4A64
:106D50001144C871FF200A4941F8340001EBC40115
:106D600048600948006820B107480068401E06498D
:106D70000860002070BD641C082CD0DB0420F9E7FB
:106D800020410020AC7900206041002070B504460D
:106D900094B10A48006808B9052070BDFFF765FF87
:106DA000FFF767FF19F030FF05460DB10820F4E743
:106DB000034804600020F0E70820EEE7604100206F
:106DC000644100202DE9FC5F054689461646494688
:106DD0002846FFF79FFF0024D0E06B4850F83400AE
:106DE000FF287DD1684800EBC4004068FF28F8D137
:106DF000FF2D75D0FFF739FF634840F8345000EBA2
:106E0000C400C0F80490604951F8340000BF4FF04E
:106E1000A042114601F5E06252F8202002F0010282
:106E20009246594850F8348000200090334602467C
:106E300001460190404618F0ACFA00BF00205249CC
:106E400001EBC401496801EBC101504A50544E495D
:106E500001EBC401496801EBC101114448704A4982
:106E600001EBC401496801EBC10111448870464936
:106E700001EBC401496801EBC1011144C870022053
:106E8000414901EBC401496801EBC101114408719A
:106E900000203D4901EBC401496801EBC1011144E7
:106EA0004871394901EBC401496801EBC101114442
:106EB0008871354800EBC4000079401C324901EB71
:106EC000C401496801EBC1011144C87100202E4979
:106ED00001EBC401496801EBC1011144087200E0F3
:106EE0004BE0294A02EBC402526802EBC202274B74
:106EF000D118254A02EBC402107919F019FD074692
:106F00008FB30020204901EBC401496801EBC101A6
:106F10001E4A1144C871FF201B4941F8340001EB9F
:106F2000C4014860184850F83480D346BBF1000FC4
:106F300009D10020009003460246014601904046D8
:106F400018F027FA09E000BF4FF0A04108460121E0
:106F500001FA08F1C0F8181500BF00BFFFF789FE5D
:106F60000320BDE8FC9FFFE709480068401C084972
:106F70000860FFF77EFE0020F3E7641C082CFFF694
:106F80002CAF0320EDE7000020410020AC79002069
:106F9000604100202DE9F04106460F461446984610
:106FA000069DB0EE000A84ED000A95ED020AB1EEEE
:106FB000400A84ED010A95ED010A84ED020A95ED7F
:106FC000020A84ED030AB0EE000A84ED040A95ED8E
:106FD000000AB1EE400A84ED050A95ED010AB1EE12
:106FE000400A84ED060A95ED000A84ED070AB0EE2A
:106FF000000A84ED080A4146204614F001FDB0EE77
:10700000000A84ED000A95ED020A84ED010A95ED6F
:10701000010AB1EE400A84ED020A95ED020AB1EED2
:10702000400A84ED030AB0EE000A84ED040A95EDEF
:10703000000A84ED050A95ED010A84ED060A95ED36
:10704000000AB1EE400A84ED070AB0EE000A84EDB2
:10705000080A3A464146204617F0A1F8242239464C
:107060002046FFF7FEF93A463146204617F097F8DA
:10707000242239463046FFF7F4F9BDE8F0810000DC
:1070800010B5054A05A1002003F082FC074A08A1BB
:10709000012003F07DFC10BD15710200424C455FDC
:1070A000436C69656E745F527800000015730200CE
:1070B000424C455F436C69656E745F547800000014
:1070C00030B50346104A1068002900DC30BD0022AC
:1070D00014E00D4C2468601C0C4CA04201D3A4F5B4
:1070E00080600B4C2468A04206D09C5C064D2D6845
:1070F0002C70054C206000E002E0521C8A42E8DB64
:1071000000BF00BFE2E70000384000201059002017
:107110003C40002070B565E03348007810B101288C
:107120005BD12BE000F058FC032800D270BD00209A
:1071300000F032FCAA2803D0012000F0E7FC1CE09C
:10714000022000F029FC0446E043C4B2012000F014
:1071500023FC2649087008460078844209D1084675
:107160000078052805DB20480078401C1E4908707F
:1071700002E0012000F0CAFC00BF32E000F02CFC6D
:107180001A490978884200D2D0E70025002406E099
:10719000204600F001FC2844C5B2601CC4B213486C
:1071A0000078401EA042F3DC10490978491E88B2DD
:1071B00000F0F2FBA84208D10C48007803F094FCE0
:1071C0000A48007800F0A2FC02E0012000F09EFCDA
:1071D00000200549087000BF03E000200249087044
:1071E00000BF00BF98E70000484000204940002051
:1071F00010B5024610480068122802D34FF0FF3045
:1072000010BD0E480C4B1B6800EB0310C1600B480F
:10721000094B1B6800EB031002700948074B064C32
:10722000246803EB0413586003480068401C024BB9
:1072300018600020E4E700004040002010590020C2
:10724000305A00202DE9F047C0B0804689461646E6
:1072500000250024701D00F0FF0AFA2E03DD601ED9
:1072600040B0BDE8F087AA200DF804002046611C5C
:10727000CCB21DF800002844C5B20DF804A0204689
:10728000611CCCB21DF800002844C5B26FEA0A00A8
:10729000C0B20DF804002046611CCCB21DF80000FD
:1072A0002844C5B20DF804802046611CCCB21DF8FC
:1072B00000002844C5B200270CE019F807000DF8BB
:1072C00004002046611CCCB21DF800002844C5B261
:1072D000781CC7B2B742F0DB2046611CCCB20DF877
:1072E0000050214668461DF0F1FFB9E708490AE061
:1072F0000A68824204D100234376136A0B6001E0DE
:1073000002F1200100BF0A68002AF1D17047000095
:107310004440002070B5002600251E48046831E076
:10732000E06800282BD005F007F91B490968451AC9
:1073300005F002F91849086005B90125E068A8427E
:1073400003D3E068401BE06001E00020E060E068FB
:10735000A8B9207A00280ADD207A401E20726068D1
:10736000E060227E207C6169FFF76CFF07E0204629
:10737000FFF7BCFFE06910B12046E1698847607EF5
:107380000643246A002CCBD13146AFF2770003F0DC
:10739000D9FA70BD444000204C4000202DE9F04156
:1073A0000446884615461E4613480768ECB184F823
:1073B0001080656126766068E0602078002803DD33
:1073C0002078401E207201E00020207201206076AB
:1073D00004E0A74201D1BDE8F0813F6A002FF8D157
:1073E0000548006820620448046032462946404649
:1073F000FFF728FF00BFEEE74440002010B5054A24
:1074000005A1002003F0C4FA064A07A1012003F0F9
:10741000BFFA10BDBD740200424C455F486F7374E3
:107420005F527800CD760200424C455F486F73741E
:107430005F5478002DE9F04104460D461B4806686C
:10744000052D01DABDE8F0816778A078C04300F02F
:10745000FF082078AA280CD147450AD1AF4208D1AD
:10746000E078052805DAE9B22046114A126890470B
:1074700019E0002014E00D4909684E1C0D498E42A8
:1074800001D3A1F580660C4909688E4206D0215CC3
:10749000064A1268117005490E6000E002E0401CC7
:1074A000A842E8DB00BF00BFCCE70000504000204E
:1074B00058400020305F00205440002070B565E047
:1074C0003348007810B101285BD12BE000F094FA2A
:1074D000032800D270BD002000F06EFAAA2803D065
:1074E000012000F037FB1CE0022000F065FA0446A2
:1074F000E043C4B2012000F05FFA26490870084654
:107500000078844209D108460078052805DB204828
:107510000078401C1E49087002E0012000F01AFBB0
:1075200000BF32E000F068FA1A490978884200D2B8
:10753000D0E70025002406E0204600F03DFA28446C
:10754000C5B2601CC4B213480078401EA042F3DCF0
:1075500010490978491E88B200F02EFAA84208D1D5
:107560000C48007803F000FB0A48007800F0F2FABB
:1075700002E0012000F0EEFA00200549087000BF8B
:1075800003E000200249087000BF00BF98E7000038
:10759000644000206540002010B502461048006895
:1075A000122802D34FF0FF3010BD0E480C4B1B6861
:1075B00000EB0310C1600B48094B1B6800EB031084
:1075C00002700948074B064C246803EB041358600B
:1075D00003480068401C024B18600020E4E70000EC
:1075E0005C400020305F00205060002001460248CF
:1075F0000160002070470000584000202DE9F0474E
:10760000C0B080468946164600250024701D00F053
:10761000FF0AFA2E02DD40B0BDE8F087AA200DF87F
:1076200004002046611CCCB21DF800002844C5B2FD
:107630000DF804A02046611CCCB21DF800002844BF
:10764000C5B26FEA0A00C0B20DF804002046611C02
:10765000CCB21DF800002844C5B20DF804802046C5
:10766000611CCCB21DF800002844C5B200270CE014
:1076700019F807000DF804002046611CCCB21DF873
:1076800000002844C5B2781CC7B2B742F0DB2046E0
:10769000611CCCB20DF80050214668461DF030FE4A
:1076A00000BFB8E708490AE00A68824204D1002313
:1076B0004376136A0B6001E002F1200100BF0A6803
:1076C000002AF1D1704700006040002070B500260C
:1076D00000251E48046831E0E06800282BD004F043
:1076E0002BFF1B490968451A04F026FF184908605A
:1076F00005B90125E068A84203D3E068401BE060BB
:1077000001E00020E060E068A8B9207A00280ADDE6
:10771000207A401E20726068E060227E207C6169D1
:10772000FFF76CFF07E02046FFF7BCFFE06910B1F0
:107730002046E1698847607E0643246A002CCBD14D
:107740003146AFF2770003F0FDF870BD60400020D5
:10775000684000202DE9F0410446884615461E4643
:1077600013480768ECB184F810806561267660687C
:10777000E0602078002803DD2078401E207201E0C0
:10778000002020720120607604E0A74201D1BDE80C
:10779000F0813F6A002FF8D1054800682062044854
:1077A0000460324629464046FFF728FF00BFEEE757
:1077B000604000200246002116E00E4850F82100EB
:1077C000904202D14FF0FF3070470A4850F8210034
:1077D00048B909480078401C074B1870054840F824
:1077E00021200020F0E7491C0329E6DB6FF00100AF
:1077F000EAE70000488200203C48002002460021C1
:1078000016E00E4850F82100904202D14FF0FF30B0
:1078100070470A4850F8210048B909480078401CD0
:10782000074B1870054840F821200020F0E7491C5C
:107830001029E6DB6FF00100EAE70000B07F0020CE
:107840000242002030B52DED048B83B0B0EE408AAB
:10785000F0EE608A3148007800285CD018EE900A7B
:10786000FFF723F841EC190B9FED2D0B53EC102B78
:10787000FFF746F804D3F4EEC88AF1EE10FA04D20A
:10788000032003B0BDEC048B30BDB1EE0E0AB4EEA4
:10789000C08AF1EE10FA01D20320F2E79FED220A2E
:1078A00028EE800ADFED210A80EE201ABCEEC10A24
:1078B00010EE100A80B2ADF806009FED1B0A28EE0C
:1078C000000ADFED1A0A80EE201ABCEEC10A10EEA3
:1078D000100A80B2ADF804004FF4C870ADF80A0089
:1078E0000020ADF808001249088901A975DF044697
:1078F000082C0ED0112C0CD05CB100BF25463DB138
:1079000000BF0CA240F2B2212846FEF783FC00BF64
:1079100000BF2046B5E70120B3E700003248002051
:1079200000000000003B9F4000007A4400409C445F
:10793000308000202E2E5C2E2E5C2E2E5C626C651C
:107940005F6366675C686F73742E63009FED0E2A39
:10795000C0EE022A9FED0D2A22EE822AB0EE421AD4
:107960009FED0B2A21EE022A22EE202ADFED092AC2
:1079700082EE223AF0EE431A90ED002A32EE212AEE
:1079800080ED002A7047000000803B45CDCC8C3F45
:1079900000007A44000061450246054800688118ED
:1079A0000448814201D3A1F5806108787047000046
:1079B0003C4000201059002002460548006881180C
:1079C0000448814201D3A1F5806108787047000026
:1079D00054400020305F0020054B1A68054B1968A1
:1079E0008A4201D3501A02E002F58063581A7047A8
:1079F000384000203C400020054B1A68054B1968B0
:107A00008A4201D3501A02E002F58063581A704787
:107A1000504000205440002070B517F074FB4FF424
:107A200096510D480186418690F82E0020F0040002
:107A3000094981F82E00084617F03DFB044600BFB7
:107A4000254635B100BF05A278212846FEF7E2FBA6
:107A500000BF00BF002070BD688000202E2E5C2E6D
:107A60002E5C2E2E5C626C655F6366675C686F736C
:107A7000742E630070B58AB0044600200990002679
:107A8000182103A8FEF706FD0020019002900025B2
:107A900004F0010008B90AB070BD12F03FFD0228E1
:107AA00000D0F8E709A808F05DFE00B9F3E701A8E7
:107AB0000FF024FD0646B6F1FF3F08D0BDF80400E4
:107AC00030B9BDF8060018B9BDF8080000B9E2E702
:107AD0000998411E03AA00200BF04CF9B0F1FF3FBA
:107AE0000ED001A903A814F023F90546002D07DBE9
:107AF0000448007810B901200249087002490D714C
:107B000000BFC8E7FA3F00207453002018E0411E70
:107B100088B20D4909680D4A1268914200D1704738
:107B200009490968491C0A4A914204D3A2F58061B7
:107B3000054A116004E004490968491C024A1160C1
:107B40000028E4D100BFEAE73C4000203840002094
:107B50001059002018E0411E88B20D4909680D4AED
:107B60001268914200D1704709490968491C0A4AC4
:107B7000914204D3A2F58061054A116004E00449F2
:107B80000968491C024A11600028E4D100BFEAE7F5
:107B90005440002050400020305F00200122014B63
:107BA0001A707047F44000200849095C01290CD183
:107BB000002206490A54891F898C31B10349891F63
:107BC000898C491E014A921F91847047F64F00200C
:107BD000004870471850002070B52DED068B064602
:107BE000164890F8540028BB1448C664144804682A
:107BF00000F03AFE0546AC4201D204F18074601BED
:107C0000FEF70EFE41EC1A0B9FED0E0B53EC102B02
:107C1000FEF786FD41EC190B9FED0C0B53EC102B7E
:107C2000FEF709FD41EC180BFEF726FE034908623A
:107C300008464462BDEC068B70BD0000A0FF00202A
:107C400004B50040FCA9F1D24D62404000000000A4
:107C50000070A740034991F8541009B9014908651B
:107C600070470000A0FF002001460348405C012847
:107C700000D170470020FCE7F64F002010B500212E
:107C8000064802F05FFE0120054908703220488056
:107C900001208880092001F075FC10BDA57E02003E
:107CA000F04F002010B51A48408800282ED001213E
:107CB000184802F047FE1648808868B914480078D2
:107CC00018B901201249087002E00020104908701C
:107CD00001200F49888014E00D48007818B90E493A
:107CE000092001F02FFC0A480078012804D14FF048
:107CF0007F41092001F026FC05488088401E044988
:107D0000888003484088401E0149488010BD00001B
:107D1000F04F0020A57E020000103FFF70B5044622
:107D2000241F4FF40070B0EB145F00D070BD083416
:107D30000120094981F854000846806C40F0020097
:107D40008864202221460448FEF78BFB2546A8695B
:107D5000C01EA86100BFE9E7A0FF00200649095C3A
:107D6000012908D0012204490A54891F898C491C21
:107D7000014A921F91847047F64F0020F0B5BFB0C2
:107D800006460F46002400253846FEF78EFB85B2D6
:107D9000F82D02D9601E3FB0F0BD07F053FB30B1A3
:107DA00000222046611CCCB20DF8002005E0012223
:107DB0002046611CCCB20DF800202046611CCCB2DC
:107DC0000DF800600DEB04002A463946FEF749FB2A
:107DD0006019C4B222466946AD20FFF733FADAE7EC
:107DE0000120064981F854000846806C40F00100EB
:107DF000886403480168014881627047A0FF002041
:107E000004B5004010B51648806D012809D05C21EA
:107E10001348FEF73FFB012011498865002081F8D7
:107E2000540026210F48FEF735FB01200D4908704C
:107E300032204880012088800B4A0CA1C82002F023
:107E4000A7FD0E4A0EA1642002F0A2FD1249AD204A
:107E5000FFF7A2FB242211491148FEF702FB10BDD7
:107E6000A0FF0020F04F0020A57E0200457863654A
:107E70007074696F6E5F4C6564000000117F0200D2
:107E8000457863657074696F6E5F556E6B6F776E62
:107E9000526573657400000057440300E4530020EA
:107EA0001850002000B589B000200AF06DFF0128AD
:107EB00011DB01AA002108460AF05CFFBDF80400AE
:107EC000ADF81C00BDF80600ADF81E00BDF80800B6
:107ED000ADF8200001E009B000BDBDF9200040F27E
:107EE000DC51884206DB0848808C002802DDFFF761
:107EF000D9FE06E0BDF920000449884201DCFFF705
:107F0000BDFE00BFE7E70000F04F002024FAFFFFAE
:107F100010B52DED048BCAB0FC210BA8FEF7BAFA00
:107F2000FC210BA8FEF7B6FA554890F8540001283A
:107F300039D15348806C00F00100002834D05048FB
:107F4000846A406AA04201D904F180744C49496AAC
:107F5000601AFEF765FC41EC190B9FED4A0B53ECE0
:107F6000102BFEF7DDFB41EC180B8DED028B444826
:107F7000006A00904248036DC26C44A10BA804F053
:107F800079FD0BA91120FFF7F9FE002873D13C48B9
:107F9000806C20F001003A4988640846806C002813
:107FA00069D181F8540066E03548806C00F0020029
:107FB000A8B322223B4B3248C1698069C01ECDE97B
:107FC0000832CDE906012E4840692D4909692C4A3D
:107FD000D2682B4B9B68CDE90232CDE904102848CA
:107FE000406827490968CDE900102548036DC26C37
:107FF0002D490BA804F03EFD0BA91120FFF7BEFE92
:10800000002838D11E48806C20F002001C4988648A
:108010000846806C20BB002081F854002BE0FFE76D
:108020001748806C00F00400D8B115482C3000903F
:108030002C38036DC26C1DA10BA804F01BFD0BA90D
:108040001120FFF79BFE58B90D48806C20F004000A
:108050000B4988640846806C10B9002081F85400F0
:1080600009E05C210648FEF715FA012004498865FD
:10807000002081F854004AB0BDEC048B10BD000014
:10808000A0FF0020FCA9F1D24D62404069643A3063
:108090007825782C307825782C25642C25660D0AD7
:1080A0000000000001040100B86F040069643A3068
:1080B0007825782C307825782C257300704770B59A
:1080C0000025002600240CE04FF4E62000EB0436E7
:1080D00030461BF0D7FF05460DB1032070BD601C74
:1080E000C4B2012CF0DB0020F8E770B500250026B3
:1080F00000240CE04FF4E82000EB043630461BF07F
:10810000C1FF05460DB1032070BD601CC4B2022C36
:10811000F0DB0020F8E770B50025002600240CE015
:108120004FF4EC2000EB043630461BF0ABFF054665
:108130000DB1032070BD601CC4B2022CF0DB002026
:10814000F8E710B504461C2221464FF4E62010F053
:1081500059F910BD7CB5002400200190DA48FFF7E2
:10816000F0FF0546D8480068D84988421FD1D64854
:10817000007E05280FDBFFF7B8FFFFF7CCFF0020DC
:10818000D149087600F0C0F918B1D1A10820FFF755
:10819000F5FD04F0CFFCCC48007E401CCA490876AF
:1081A00000F0B2F918B1CAA10820FFF7E7FDCD48E9
:1081B00015F071FA002436E004EB4401CA4A52F883
:1081C0002100FEF772F9064604EB4400C64A52F855
:1081D000201001AB3246C3481AF06BFB08BB04EB1E
:1081E0004400C14901EB8000007A9DF804108842E8
:1081F00017D104EB4401BC4A52F82100FEF755F9AF
:10820000064601A8009004EB4400B74A02EB800048
:10821000436804EB440052F820103246B1481AF08B
:108220000AFB601C84B21C2CC6DBB0480068A7495E
:10823000884276D0FFF759FFFFF76DFF9421AB48D6
:10824000FEF728F9A148A9490860002008719E4856
:1082500000689E49884231D100240DE09A48001DF3
:10826000015DA248801D015597480A30015D9F4875
:1082700033300155601C84B2062CEFDB002401E092
:10828000601C84B2062CFBDB002401E0601C84B27D
:10829000062CFBDB8C4801699448C1628A48818ABC
:1082A000924801868848807D904981F82800864858
:1082B000C07D08718448807E48710AE01C21824894
:1082C000FEF7E8F800F020F918B181A10820FFF7C7
:1082D00055FD00241EE004EB4401834A52F82100BE
:1082E000FEF7E3F8064604EB44007F4901EB80000B
:1082F000007A009004EB44000A4602EB80004368D9
:1083000004EB440052F82010324676481AF028FA5E
:10831000601C84B21C2CDEDB002074490860002441
:1083200037E044E004EB44016F4A52F82100FEF7C5
:10833000BCF8064604EB44006B4A52F8201001AB2F
:10834000324668481AF0B5FA08BB04EB44006649A7
:1083500001EB8000007A9DF80410884217D104EBED
:108360004401614A52F82100FEF79FF8064601A831
:10837000009004EB44005C4A02EB8000436804EB8D
:10838000440052F82010324656481AF054FA601C45
:1083900084B21C2CC6DB554800684C49884204D086
:1083A00053A10820FFF7EAFC7CBD04F0C3FB0024C6
:1083B00085E004EB44014C4A52F82100FEF775F8C1
:1083C000064604EB4400484A52F8201001AB3246FE
:1083D00044481AF06EFAE0BB04EB4400424901EB5A
:1083E0008000007A9DF80410884218D104EB440103
:1083F0003D4A52F82100FEF758F8064601A80090C1
:1084000004EB4400384A02EB8000436804EB44006C
:1084100052F82010324633481AF00DFA4DE004EBC2
:108420004401314A52F82100FEF73FF8064604EBBA
:1084300044002D4A52F8201032462A481AF0D5F945
:1084400004EB4401284A52F82100FEF72EF80646B4
:1084500000E015E004EB4400234901EB8000007AC2
:10846000009004EB44000A4602EB8000436804EBF2
:10847000440052F8201032461A481AF071F91CE0F4
:1084800004EB4401184A52F82100FEF70EF80646A4
:1084900004EB4400144901EB8000007A009004EBE7
:1084A00044000A4602EB8000436804EB440052F8A3
:1084B000201032460B481AF053F9601C84B21C2C71
:1084C000FFF677AF00BF6FE708540020AA5555AA02
:1084D00073617665206261636B7570206661696C9B
:1084E00000000000C43F002008680400745300200E
:1084F000466C617368207772697465206865616491
:10850000206661696C00000070B5002500261048E7
:108510001049086000240CE04FF4E62000EB04361C
:1085200030461BF0AFFD05460DB1032070BD601C49
:10853000C4B2012CF0DB072206494FF4E6201BF001
:10854000E7FD05460DB10220F0E70020EEE7000050
:10855000AA5555AA08540020F8B50025002422E0A9
:1085600004EB4401124A52F82100FDF79EFF064633
:1085700004EB44000E4901EB8000007A009004EB0C
:1085800044000A4602EB8000436804EB440052F8C2
:108590002010324607481AF0BAF905460DB10220FC
:1085A000F8BD601CC4B21C2CDADB0020F8E7000028
:1085B00008680400C43F0020F8B506460F4614467C
:1085C00033212248FDF766FF012020493C3981F81C
:1085D0003C00012E0CD06FF48050304478B1B0F5DF
:1085E000405F1CD06FF440510844002822D10DE0B8
:1085F000322217A11548401CFDF733FF21E032223B
:1086000019A11248401CFDF72CFF1AE025461DA1B8
:108610000E48401CD5E9003204F02CFA11E0254642
:10862000286800901EA10948401CD5E9013204F0D9
:1086300021FA06E03A461FA10448401C04F01AFA49
:1086400000BF00BFFFF788FFF8BD0000B053002057
:1086500053443A20415353455254494F4E204641CA
:10866000494C45440D0A000053443A20494E5641B6
:108670004C4944204D454D4F5259204143434553A9
:10868000530D0A00415353455254494F4E20464121
:10869000494C45442025733A25750D0A0000000019
:1086A0006572726F723A25752C25733A25750D0A1D
:1086B00000000000554E4B4E4F574E204641554C42
:1086C00054203078253038580A000000FEB549485B
:1086D000406AB0F5006F7CD208F070FD074608F0E4
:1086E00073FD3D184FF07F4000EA05604FF47F01B5
:1086F00001EA052108434FF47F4101EA15210843AF
:1087000040EA156002903C48007801280ED1FFF73E
:1087100002FD28B139A10B20FFF730FB0220FEBD7E
:108720000021344841620020334908703149496AC8
:108730004FF4EC2202EB8100012202A91BF0E8FCBD
:1087400006460EB10220EAE72A48406A401C294941
:10875000486208464169C16181690162FFF7FCFE18
:1087600018B12AA10820FFF709FB0424002001907A
:1087700038E004EB44012B4A52F82100FDF795FE46
:10878000074604EB4400274A52F8201001AB3A4652
:1087900025481AF08EF818BB04EB4400214901EB80
:1087A0008000007A9DF80410884219D104EB44013E
:1087B0001C4A52F82100FDF778FE074601A80090F8
:1087C00004EB4400174A02EB8000436804EB4400CA
:1087D00000E00AE052F820103A4613481AF02BF84D
:1087E000601CC4B2052CC4DB01E0022097E7002026
:1087F00095E7000074530020E03F0020636C656142
:10880000722073746570206661696C0073617665AF
:1088100020696E666F726D6174696F6E2066616942
:108820006C00000008680400C43F002000200D49CF
:10883000096891ED070ABCEEC00A10EE101AC8B222
:108840000A2806DD0A2190FBF1F000EB80014906C1
:10885000080E642801DD642002E0002800DC00200E
:1088600070470000904000200148006870470000F9
:1088700018410020094989790170084949794170F6
:108880000649097981700549C978C1700349897819
:108890000171024949784171704700000642002089
:1088A00000BFEFF30880804600BFEFF3098000BFF0
:1088B0004046FFF733FA0A2404B90DE000BF4FF435
:1088C0007A7505B904E0054EAF013846B04700BFE0
:1088D000601E041EF3D100BF04F00CF98167040090
:1088E00010B50021132016F076FF012017F008FDC7
:1088F0000021142016F06FFF012017F001FD012167
:10890000132016F068FF012017F0FAFC0021132055
:1089100016F061FF10BD1CB5002000900346012237
:1089200011460190132016F05CFD132016F034FE62
:10893000132016F0B0FE00200090034601221146DD
:108940000190142016F04DFD142016F025FE142081
:1089500016F0A1FE1CBD10B50021132016F03BFF40
:108960000121142016F037FF012017F0C9FC012166
:10897000132016F030FF012017F0C2FC0021132055
:1089800016F029FF10BD2DE9F04107460E461546A9
:108990009846002400F084F8384600F057F800F0BC
:1089A000AFF810B90020BDE8F081304600F04EF875
:1089B00000F0A6F808B90020F5E700F071F8791C7E
:1089C000C8B200F043F800F09BF808B90020EAE7CD
:1089D000002406E000F012F82855FFF781FF601C24
:1089E000C4B2A8F10100A042F4DC00F007F8285559
:1089F000FFF7B1FF00F06CF80120D4E770B5002557
:108A00000121142016F0E7FE00BF17E06006040EF7
:108A10000021132016F0DFFE052017F071FC012164
:108A2000132016F0D8FE052017F06AFC142016F06B
:108A30000EFE08B144F00104681CC5B2082DE5DB48
:108A40000021132016F0C7FE204670BD70B5044605
:108A5000002500BF1DE00021132016F0BCFE0520FC
:108A600017F04EFC04F0800020B10121142016F014
:108A7000B2FE03E00021142016F0ADFE6006040EE5
:108A80000121132016F0A7FE052017F039FC681C01
:108A9000C5B2082DDFDB0021132016F09CFE70BD4F
:108AA00010B50121142016F096FE0121132016F0B6
:108AB00092FE052017F024FC0021142016F08BFEF6
:108AC000052017F01DFC0021132016F084FE10BDB8
:108AD00010B50021132016F07EFE0021142016F0A0
:108AE0007AFE052017F00CFC0121132016F073FE0E
:108AF0000121142016F06FFE052017F001FC10BDB7
:108B000010B500240121142016F065FE012017F095
:108B1000F7FB0121132016F05EFE0BE0601CC0B2D3
:108B20000446322803DBFFF7D3FF002010BD0120ED
:108B300017F0E6FB142016F08AFD0028EED1002184
:108B4000132016F048FE0120F0E72DE9F0418046A1
:108B50000D4616461F460024FFF7A2FF4046FFF7CA
:108B600075FFFFF7CDFF10B90020BDE8F081284662
:108B7000FFF76CFFFFF7C4FF08B90020F5E70024FA
:108B800009E0305DFFF762FFFFF7BAFF08B9002088
:108B9000EBE7601CC4B2BC42F3DBFFF799FF012096
:108BA000E3E710B500210E2016F079FE012017F042
:108BB000BFFB00210C2016F072FE012017F0B8FB5D
:108BC00001210E2016F06BFE012017F0B1FB0021F1
:108BD0000E2016F064FE10BD1CB500200090034668
:108BE0000122114601900E2016F04BFC0E2016F0CB
:108BF000F1FC0E2016F065FD0020009003460122D6
:108C0000114601900C2016F03CFC0C2016F0E2FC02
:108C10000C2016F056FD1CBD10B500210E2016F0DC
:108C20003EFE01210C2016F03AFE012017F080FBD9
:108C300001210E2016F033FE012017F079FB0021F0
:108C40000E2016F02CFE10BD2DE9F04107460E4611
:108C500015469846002400F084F8384600F057F88E
:108C600000F0AFF810B90020BDE8F081304600F008
:108C70004EF800F0A6F808B90020F5E700F071F80A
:108C8000791CC8B200F043F800F09BF808B9002046
:108C9000EAE7002406E000F012F82855FFF781FF0C
:108CA000601CC4B2A8F10100A042F4DC00F007F897
:108CB0002855FFF7B1FF00F06CF80120D4E770B53C
:108CC000002501210C2016F0EAFD00BF17E0600628
:108CD000040E00210E2016F0E2FD052017F028FBFF
:108CE00001210E2016F0DBFD052017F021FB0C20E2
:108CF00016F0C5FC08B144F00104681CC5B2082D8B
:108D0000E5DB00210E2016F0CAFD204670BD70B5CF
:108D10000446002500BF1DE000210E2016F0BFFD17
:108D2000052017F005FB04F0800020B101210C2084
:108D300016F0B5FD03E000210C2016F0B0FD600632
:108D4000040E01210E2016F0AAFD052017F0F0FAFE
:108D5000681CC5B2082DDFDB00210E2016F09FFD38
:108D600070BD10B501210C2016F099FD01210E20D7
:108D700016F095FD052017F0DBFA00210C2016F007
:108D80008EFD052017F0D4FA00210E2016F087FD85
:108D900010BD10B500210E2016F081FD00210C2021
:108DA00016F07DFD052017F0C3FA01210E2016F004
:108DB00076FD01210C2016F072FD052017F0B8FA9F
:108DC00010BD10B5002401210C2016F068FD012013
:108DD00017F0AEFA01210E2016F061FD0BE0601CC9
:108DE000C0B20446322803DBFFF7D3FF002010BDDA
:108DF000012017F09DFA0C2016F041FC0028EED15E
:108E000000210E2016F04BFD0120F0E72DE9F04186
:108E100080460D4616461F460024FFF7A2FF404637
:108E2000FFF775FFFFF7CDFF10B90020BDE8F08117
:108E30002846FFF76CFFFFF7C4FF08B90020F5E7ED
:108E4000002409E0305DFFF762FFFFF7BAFF08B9C1
:108E50000020EBE7601CC4B2BC42F3DBFFF799FFD4
:108E60000120E3E710B50548007828B1044B054A16
:108E70000549064800F0DAF810BD00004C48002013
:108E80008DAD03006048002050480020EA83002098
:108E900001200149087070474C480020002001491A
:108EA000087070474C4800202DE9FC5F05460E46CF
:108EB00017469846DDE90CB9DDF838A0424800783D
:108EC00068B15B46424639463046CDE9009A1AF011
:108ED0001DF93E49A1F1500011F010F80CE05B467D
:108EE000424639463046CDE9009A0CF0B5F937498B
:108EF000A1F150000CF062F9304615F069FA044611
:108F0000002C5ED0CDB33048007828B12F495039BD
:108F10002F481AF08FFA54E02E4890F850302B4822
:108F2000503890F850102B4A0CF070F92A49A1F1F2
:108F300050000CF057F928485038B0F85200401C47
:108F400025495039A1F85200084690F8521090F87F
:108F50005000401C204A503A11541046B0F85200BC
:108F60000012114691F850105054104690F85030AD
:108F7000042100201CF0ECF923E0FFE713485038EF
:108F8000B0F85200401C11495039A1F8520008466F
:108F900090F8521090F85000401C0C4A503A11546E
:108FA0001046B0F852000012114691F8501050547B
:108FB000104690F85000801CC3B2042100201CF021
:108FC000C7F9BDE8FC9F00004C48002092830020B8
:108FD00050480020EE820020E683002070B5044651
:108FE0000D46E07804281AD16278211D0C48FDF75F
:108FF00038FA6078C01F0A4981F850006078801EF6
:10900000215C6078C01E205C41EA00200449A1F880
:1090100052000448007810B103481AF00BFA70BDF2
:10902000EE8200204C480020604800202DE9F041ED
:1090300004460E4615461F466548007810B10128C3
:109040000CD10CE06889002808DD01206049087017
:1090500028461AF0A5FA30461AF0A2FAB5E008E060
:1090600004F1540128461AF005FAB4F8A60059494B
:109070000880688971898842F2DC6889002867DD88
:1090800004F1540128461AF0F5F952480088401CB2
:1090900050490880B4F8A6000988884259D000BF1A
:1090A0004D480088401C4C4908804A480088401CB4
:1090B00048490880214630461AF0DCF9B4F85200DD
:1090C0004449098888423BD1214630461AF0D2F9FA
:1090D00094F8A43094F8501004F154022046B84794
:1090E0003E49A1F1500010F01BFF3C485038B0F849
:1090F0005200401C39495039A1F85200084690F8F6
:10910000521090F85000401C344A503A1154104606
:10911000B0F852000012114691F850105054114608
:10912000B1F8520000EBD0714910A0EB410131B908
:10913000104690F85030042100201CF009F907E097
:109140007089002803DC00202149087000E0A7E7AF
:109150003AE0214630461AF08DF994F8A43094F89C
:10916000501004F154022046B8471C49A1F15000A8
:1091700010F0D6FE19485038B0F85200401C17497C
:109180005039A1F85200084690F8521090F850005B
:10919000401C124A503A11541046B0F852000012C6
:1091A000114691F8501050541146B1F8520000EB9E
:1091B000D0714910A0EB410131B9104690F8503000
:1091C000042100201CF0C4F800BF00BFBDE8F081FE
:1091D0007048002072480020C03F0020E683002035
:1091E00070B505460C460020264908602648002137
:1091F00001604160816025480160416081604FF4F9
:10920000A2712348FDF746F9224800210160416020
:1092100081602148016041608160204801604160B7
:10922000816024211E48FDF735F924211D48FDF7F2
:1092300031F96C211C48FDF72DF94FF4A2711B4840
:10924000FDF728F924211A48FDF724F924211948AB
:10925000FDF720F924211248FDF71CF924211148BB
:10926000FDF718F9144890ED000A2146114811F055
:10927000A7FC24220F491148FDF7F3F800201049FC
:10928000086070BDD84900201C8E0020288E002068
:10929000508A0020948B0020048E0020108E002025
:1092A000A08B0020C48B0020E88B0020548C002071
:1092B000988D0020BC8D0020D0490020E08D00203A
:1092C000FC4900202DE9F0432DED048B87B0814649
:1092D0000D4600270026182101A8FDF7DBF8B0464F
:1092E0000024288810FB00F06A8812FB0200AA887C
:1092F00012FB020000EE100AB8EEC00A10EE101ABF
:109300000846FDF7D2FA41EC190BB0EE490AF0EE2F
:10931000690A04F0F9FAB0EE408AF0EE608A51EC86
:10932000180BFDF78AFA06462A48007801280CD166
:1093300000202849087000BF04E0274840F8246056
:10934000601CC4B2062CF8DB0DE0002407E02249C3
:10935000601C51F8200041F82400601CC4B2052CA8
:10936000F5DB1D48466118221B4901A8FDF779F875
:1093700000211FE0002017E001AA52F82030944697
:10938000421C5CF8222093420CDD01AB421C53F8D6
:10939000228001AA52F82030421C4CF8223001AA47
:1093A00042F82080421CD0B2C1F105028242E3DCC7
:1093B000481CC1B20529DDDB01990698401AB0F5B9
:1093C0007A7F00DB0127384607B0BDEC048BBDE88F
:1093D000F0830000A44000208471002010B501211A
:1093E000102016F0BEF900200149087010BD0000E1
:1093F000B44000202DE9F041012002F0F5F8FF23F0
:109400001A461946112002F0F5F8032002F002F97D
:1094100001F0FEFB00231A466021164801F0FCFB18
:1094200015490860102001210A46002306241D4624
:1094300000BF4FF0A0473E4641EA420747EA830794
:1094400047EA042747EA054C06F5E06747F820C0DD
:1094500000BF002116F085F9084A09A1052001F096
:1094600097FA084802F008F9074803F0DBFABDE86C
:10947000F08100009C710020B04000208D9402001B
:109480004C454400134903002549030010B500244E
:109490002048007810B1012835D126E01E48007818
:1094A00010B300201C49087009240DE01B4810F877
:1094B0003400002806DD194901EBC401486803F0B7
:1094C000A9F903E0601EC4B2002CEFDC00BF24B990
:1094D0000121102016F045F906E00021102016F0B9
:1094E00040F901200B49087011E00B48007818B1D1
:1094F00000200849087005E001220421084800689E
:1095000002F08EF803E000200249087000BF00BF9F
:1095100010BD0000B5400020B44000205C72002067
:10952000B04000200A2800DB7047044A02EBC0026A
:1095300051600122024B1A7000BFF5E75C720020F7
:10954000B44000200A2800DB70470C4A12F8302093
:10955000012A06D1094A02EBC00252688A4200D1B0
:10956000F2E70122054B03F830201A4602EBC00255
:1095700051600122024B1A7000BFE5E75C720020C7
:10958000B44000200A2800DB7047074911F830106A
:1095900001B9F9E70021044A02F830100121034A19
:1095A000117000BFF0E700005C720020B4400020A2
:1095B00010B50021052016F023F9012016F0ACFEAD
:1095C0000021042016F01CF9012016F0A5FE01214F
:1095D000052016F015F9012016F09EFE0021052049
:1095E00016F00EF910BD1CB50020009003460122B4
:1095F00011460190052015F008FF052015F0DBFF4E
:10960000052016F053F80020062103460122CDE97B
:1096100000101146042015F0F8FE042015F0CBFFD1
:10962000042016F043F8062015F077FF01210620EC
:1096300016F0E6F8032015F070FF1CBD10B50021F0
:10964000052016F0DDF80121042016F0D9F80120DC
:1096500016F062FE0121052016F0D2F8012016F066
:109660005BFE0021052016F0CBF810BD2DE9F0417E
:1096700007460E4615469846002400F084F8384602
:1096800000F057F800F0BDF810B90020BDE8F081F7
:10969000304600F04EF800F0B4F808B90020F5E7C5
:1096A00000F071F8791CC8B200F043F800F0A9F896
:1096B00008B90020EAE7002406E000F012F8285577
:1096C000FFF776FF601CC4B2A8F10100A042F4DCF1
:1096D00000F007F82855FFF7B1FF00F06CF8012003
:1096E000D4E770B500250121042016F089F800BFE9
:1096F00017E06006040E0021052016F081F8052011
:1097000016F00AFE0121052016F07AF8052016F061
:1097100003FE042015F0A7FF08B144F00104681C03
:10972000C5B2082DE5DB0021052016F069F82046BA
:1097300070BD70B50446002500BF1DE00021052066
:1097400016F05EF8052016F0E7FD04F0800020B169
:109750000121042016F054F803E00021042016F043
:109760004FF86006040E0121052016F049F8052087
:1097700016F0D2FD681CC5B2082DDFDB00210520E4
:1097800016F03EF870BD10B50121042016F038F82F
:109790000121052016F034F8052016F0BDFD00214A
:1097A000042016F02DF8052016F0B6FD0021052046
:1097B00016F026F810BD10B50021052016F020F88F
:1097C0000021042016F01CF8052016F0A5FD01214B
:1097D000052016F015F80121042016F011F80520D7
:1097E00016F09AFD10BD10B5052015F07EFE042080
:1097F00015F07BFE062015F078FE032015F075FEAF
:1098000010BD10B500240121042015F0F9FF01203E
:1098100016F082FD0121052015F0F2FF0BE0601C1F
:10982000C0B20446322803DBFFF7C5FF002010BD9D
:10983000012016F071FD042015F015FF0028EED16F
:109840000021052015F0DCFF0120F0E72DE9F041B3
:1098500080460D4616461F460024FFF794FF4046FB
:10986000FFF767FFFFF7CDFF10B90020BDE8F081DB
:109870002846FFF75EFFFFF7C4FF08B90020F5E7B1
:10988000002409E0305DFFF754FFFFF7BAFF08B985
:109890000020EBE7601CC4B2BC42F3DBFFF78BFF98
:1098A0000120E3E77CB51448007900B97CBD06F0DF
:1098B000E5FDF8B1002511F0D7F84042C6B20F48D7
:1098C000058800242A122146641C0DF80120EAB202
:1098D0002146641C0DF801202146641C0DF801602E
:1098E00023466A4603210020FDF758FD0020034966
:1098F000088000BF00BFD9E774530020C03F00209C
:109900002DE9F041022001210A4600242346254684
:1099100000BF4FF0A0473E4641EA420747EA8407AE
:1099200047EA032747EA054C06F5E06747F820C0F9
:1099300000BF00BF002115F0F7FEC82000F01AF8A4
:10994000084802F051FE084A08A1002001F020F862
:109950000121054800F0F6FF0549A420FDF748FC69
:10996000BDE8F081999902003D9A02004D54000033
:109970003D42030010B504464CB105480460012186
:10998000022015F0D1FE0121024800F0DBFF10BDDE
:109990006C4000203D9A020010B504462348006840
:1099A000002842D02148006868B320480068401E63
:1099B0001E4908601E480068082809D001210220BD
:1099C00015F0B2FE1A480068401C194908600CE006
:1099D00018480068022808D016480068401C15493D
:1099E00008600021022015F09FFE11480068082839
:1099F00010D11048006802280CD100200D490860E1
:109A00000B49086006E00020084908600949086021
:109A1000074908600548006838B90021022015F0A0
:109A200083FE0021044800F08DFF10BD6C40002033
:109A300074400020704000203D9A020070470000F2
:109A4000DFED150AC0ED000ADFED140AC0ED010AD2
:109A5000F7EE000AC0ED020ADFED0F0AC0ED030ABF
:109A6000DFED0D0AC0ED040ADFED0B0AC0ED050ABB
:109A7000DFED090AC0ED060ADFED070AC0ED070AAF
:109A8000DFED050AC0ED080AF7EE000A80EE801A45
:109A900080ED091A70470000000000000000C84275
:109AA000014890ED0B0A704778540020014890ED72
:109AB0000A0A704778540020014890ED0C0A70475C
:109AC00078540020F0EE400AF6EE001A60EEA11A7B
:109AD000B0EE611AB0EE600A10EE100A0C49A1EB6C
:109AE000600000EE100A21EE002AF7EE081A42EE9E
:109AF000401A61EE801AB0EE610A21EE002AF7EEFC
:109B0000081A42EE401A61EE801AB0EE610A704700
:109B1000DF59375F2DE9F041C0B007468846164649
:109B200000240025AA200DF804002046641C1DF81E
:109B300000002844C5B205200DF804002046641C2E
:109B40001DF800002844C5B2AF200DF804002046DF
:109B5000641C1DF800002844C5B20DF804702046AE
:109B6000641C1DF800002844C5B2F0B20DF80400D2
:109B70002046641C1DF800002844C5B200200AE0FD
:109B800018F800100DF804102146641C1DF801108F
:109B90002944CDB2401CB042F2DB2046641C0DF8D3
:109BA0000050A1B268461BF091FB40B0BDE8F081C7
:109BB00010B52DED108B98B00446F0EE409AB0EE43
:109BC00060AAF0EE41AAF0EE61CAB0EE42BAF0EE41
:109BD00062BAB0EE43CAF0EE638AB0EE449A9FEDEB
:109BE000FE0A84ED110AC4ED12CA84ED13BAC4ED65
:109BF00014BAF5EEC0CAF1EE10FA09D1B5EEC0BA4A
:109C0000F1EE10FA04D1F5EEC0BAF1EE10FA7CD004
:109C10006CEEAC0A4BEE0B0A4BEEAB0AB0EE600AF0
:109C2000FFF750FFB0EE408A2CEE880AF0EE40CAF3
:109C30002BEE080AB0EE40BA2BEE880AF0EE40BADE
:109C40006CEE0C0A48EEA80A49EE090AB0EE600A6A
:109C5000FFF738FFB0EE408A2CEE080AB0EE40CA9B
:109C600028EE880AF0EE408A29EE080AB0EE409A03
:109C700094ED020A20EE000A8DED170A94ED020A17
:109C8000D4ED030A20EE20EA94ED020AD4ED040A92
:109C900020EE20DA94ED020AD4ED050A20EE200A27
:109CA0008DED160A94ED030A20EE000A8DED150ADB
:109CB00094ED030AD4ED040A20EE200A8DED140A77
:109CC00094ED030AD4ED050A60EE20DA94ED040A5F
:109CD00060EE00EA94ED040AD4ED050A20EE20FAC5
:109CE00094ED050A60EE00FAB6EE000A30EE6E0A58
:109CF00030EE6F0A20EE0C1A9DED140ADDED160A07
:109D000070EE600AB0EE410A00E045E108EEA00AFC
:109D10007DEE8D0A09EE200AF0EE000A60EE200AC0
:109D2000CDED130A9DED140ADDED160A30EE200A82
:109D300060EE0C0A9DED150AB6EE001A31EE400AEF
:109D400030EE6F1AB0EE600A08EE810A7FEE4E0A1E
:109D500009EE200AF0EE000A60EE200ACDED120AAC
:109D6000DDED130A20EEA01ADDED120A00EEA01AB6
:109D7000B0EE410A03F005FE8DED110A3DEECD0A6D
:109D800020EE0C0A7FEE0E0A08EEA00ADDED150AA1
:109D9000B6EE001A71EE600A70EEEE0A09EE200AC5
:109DA000F0EE000A20EE200A8DED100A3DEECD0AFD
:109DB0008DED0F0A3EEE0F0A8DED0E0A9DED170A8E
:109DC000F6EE000A30EE600A30EE2F0A8DED0D0A35
:109DD000B6EE000A30EE6E0A70EE6F0A9DED110AC3
:109DE00020EE800A3DEECD1ADDED100A00EE810A6C
:109DF0008DED0C0A9DED140ADDED160A70EE600A79
:109E00009DED110A20EE800A3EEE0F1ADDED100ADC
:109E100000EE810A8DED0B0A7DEE2D0A9DED110AF3
:109E200020EE801A9DED150AF6EE000A30EEC00A0B
:109E300070EE6E1ADDED100AB0EE410A00EEA10AD6
:109E40008DED0A0A9DED0D0A6BEE000A9DED0E0ADE
:109E50004BEEC00A9DED0A0A28EE801A9DED0B0A12
:109E600009EE401A30EE810A8DED090A9DED0F0AC8
:109E70006BEE800A9DED0D0A4CEEC00A9DED0C0ABA
:109E800029EE001A9DED0A0A0CEE401A30EE810A06
:109E90008DED080A9DED0E0A6CEE800A9DED0F0A0D
:109EA0004BEE400A9DED0B0A2CEE001A9DED0C0ABC
:109EB00008EEC01A30EE810A8DED070A94ED000A13
:109EC000B5EEC00AF1EE10FA3CDD94ED060A94ED11
:109ED000001ADDED090A61EE200A94ED091A00EE80
:109EE000810A84ED060A94ED070A94ED001ADDED6F
:109EF000080A61EE200A94ED091A00EE810A84ED49
:109F0000070A94ED080A94ED001ADDED070A61EEE8
:109F1000200A94ED091A00EE810A84ED080A94EDF6
:109F2000060A30EE290AF0EE409A94ED070A30EE68
:109F30000A0AB0EE40AA94ED080A30EE2A0AF0EEC2
:109F400040AA0BE09FED240A84ED060A9FED220A49
:109F500084ED070A9FED200A84ED080A94ED011AAA
:109F60009DED090AF0EE690A41EE000AF0EE609AF2
:109F700094ED011A9DED080AF0EE4A0A41EE000A3E
:109F8000B0EE60AA94ED011A9DED070AF0EE6A0AA0
:109F900041EE000AF0EE60AA94ED090AF6EE000A1E
:109FA00020EE200A20EE290AF0EE409A94ED090AEC
:109FB000F6EE000A20EE200A20EE0A0AB0EE40AAD1
:109FC00094ED090AF6EE000A20EE200A20EE2A0A95
:109FD000F0EE40AA02E000000000000094ED020A4A
:109FE0008DED060A94ED030A8DED050A94ED040A41
:109FF0008DED040A9DED050AB1EE400A60EE290AD6
:10A000009DED040A40EE4A0A94ED050A40EE6A0A04
:10A0100094ED020A30EE800A84ED020A9DED060AF4
:10A0200020EE290ADDED040A00EEAA0AD4ED050AA5
:10A0300000EECA0AD4ED030A30EE200A84ED030ACA
:10A040009DED060A60EE0A0A9DED050A40EE6A0AD9
:10A0500094ED050A40EE290A94ED040A30EE800AD8
:10A0600084ED040A9DED060A20EE2A0ADDED050ABC
:10A0700000EE8A0ADDED040A00EEE90AD4ED050AD5
:10A0800030EE200A84ED050AD4ED020A60EEA00A43
:10A0900094ED031AD4ED031A41EE210A94ED041A4B
:10A0A000D4ED041A41EE210A94ED051AD4ED051AF7
:10A0B00041EE210AB0EE600AFFF704FDB0EE408ADF
:10A0C00094ED020A20EE080A84ED020A94ED030AD8
:10A0D00020EE080A84ED030A94ED040A20EE080A33
:10A0E00084ED040A94ED050A20EE080A84ED050AC1
:10A0F000D4ED031A94ED032AB6EE001A01EEC21A4B
:10A10000D4ED041A94ED042A01EEC21AF0EE410ACD
:10A1100094ED021AD4ED031A21EE211AD4ED041A9B
:10A1200094ED052A01EE821AB0EE410A03F0F0F92F
:10A13000DFED390A20EE200A84ED0A0AD4ED030A85
:10A1400094ED051A60EE810A94ED021AD4ED041A1A
:10A1500041EE610AB8EE001A60EE810AB0EE600AC4
:10A1600002F0DAFEDFED2C0A20EE200A84ED0B0A65
:10A17000D4ED041A94ED042AB6EE001A01EEC21AC8
:10A18000D4ED051A94ED052A01EEC21AF0EE410A4B
:10A1900094ED031AD4ED041A21EE211AD4ED021A1B
:10A1A00094ED052A01EE821AB0EE410A03F0B0F9EF
:10A1B000DFED190A20EE200A84ED0C0A94ED020A64
:10A1C00084ED0D0A94ED030A84ED0E0A94ED040A61
:10A1D00084ED0F0A94ED050A84ED100A04F144029F
:10A1E00004F13401684619F0BCF804F1340019F0A8
:10A1F000A5F804F13402694604F1440019F0B1F8FD
:10A2000094ED140AF7EE000A30EE600A84ED140AA9
:10A2100018B0BDEC108B10BDE12E654210B54FF4A7
:10A22000807014F072FF80B14FF4807014F076FFEC
:10A23000012014F07DFF2048407930B901201E49EB
:10A24000487108460168002088474FF4827014F076
:10A250005CFF50B14FF4827014F060FF022014F0E4
:10A2600067FF15480168012088474FF4887014F093
:10A270004CFF50B14FF4887014F050FF102014F0D0
:10A2800057FF0D480168022088474FF4867014F08C
:10A290003CFF80B10020094908604FF4867014F03B
:10A2A0003DFF082014F044FF002003498871084650
:10A2B00001680320884710BDA44A0020340C0040E8
:10A2C00010B51CF0E1F800F013F8FFF793F8FFF772
:10A2D00017FBFDF73FFFFDF795FD10BD10B50249D7
:10A2E000024811F0C1FC10BDB44A002000C001407A
:10A2F00010B5034A03A147F2305000F049FB10BDEE
:10A30000A1A30200505752002DE9F041FFF766F873
:10A3100008F010FD0DF02AF90220002161B900BFFC
:10A3200000BF4FF0A0421346012505FA00F2C3F822
:10A330000C2500BF00BF0CE000BF00BF4FF0A042E3
:10A340001346012505FA00F2C3F8082500BF00BF37
:10A3500000BF00BFC82014F0FDFEFCF786FC0421FE
:10A360001C20FCF7D7FC1C220020022100231D46E4
:10A370001E4600BF4FF0A04C674643EA450C4CEA2E
:10A38000800C4CEA062C4CEA014C07F5E06848F8D2
:10A3900022C000BF00BF33DF0446BDE8F0810000EB
:10A3A00010B5FEF743FA002833D10FF0F5FF01286E
:10A3B0002FD1FEF78BF918B116A10D20FDF7DEFCA9
:10A3C000242218491848FCF74CF800201749487611
:10A3D000FEF79AF818B116A10D20FDF7CFFCFEF795
:10A3E000BBF818B118A10D20FDF7C8FC4FF47A7026
:10A3F000FFF7C0FA0DF068FF002406E005F0C2F890
:10A40000642014F0A7FE601CC4B20A2CF6DBFFF730
:10A410007BFF10BD73617665207374657020666183
:10A42000696C000018500020E453002008540020FC
:10A430007077722073617665206261636B7570203E
:10A440006661696C00000000707772207361766548
:10A4500020696E666F726D6174696F6E20666169E6
:10A460006C00000010B5044694F9130010F1140FAD
:10A4700028DDA08B102825D11348007810BBA069D7
:10A48000007A46281ED1A069407A55281AD1A069C1
:10A49000807A4E2816D1A069C07A5F2812D1012097
:10A4A0000949087010210948FBF7F4FF0749A06922
:10A4B00082680A60C0684860002000E0401CA18BF0
:10A4C0008142FBDC10BD000033400020005500201D
:10A4D00010B52DED048BF0EE408AB0EE608A9FED52
:10A4E000D20AB0EE409AD148006890F8210020B11D
:10A4F000012870D002286CD1D7E0B3EE040AB4EE84
:10A50000C08AF1EE10FA1BDD0220C849096881F803
:10A510002100B0EE680A0AF0F7FBC448006880ED3D
:10A52000050AC2480068D0ED050AB0EE600AF0EEF8
:10A53000490A12F01BFDBD48006880ED060A48E09C
:10A54000B0EE680A02F0E8F8B848006880ED050A45
:10A550000120B649096881F82100B2EE040AC8EE6C
:10A56000800AF0EE609AB0EE690A10F093FFAF48EF
:10A570000068D0ED050A30EE600AF2EE0E0AB4EE85
:10A58000E00AF1EE10FA16DCB2EE040AC8EE800A18
:10A59000F0EE609AB0EE690A10F07CFFA348006804
:10A5A000D0ED050A30EE600AFAEE0E0AB4EEE00ACB
:10A5B000F1EE10FA0DD2B2EE040AC8EE800AF0EE07
:10A5C000609AB0EE690A10F065FF9848006880ED67
:10A5D000050A20E1FFE7B3EE040AB4EEC08AF1EE0B
:10A5E00010FA19DD02209149096881F821009FEDD8
:10A5F000900A8E48006880ED030A8C480068D0ED10
:10A60000050AB0EE600AF0EE490A12F0AFFC874886
:10A61000006880ED060A47E0B0EE680A02F07CF8B8
:10A620008248006880ED040A8048006890ED040AC2
:10A630007E480068D0ED050A30EE600AF2EE0E0AA0
:10A64000B4EEE00AF1EE10FA10DC7848006890ED04
:10A65000040A76480068D0ED050A30EE600AFAEE8A
:10A660000E0AB4EEE00AF1EE10FA08D26F48006864
:10A6700090ED040A6D48006880ED050A14E06B480F
:10A68000006890ED050A69480068D0ED040AB4EE50
:10A69000E00AF1EE10FA07DD6448006890ED040A64
:10A6A0006248006880ED050AB5E0B3EE040AB4EE36
:10A6B000C08AF1EE10FA27D201205C49096881F8BE
:10A6C0002100B2EE040AC8EE800A58480068C0EDC6
:10A6D000000A5648006890ED050ADFED560AB4EE10
:10A6E000E00AF1EE10FA0EDD0AF06EFB00280AD047
:10A6F0001E2014F0A0FF002805D19FED4F0A4B4803
:10A70000006880ED050A85E04848006890ED050A7C
:10A71000DFED4A0AB4EEE00AF1EE10FA00DD7AE06D
:10A72000F7EE000A414800681830B0EE480AFDF71D
:10A730000DF93E480068D0ED060AB0EE600AF0EE72
:10A74000490A01F0DDFF3948006880ED020AB0EEE9
:10A75000680A0AF0D9FA3548006880ED040A9FEDCE
:10A76000380AC8EE000A31480068C0ED030A2F48D5
:10A77000006890ED030AF7EE000AB4EEE00AF1EE8D
:10A7800010FA05DDB7EE000A2848006880ED030ADC
:10A790002648006890ED030AF7EE000A30EEC00A82
:10A7A00022480068D0ED040A20EE200A1F48006805
:10A7B000D0ED030A1D48006890ED021A00EE810AF0
:10A7C0001A48006880ED040A1848006890ED050AF0
:10A7D00016480068D0ED040AB4EEE00AF1EE10FA73
:10A7E00007D21248006890ED040A1048006880ED16
:10A7F000050A0E48006890ED050ADFED0F0AB4EE79
:10A80000E00AF1EE10FA05DB9FED0C0A074800683C
:10A8100080ED050A00BF00BF0448006890ED050AFE
:10A82000BDEC048B10BD00000000AF439040002041
:10A83000000000003333C6420000C842CDCCC742FE
:10A8400000007A4410B54FF496610348FBF722FEEE
:10A8500000200249087010BD404B0020D63D00206A
:10A8600070B50025002400BF50E004EB8401324A9B
:10A8700002EB81018868FDF7AFF904EB84002E49F3
:10A8800001EB8000007B00B93EE004EB84002A4924
:10A8900001EB8000806870B32848066804EB8400F0
:10A8A00001EB8000408838B904EB8401224A02EBB6
:10A8B0008101886880471DE001F03EFE04EB8401C1
:10A8C0001D4A02EB81014968401A04EB840102EB46
:10A8D0008101498888420DD301F02EFE04EB8401EA
:10A8E000154A02EB8101486004EB840102EB81010F
:10A8F0008868804700BF04EB84010F4A02EB8101A6
:10A900008868FDF7A7F900BF601CC4B20C48007846
:10A910008442AADB002408E004EB8400064911F815
:10A92000200000B10125601CC4B2054800788442B3
:10A93000F2DB284670BD0000404B002004B500400B
:10A94000D63D002030B50246002017E000EB800322
:10A950000D4C04EB83039B6893420DD100EB800305
:10A9600014F823308B4206D001F0010300EB800481
:10A97000054D05F8243030BD431CD8B2034B1B787D
:10A980009842E3DB00BFF6E7404B0020D63D0020B5
:10A990002DE9F04105460F461646002421E004EB60
:10A9A00084002E4901EB80008068B04217D101205D
:10A9B00004EB8401294A02EB8101087304EB840053
:10A9C000114601EB8000458001F0B6FD04EB8401E7
:10A9D000224A02EB810148600120BDE8F081601C41
:10A9E000C4B21F4800788442D9DB1D4800783C2857
:10A9F00002DB4FF0FF30F0E71948007800EB8000F1
:10AA0000164901EB8000866001201549097801EBA9
:10AA10008101124A02EB810108731148007800EBB2
:10AA20008000114601EB8000458001F085FD0C4956
:10AA3000097801EB8101094A02EB8101486008486D
:10AA4000007800EB8000114601EB800007610448AC
:10AA50000078401C024908700020BEE7404B0020EF
:10AA6000D63D002010B50146002015E000EB800225
:10AA70000C4B03EB820292688A420BD1002200EB5E
:10AA80008003084C04EB83031A7300EB800304F883
:10AA9000232010BD421CD0B2034A12789042E5DB5D
:10AAA00000BFF6E7404B0020D63D002010B502461F
:10AAB00000200FE000EB8003094C04EB83039B684C
:10AAC000934205D100EB800304EB8303598010BD52
:10AAD000431CD8B2034B1B789842EBDB00BFF6E770
:10AAE000404B0020D63D00202DE9F04105460320D3
:10AAF000FCF752FF0746052D01DABDE8F08100247E
:10AB000026E0174800EB04100078B8421FD1144823
:10AB100000EB0410C068D0B1002609E0311D88B2F6
:10AB2000FCF73AFF0E4901EB041149688855761C81
:10AB3000681FB042F2DC0A4901EB04110872084AAE
:10AB400002EB041002EB0412D168884704E0641C95
:10AB5000044800688442D4D300BF00BFCDE70000A2
:10AB60001059002040400020F0B5C1B00546032038
:10AB7000FCF722FF0746052F12DA002406E0211D0C
:10AB800088B2FCF719FF01A90855641C681FA04290
:10AB9000F5DCC3B201AA39460020FCF7DBFD00BF9B
:10ABA000052D01DA41B0F0BD002426E0164800EB87
:10ABB00004100078B8421FD1134800EB0410C0689D
:10ABC000D0B1002609E0311D88B2FCF7F5FE0E4930
:10ABD00001EB041149688855761C681FB042F2DC0D
:10ABE000094901EB04110872074A02EB041002EB59
:10ABF0000412D168884704E0641C04480068844259
:10AC0000D4D300BF00BFCDE7305F00205C40002000
:10AC100010B500F025F810BD2DE9F04107460C46AF
:10AC200015461E460848807A30B1002000F0ECFC42
:10AC300000F00EF8FFF7ECFF0448076084808560A1
:10AC4000C660BDE8F0810000084100209C7900202A
:10AC500010B5024815F0FCFC10BD000000410020BA
:10AC600070B50025084809490268094815F024FC18
:10AC7000044604B16D1E681C20B9064A06A10020D6
:10AC8000FFF786FE70BD000014410020084100203F
:10AC9000004100207D35030070776D5F696E697437
:10ACA0000000000010B5034A1068034A1168884785
:10ACB00010BD0000F84A0020F44A002010B504221C
:10ACC0000021024810F074FF10BD00000040024057
:10ACD0002DE9F0472DED068B86B005460E4617464A
:10ACE0004FF00008C146C246002005E035F91010BB
:10ACF00003AA42F82010401C0328F7DB059800281F
:10AD000001DB014600E041428846002004E036F9BC
:10AD100010104DF82010401C0328F8DB0298002882
:10AD200001DB014600E041428946ED4800780328F6
:10AD30000CDBEC484068EB490860084680684860D6
:10AD40000220E74908700120E7490860E4480178DB
:10AD50000078401CE24A1070E24840F82180E34845
:10AD6000007803280CDBE2484068E14908600846A7
:10AD7000806848600220DD4908700120DA490860D7
:10AD8000DA4801780078401CD84A1070D84840F85A
:10AD90002190D848007803280CDBD7484088D64952
:10ADA00008800846808848800220D2490870012027
:10ADB000CD490860B888404201B2CE480278007898
:10ADC000401CCC4B1870CC4820F81210C6480068C4
:10ADD00001287DD1C3488068C2494968401A12D40D
:10ADE000C648008820B9BF488068C549086011E09E
:10ADF000BC488068C249096888420BDDB948806850
:10AE0000BF49086006E0BD48008818B9B5488068A9
:10AE1000BC490860B6488068B5494968401A12D4F0
:10AE2000B948008820B9B2488068B849086011E084
:10AE3000AF488068B549096888420BDDAC48806836
:10AE4000B249086006E0B048008818B9A848806890
:10AE5000AF490860A3488068AA490968401A40F2CF
:10AE60004C41884212DD0120A44908809D48806839
:10AE7000A4490968401AA7490968884206DD99482B
:10AE80008068A0490968401AA2490860984880680B
:10AE90009F490968401A40F24C41884212DD012066
:10AEA000994908809248806899490968401A9A49E6
:10AEB0000968884206DD8E48806895490968401A0D
:10AEC00095490860874880688E490968401A00E003
:10AED000ECE040F2EE21884227DD8E480068FBF767
:10AEE0008EFC41EC1A0B9FED8D0B53EC102BFBF7F6
:10AEF000A5FB41EC180B7B498968814A1268501AFE
:10AF0000FBF77DFC41EC190B53EC182BFBF7F8FC1D
:10AF100012D27448806873494968441A002C01DBD6
:10AF2000204600E06042642806DA00207349088069
:10AF300040F24C40774908606D4880687449096860
:10AF4000401A40F2EE21884227DD73480068FBF783
:10AF500056FC41EC1A0B9FED710B53EC102BFBF7D9
:10AF60006DFB41EC180B62498968684A1268501AF7
:10AF7000FBF745FC41EC190B53EC182BFBF7C0FC1D
:10AF800012D25B4880685A494968441A002C01DB98
:10AF9000204600E06042642806DA00205A49088012
:10AFA00040F24C405C4908605648006810B90020E7
:10AFB000524908805648006810B90020524908805C
:10AFC0005848008838BB5848B0F90000B0F5967F63
:10AFD00005DA55480088401C00B25349088000201B
:10AFE0005249088045480088012803D04648008817
:10AFF00001280AD14C48B0F90000082805DB4FF0C1
:10B00000010A01204749088062E04FF0000A002051
:10B01000444908805CE04FF0000A4448B0F9000061
:10B02000B0F5967F05DA41480088401C00B23F49E0
:10B03000088000203C4908803C4BB3F90030062BC7
:10B0400030DB2E4B1B886BBB2B4BB3F90030A3F5C9
:10B05000FA62002A01DB134600E05342B3F5967F03
:10B0600019DC254BB3F90230A3F5FA61002901DBA5
:10B070000B4600E04B42B3F5967F0CDC1E4BB3F958
:10B080000430A3F5FA60002801DB034600E04342E8
:10B09000B3F5967F06DD1C4B1B881BB900202149A8
:10B0A000088015E001201F49088011E04FF0000AD8
:10B0B0000C488068134908600A4880681049086095
:10B0C0000B48806812490860094880680F49086089
:10B0D0000AF0FF0006B0BDEC068BBDE8F08700006B
:10B0E000404A00205C9200204C4A0020414A002047
:10B0F00068920020484A0020504A00202A4A002036
:10B10000344A0020304A00202C4A00203C4A0020CB
:10B11000384A0020584A00205C4A00209A999999A0
:10B120009999D93F464A0020444A0020424A0020CB
:10B13000FEB54FF4827014F063FE002837D04FF450
:10B14000827014F067FE6C4890F82E0018B16A48BF
:10B1500090F82F0058B300208DF800006648406832
:10B16000019065480189ADF80810C06818B9002041
:10B170006149087412E06048008B5F4948830846C3
:10B18000C06848600846008B08810020C8600846F7
:10B1900090F82E0010B9002014F05EFE56480168A9
:10B1A000684688470020544981F82F0000BF524864
:10B1B00090F82E00002852D04FF4807014F020FE3A
:10B1C00000284CD04FF4807014F024FE4A48408B85
:10B1D000494991F82D10884216DD4748408B464971
:10B1E00091F82D10401A444948830A4612890B46AB
:10B1F0005B8BD21A0B465B6803EB42000A4692F85F
:10B200002D1014F0E9FD23E03B48408B3A4991F8BA
:10B210002D1088420FD13848C06860B101203649EE
:10B2200081F82F00002048830A4692F82D10D0683C
:10B2300014F0D2FD0CE03048408B2F4991F82D10CE
:10B24000884205D101202C4981F82F000020488335
:10B250004FF4827014F0DEFD042014F0FDFD4FF475
:10B26000887014F0CDFD70B14FF4887014F0D2FDE9
:10B2700000202149087402208DF80000084601686A
:10B280006846884700BF4FF48A7014F0B9FD38B1A2
:10B290004FF48A7014F0BEFD0020174908742AE0AC
:10B2A0001548456924E0B5FA85F64FF00040F040B6
:10B2B0008543B00000F58C74204614F0A1FDB8B1B0
:10B2C000204614F0A7FD01208DF80000A4F58C7035
:10B2D000C0F3C7008DF80400A4F58C70012121EAA9
:10B2E00090018DF80510044801686846884700BF42
:10B2F000002DD8D100BFFEBD7C9300200246002166
:10B3000006E00548405C904201D100207047491C8E
:10B310000029F6D00220F9E7486A040070B5054616
:10B320000C462846FFF7EAFF061E01D0304670BDE6
:10B33000012C04D10121284614F030FA04E01CB994
:10B340000021284614F02AFA0020F0E710B5002466
:10B3500009E00D49085D0121FFF7E0FF0A49085D9A
:10B3600014F0B7F8641C002CF3D0084813F0E3FF86
:10B37000032014F0AEF8042014F0ABF8052014F00C
:10B38000A8F8002010BD0000486A0400186A0400F4
:10B390007FB50025174B0FCB8DE80F0003208DF8EC
:10B3A000020004208DF8010005208DF80000002027
:10B3B0008DF80C004FF00040029006208DF804003C
:10B3C00000230D4A69460D4813F058FF064606B1A2
:10B3D0006D1E002404E00A49085D14F092F8641C14
:10B3E000002CF8D0681C20B9064A07A10020FFF7FE
:10B3F000CFFA7FBD4C6A0400855F0400186A040020
:10B40000486A04000D360300737069305F696E6925
:10B4100074000000F8B506460F4614461D46234644
:10B42000002239463046009500F04EF8F8BDF8B5D8
:10B4300006460F4614461D4623460122394630462D
:10B44000009500F041F8F8BD2DE9F84F05460E468D
:10B4500017469846DDF8289042F2107A2846FFF702
:10B460004DFF041E02D02046BDE8F88F002128467B
:10B47000FFF754FF00201249087043463A46314610
:10B480001048CDF8009013F03DFF04460CB10120A8
:10B49000EAE70AE0BAF10000AAF1010A05D10121A8
:10B4A0002846FFF73BFF0120DEE70548007800282B
:10B4B000F0D001212846FFF731FF0020D4E700003B
:10B4C00072410020186A04002DE9FC4781460D46B0
:10B4D00090461E460A9C4846FFF710FF071E02D002
:10B4E0003846BDE8FC87812C01D90320F9E7B8F183
:10B4F000000F16D145F080000190601CC0B2144BC3
:10B50000012201A900904846FFF79EFF07460FB1B0
:10B510003846E6E722460E49491C3046FAF7A1FFB5
:10B5200013E00B48057022463146401CFAF799FF9C
:10B5300000200090601CC2B2002305494846FFF776
:10B5400083FF07460FB13846CBE70020C9E700006C
:10B55000147A002010B50249024810F0D7FB10BD44
:10B56000C49300200030004010B503494FF0402044
:10B5700010F0CCFB10BD0000E893002010B502498C
:10B58000024810F0C3FB10BD0C94002000300240B4
:10B5900070B50A4813F08FFD044600BF254635B14B
:10B5A00000BF07A262212846FAF734FE00BF00BFA1
:10B5B0000CB1062070BD0020FCE700006880002070
:10B5C0002E2E5C2E2E5C2E2E5C626C655F63666791
:10B5D0005C686F73742E630010B513F094FD10BD9A
:10B5E00010B514F059FD10BD0149487170470000B5
:10B5F0000841002030B5034D28706970AA70EB70C7
:10B6000030BD0000084100200149887270470000E9
:10B6100008410020014908817047000008410020CE
:10B6200070B504460D46164633462A462146024862
:10B6300014F0CCFF70BD00000041002001480078EC
:10B64000704700000542002010B500240BE00848B8
:10B6500050F8240028B1064850F824104FF47A70AE
:10B660008847601CC4B2034800788442EFDB10BDF9
:10B67000144B0020D43D00200246002117E00E4864
:10B6800050F82100904202D14FF0FF3070470A4835
:10B6900050F8210048B909480078401C074B187041
:10B6A000054840F821200020F0E7481CC1B20529D8
:10B6B000E5DB6FF00100E9E7144B0020D43D0020EA
:10B6C00002460020002100BF27E0411C22E000EBE1
:10B6D000C0030B4402EB8303D3ED000A01EBC1036B
:10B6E000034402EB830393ED001A70EE810AB6EE79
:10B6F000001A20EE810A00EBC0030B4402EB830327
:10B7000083ED000A01EBC103034402EB830383EDE5
:10B71000000A491C0929DADB401C0928D5DB7047DF
:10B7200090ED031AD0ED061A01EE801A80ED031A8F
:10B7300090ED041AD0ED071A01EE801A80ED041A7C
:10B7400090ED051AD0ED081A01EE801A80ED051A69
:10B7500090ED0C1AD0ED0F1A01EE801A80ED0C1A44
:10B7600090ED0D1AD0ED101A01EE801A80ED0D1A31
:10B7700090ED0E1AD0ED111A01EE801A80ED0E1A1E
:10B7800090ED151AD0ED181A01EE801A80ED151AF9
:10B7900090ED161AD0ED191A01EE801A80ED161AE6
:10B7A00090ED171AD0ED1A1A01EE801A80ED171AD3
:10B7B00090ED1B1AD0ED361A01EE801A80ED1B1A9F
:10B7C00090ED1C1AD0ED371A01EE801A80ED1C1A8C
:10B7D00090ED1D1AD0ED381A01EE801A80ED1D1A79
:10B7E00090ED241AD0ED3F1A01EE801A80ED241A54
:10B7F00090ED251AD0ED401A01EE801A80ED251A41
:10B8000090ED261AD0ED411A01EE801A80ED261A2D
:10B8100090ED2D1AD0ED481A01EE801A80ED2D1A08
:10B8200090ED2E1AD0ED491A01EE801A80ED2E1AF5
:10B8300090ED2F1AD0ED4A1A01EE801A80ED2F1AE2
:10B8400090ED1E1AD0ED391A01EE801AD0ED211AB2
:10B8500090ED3C2A42EE001A00EE211A80ED1E1AED
:10B8600090ED1F1AD0ED3A1A01EE801AD0ED221A8F
:10B8700090ED3D2A42EE001A00EE211A80ED1F1ACB
:10B8800090ED201AD0ED3B1A01EE801AD0ED231A6C
:10B8900090ED3E2A42EE001A00EE211A80ED201AA9
:10B8A00090ED271AD0ED421A01EE801AD0ED2A1A37
:10B8B00090ED452A42EE001A00EE211A80ED271A7B
:10B8C00090ED281AD0ED431A01EE801AD0ED2B1A14
:10B8D00090ED462A42EE001A00EE211A80ED281A59
:10B8E00090ED291AD0ED441A01EE801AD0ED2C1AF1
:10B8F00090ED472A42EE001A00EE211A80ED291A37
:10B9000090ED301AD0ED4B1A01EE801AD0ED331ABB
:10B9100090ED4E2A42EE001A00EE211A80ED301A08
:10B9200090ED311AD0ED4C1A01EE801AD0ED341A98
:10B9300090ED4F2A42EE001A00EE211A80ED311AE6
:10B9400090ED321AD0ED4D1A01EE801AD0ED351A75
:10B9500090ED502A42EE001A00EE211A80ED321AC4
:10B9600090ED211AD0ED3C1A01EE801AD1ED021AA9
:10B9700061EE801A90ED1C2A01EE821AD1ED011AB7
:10B9800061EE801A90ED1D2A01EEC21A80ED211A97
:10B9900090ED221AD0ED3D1A01EE801AD1ED021A77
:10B9A00061EE801A90ED1B2A01EEC21AD1ED001A49
:10B9B00061EE801A90ED1D2A01EE821A80ED221AA6
:10B9C00090ED231AD0ED3E1A01EE801AD1ED011A46
:10B9D00061EE801A90ED1B2A01EE821AD1ED001A59
:10B9E00061EE801A90ED1C2A01EEC21A80ED231A36
:10B9F00090ED2A1AD0ED451A01EE801AD1ED021A07
:10BA000061EE801A90ED252A01EE821AD1ED011A1D
:10BA100061EE801A90ED262A01EEC21A80ED2A1AF4
:10BA200090ED2B1AD0ED461A01EE801AD1ED021AD4
:10BA300061EE801A90ED242A01EEC21AD1ED001AAF
:10BA400061EE801A90ED262A01EE821A80ED2B1A03
:10BA500090ED2C1AD0ED471A01EE801AD1ED011AA3
:10BA600061EE801A90ED242A01EE821AD1ED001ABF
:10BA700061EE801A90ED252A01EEC21A80ED2C1A93
:10BA800090ED331AD0ED4E1A01EE801AD1ED021A64
:10BA900061EE801A90ED2E2A01EE821AD1ED011A84
:10BAA00061EE801A90ED2F2A01EEC21A80ED331A52
:10BAB00090ED341AD0ED4F1A01EE801AD1ED021A32
:10BAC00061EE801A90ED2D2A01EEC21AD1ED001A16
:10BAD00061EE801A90ED2F2A01EE821A80ED341A61
:10BAE00090ED351AD0ED501A01EE801AD1ED011A01
:10BAF00061EE801A90ED2D2A01EE821AD1ED001A26
:10BB000061EE801A90ED2E2A01EEC21A80ED351AF0
:10BB100090ED091AD1ED021A61EE211A90ED361A54
:10BB200001EE801AD0ED121A91ED012A61EE821A0F
:10BB300001EEC01A80ED361A90ED0A1AD1ED021A04
:10BB400061EE211A90ED371A01EE801AD0ED131A2A
:10BB500091ED012A61EE821A01EEC01A80ED371ACA
:10BB600090ED0B1AD1ED021A61EE211A90ED381A00
:10BB700001EE801AD0ED141A91ED012A61EE821ABD
:10BB800001EEC01A80ED381A90ED001AD1ED021ABC
:10BB900061EE211A90ED3F1A01EEC01AD0ED121A93
:10BBA00091ED002A61EE821A01EE801A80ED3F1AB3
:10BBB00090ED011AD1ED021A61EE211A90ED401AB2
:10BBC00001EEC01AD0ED131A91ED002A61EE821A2F
:10BBD00001EE801A80ED401A90ED021AD1ED021AA2
:10BBE00061EE211A90ED411A01EEC01AD0ED141A3F
:10BBF00091ED002A61EE821A01EE801A80ED411A61
:10BC000090ED001AD1ED011A61EE211A90ED481A5B
:10BC100001EE801AD0ED091A91ED002A61EE821A28
:10BC200001EEC01A80ED481A90ED011AD1ED011A0B
:10BC300061EE211A90ED491A01EE801AD0ED0A1A30
:10BC400091ED002A61EE821A01EEC01A80ED491AC8
:10BC500090ED021AD1ED011A61EE211A90ED4A1A07
:10BC600001EE801AD0ED0B1A91ED002A61EE821AD6
:10BC700001EEC01A80ED4A1A90ED391AD0ED3C1A47
:10BC800000EE211AD0ED0C1A91ED022A61EE821A13
:10BC900001EE801AD0ED151A91ED012A61EE821A9B
:10BCA00001EEC01A80ED391A90ED3A1AD0ED3D1A26
:10BCB00000EE211AD0ED0D1A91ED022A61EE821AE2
:10BCC00001EE801AD0ED161A91ED012A61EE821A6A
:10BCD00001EEC01A80ED3A1A90ED3B1AD0ED3E1AF3
:10BCE00000EE211AD0ED0E1A91ED022A61EE821AB1
:10BCF00001EE801AD0ED171A91ED012A61EE821A39
:10BD000001EEC01A80ED3B1A90ED421AD0ED451AB3
:10BD100000EE211AD0ED031A91ED022A61EE821A8B
:10BD200001EEC01AD0ED151A91ED002A61EE821ACB
:10BD300001EE801A80ED421A90ED431AD0ED461ABA
:10BD400000EE211AD0ED041A91ED022A61EE821A5A
:10BD500001EEC01AD0ED161A91ED002A61EE821A9A
:10BD600001EE801A80ED431A90ED441AD0ED471A87
:10BD700000EE211AD0ED051A91ED022A61EE821A29
:10BD800001EEC01AD0ED171A91ED002A61EE821A69
:10BD900001EE801A80ED441A90ED4B1AD0ED4E1A48
:10BDA00000EE211AD0ED031A91ED012A61EE821AFC
:10BDB00001EE801AD0ED0C1A91ED002A61EE821A84
:10BDC00001EEC01A80ED4B1A90ED4C1AD0ED4F1ACF
:10BDD00000EE211AD0ED041A91ED012A61EE821ACB
:10BDE00001EE801AD0ED0D1A91ED002A61EE821A53
:10BDF00001EEC01A80ED4C1A90ED4D1AD0ED501A9C
:10BE000000EE211AD0ED051A91ED012A61EE821A99
:10BE100001EE801AD0ED0E1A91ED002A61EE821A21
:10BE200001EEC01A80ED4D1A90ED0F1AD1ED021AF5
:10BE300061EE211A90ED3C1A01EE801AD0ED181A2D
:10BE400091ED012A61EE821A01EEC01AD1ED021ABB
:10BE500061EE801A90ED372A01EE821AD1ED011AB7
:10BE600061EE801A90ED382A01EEC21A80ED3C1A7C
:10BE700090ED101AD1ED021A61EE211A90ED3D1AE3
:10BE800001EE801AD0ED191A91ED012A61EE821AA5
:10BE900001EEC01AD1ED021A61EE801A90ED362A39
:10BEA00001EEC21AD1ED001A61EE801A90ED382A27
:10BEB00001EE821A80ED3D1A90ED111AD1ED021AB1
:10BEC00061EE211A90ED3E1A01EE801AD0ED1A1A99
:10BED00091ED012A61EE821A01EEC01AD1ED011A2C
:10BEE00061EE801A90ED362A01EE821AD1ED001A29
:10BEF00061EE801A90ED372A01EEC21A80ED3E1AEB
:10BF000090ED061AD1ED021A61EE211A90ED451A54
:10BF100001EEC01AD0ED181A91ED002A61EE821AD6
:10BF200001EE801AD1ED021A61EE801A90ED402ADE
:10BF300001EE821AD1ED011A61EE801A90ED412ACC
:10BF400001EEC21A80ED451A90ED071AD1ED021AE2
:10BF500061EE211A90ED461A01EEC01AD0ED191AC1
:10BF600091ED002A61EE821A01EE801AD1ED021ADB
:10BF700061EE801A90ED3F2A01EEC21AD1ED001A4F
:10BF800061EE801A90ED412A01EE821A80ED461A88
:10BF900090ED081AD1ED021A61EE211A90ED471AC0
:10BFA00001EEC01AD0ED1A1A91ED002A61EE821A44
:10BFB00001EE801AD1ED011A61EE801A90ED3F2A50
:10BFC00001EE821AD1ED001A61EE801A90ED402A3E
:10BFD00001EEC21A80ED471A90ED061AD1ED011A52
:10BFE00061EE211A90ED4E1A01EE801AD0ED0F1A73
:10BFF00091ED002A61EE821A01EEC01AD1ED021A0B
:10C0000061EE801A90ED492A01EE821AD1ED011AF3
:10C0100061EE801A90ED4A2A01EEC21A80ED4E1AA6
:10C0200090ED071AD1ED011A61EE211A90ED4F1A29
:10C0300001EE801AD0ED101A91ED002A61EE821AFD
:10C0400001EEC01AD1ED021A61EE801A90ED482A75
:10C0500001EEC21AD1ED001A61EE801A90ED4A2A63
:10C0600001EE821A80ED4F1A90ED081AD1ED011AF7
:10C0700061EE211A90ED501A01EE801AD0ED111ADE
:10C0800091ED002A61EE821A01EEC01AD1ED011A7B
:10C0900061EE801A90ED482A01EE821AD1ED001A65
:10C0A00061EE801A90ED492A01EEC21A80ED501A15
:10C0B00090ED011AD1ED021A61EE211A90ED061AE7
:10C0C00001EE801AD0ED021A91ED012A61EE821A7A
:10C0D00001EEC01A80ED061A90ED001AD1ED021A99
:10C0E00061EE211A90ED071A01EEC01AD0ED021A86
:10C0F00091ED002A61EE821A01EE801A80ED071A96
:10C1000090ED001AD1ED011A61EE211A90ED081A96
:10C1100001EE801AD0ED011A91ED002A61EE821A2B
:10C1200001EEC01A80ED081A90ED0A1AD1ED021A3C
:10C1300061EE211A90ED0F1A01EE801AD0ED0B1A64
:10C1400091ED012A61EE821A01EEC01A80ED0F1AFC
:10C1500090ED091AD1ED021A61EE211A90ED101A34
:10C1600001EEC01AD0ED0B1A91ED002A61EE821A91
:10C1700001EE801A80ED101A90ED091AD1ED011A26
:10C1800061EE211A90ED111A01EE801AD0ED0A1A13
:10C1900091ED002A61EE821A01EEC01A80ED111AAB
:10C1A00090ED131AD1ED021A61EE211A90ED181AD2
:10C1B00001EE801AD0ED141A91ED012A61EE821A77
:10C1C00001EEC01A80ED181A90ED121AD1ED021A84
:10C1D00061EE211A90ED191A01EEC01AD0ED141A71
:10C1E00091ED002A61EE821A01EE801A80ED191A93
:10C1F00090ED121AD1ED011A61EE211A90ED1A1A82
:10C2000001EE801AD0ED131A91ED002A61EE821A28
:10C2100001EEC01A80ED1A1A9FED191A20EE011ACC
:10C2200061EE000A002210E002EBC203134400EBAF
:10C23000830393ED001A31EE201A02EBC20313447C
:10C2400000EB830383ED001A521C032AECDB062269
:10C2500012E002EBC203134400EB830393ED001AD8
:10C26000DFED081A00EEA11A02EBC203134400EB43
:10C27000830383ED001A521C092AEADB7047000091
:10C2800017B7D1380000C84201480249086070471A
:10C290000090D0030C4B002010B512F0EDF828B13F
:10C2A00095480088C0F304209449086012F03CF9D6
:10C2B00010B193489349486712F072F930B18E4833
:10C2C000E0380068C0F342308F49086012F094F9FA
:10C2D00028B18E48006820F080708C49086012F008
:10C2E000A9F948B100208A4908604FF08041C1F89F
:10C2F00010018549091F086012F0C8F918B1032020
:10C3000081496431086012F0DFF968B10520814984
:10C31000086001207F497831086000207D4908319C
:10C3200008603F20091F086012F0ECF9002855D082
:10C330007148E0300068784908606F48E430006870
:10C34000091D08606C48E8300068091D08606A48EB
:10C35000EC300068091D08606748F0300068091D6E
:10C3600008606548F4300068091D08606248F830CC
:10C3700000686949203108605F48FC300068091D89
:10C38000086066480068091D08606448001D006870
:10C39000091D0860614808300068091D08605F4891
:10C3A0000C300068091D08605C48103000685A496C
:10C3B00040310860594814300068091D086057482A
:10C3C00018300068091D086054481C300068091DB9
:10C3D0000860524820300068091D086012F020F8FB
:10C3E00030B14548CC38006800F04F004C49086037
:10C3F00012F06EF840B14B48006800F0010018B12F
:10C400006FF001004749086012F0ACF828B14648C7
:10C41000006840F48060444908603C487438006813
:10C4200040F4700039497439086000BF00BF00BF94
:10C43000BFF34F8F00BF00BF00BF00BF00BF00BFF2
:10C44000BFF36F8F00BF00BF00BF3848006800F027
:10C450000100F0B101203649086000BF354800688E
:10C460000028FBD03148006820F001004FF0102177
:10C47000C1F80C0200BF2F4800680028FBD0002044
:10C480002B49086000BF2B4800680028FBD000F053
:10C4900071FB26480C38006800F0004028B923489A
:10C4A0000838006800F0004018B3012020490860F7
:10C4B00000BF204800680028FBD015201B490C391C
:10C4C000086000BF1B4800680028FBD015211748F2
:10C4D0000838016000BF174800680028FBD0002022
:10C4E0001349086000BF134800680028FBD000F023
:10C4F00041FBFFF7C9FE10BD240300104035014089
:10C500000DF0ADBA00C007403C050040FCED00E076
:10C510000C0100401056004020C5004024040010CB
:10C52000E40E0040000400403C1700400C120010D4
:10C5300004E5014000E40140014800687047000044
:10C54000FC4000207CB500251B4903C9CDE9000152
:10C5500002208DF802000020ADF80000174A69465D
:10C56000174814F01DF9044604B16D1E0123212261
:10C570000021134814F0A0F8044664B101232122DD
:10C5800000210F4814F098F8044624B10D4A0EA17A
:10C590000020FEF7FDF90A4814F0E6F8084814F008
:10C5A000EFF80C4800F03EFA681C20B90A4A0BA1CB
:10C5B0000020FEF7EDF97CBDF0690400713C040039
:10C5C000E8690400AD3503007274635F636F6E66E3
:10C5D00069670000414A0300DD3503007274635F40
:10C5E000696E6974000000000246002112E00C48E8
:10C5F00050F82100904202D16FF0010070470848C6
:10C6000050F8210020B9064840F821200020F5E725
:10C61000481CC1B20A29EADB4FF0FF30EEE7000008
:10C620006479002010B503460021002214E00D4873
:10C6300050F8220098420DD1114607E0094C481CE1
:10C6400054F8200044F82100481CC1B20929F5DB48
:10C65000002010BD501CC2B20A2AE8DB4FF0FF30A8
:10C66000F7E700006479002010B5FFF76BFF0BF0CF
:10C6700003FF06F001FB0DF05DFEFAF701FDFAF78E
:10C68000BDFE0EF03BF80DF05DFF0DF0CFFE03F0A8
:10C690005FFD03F02FF804F0BDF804F00FFB02F08B
:10C6A0002BFF04F097FD03F0EFFE04F073F904F0A4
:10C6B00089F903F08FFC04F009FF03F0D3FC04F0C8
:10C6C0009DFC02F027FC04F0D9F804F017FB19F0E8
:10C6D000DFFF0BF0F9FD10BD10B5FEF7C1F850B942
:10C6E000FEF7B2FF0EF0AAF9044617F015FA034957
:10C6F000086000F07DF9FBF7E1FC10BDD03D0020A3
:10C70000B0EE401A81EE200ADFED021A20EE210A77
:10C71000704700000000C84210B52DED048BB0EE4C
:10C72000408A9FED260AB0EE409A9FED240AF0EE73
:10C73000408A2348006890F8230060B1B2EE040AF2
:10C74000C8EE000A1E480068C0ED000A00201C491F
:10C75000096881F82300B2EE040AC8EE000AF0EE80
:10C76000609A17480068DFED170AB0EE690A0BF00F
:10C77000BBFDF0EE408A9FED140AF4EEC08AF1EEA4
:10C7800010FA04D29FED0D0AB0EE409A11E09FED31
:10C790000F0AF4EEC08AF1EE10FA04DD9FED0C0AE8
:10C7A000B0EE409A05E0B0EE680A0EF073FEB0EE0F
:10C7B000409AB0EE490ABDEC048B10BD00000000A9
:10C7C000904000200AD7233C0000A0430000D24341
:10C7D0000000C84208B500BF4FF480700B494058B4
:10C7E00008B1012000E0002078B1094800688047C6
:10C7F00000BF00204FF48071044A8850084611465B
:10C800004058009000BF00BF00BF08BD00000140BD
:10C81000C04A00202DE9F0410246C2F30744C2F3AA
:10C820000726D5B2802300200021CCE0880006EA4C
:10C830000307D7B1664F3F88DFF898C12CF8107016
:10C84000634FB7F802C0DFF88C81471C28F817C087
:10C850005F4FB7F804C0871C28F817C05C4FB7F8C3
:10C8600006C0C71C28F817C019E05B4F3F88DFF8E7
:10C8700064C12CF81070584FB7F802C0DFF854812B
:10C88000471C28F817C0544FB7F804C0871C28F875
:10C8900017C0514FB7F806C0C71C28F817C088004A
:10C8A00004EA030717B34A4FB7F800C0494F4037AF
:10C8B00027F810C0464FB7F80280464F403700F1C6
:10C8C000010C27F81C80424FB7F80480414F4037D5
:10C8D00000F1020C27F81C803D4FB7F806803D4F51
:10C8E000403700F1030C27F81C8021E03A4FB7F8DD
:10C8F00000C0384F403727F810C0374FB7F80280D4
:10C90000344F403700F1010C27F81C80324FB7F844
:10C910000480304F403700F1020C27F81C802E4F66
:10C92000B7F806802B4F403700F1030C27F81C8026
:10C93000880005EA030717B3254FB7F800C0254F55
:10C94000803727F810C0224FB7F80280214F803778
:10C9500000F1010C27F81C801D4FB7F804801D4F13
:10C96000803700F1020C27F81C80194FB7F80680B9
:10C97000184F803700F1030C27F81C8021E0164F78
:10C98000B7F800C0134F803727F810C0124FB7F820
:10C990000280104F803700F1010C27F81C800E4FE9
:10C9A000B7F804800B4F803700F1020C27F81C8089
:10C9B000094FB7F80680074F803700F1030C27F8BE
:10C9C0001C805B08491C0829FFF630AFBDE8F081E8
:10C9D000D86904009C710020E069040010B50122B0
:10C9E000042102480068FEF71BFE10BDB040002085
:10C9F00010B500240BE0084850F8240028B1064880
:10CA000050F82410054800688847601CC4B20448E8
:10CA100000788442EFDB10BD284B0020D03D002081
:10CA2000D53D00200246002117E00E4850F82100B5
:10CA3000904202D14FF0FF3070470A4850F8210071
:10CA400048B909480078401C074B1870054840F861
:10CA500021200020F0E7481CC1B20629E5DB6FF079
:10CA60000100E9E7284B0020D53D002010B50BF070
:10CA70002BFC10BD0FB4084B10B504A902AA0398F3
:10CA800001F0CAFC044602A9002002F05CF820462E
:10CA900010BC5DF814FB000047EB020003B40198E2
:10CAA0004100009850EAC12018BF04204A0D18BF69
:10CAB00040F0010040F2FF72B2EB515F08BF40F05E
:10CAC0000200012808BF052002B07047410008029B
:10CAD00018BF04200A0E18BF40F001004FF07F423B
:10CAE00032EA010108BF40F00200012808BF05201A
:10CAF0007047000000BF00BF00BFBFF34F8F00BFF3
:10CB000000BF00BF0948006800F4E060084908431E
:10CB1000001D0649086000BF00BF00BFBFF34F8F74
:10CB200000BF00BF00BF00BF00BFFDE70CED00E08D
:10CB30000000FA0500BF00BF00BFBFF34F8F00BF6A
:10CB400000BF00BF0948006800F4E06008490843DE
:10CB5000001D0649086000BF00BF00BFBFF34F8F34
:10CB600000BF00BF00BF00BF00BFFDE70CED00E04D
:10CB70000000FA0500BF00BF00BFBFF34F8F00BF2A
:10CB800000BF00BF0948006800F4E060084908439E
:10CB9000001D0649086000BF00BF00BFBFF34F8FF4
:10CBA00000BF00BF00BF00BF00BFFDE70CED00E00D
:10CBB0000000FA050000000070B5C1482DED020B21
:10CBC0002DED0E8B82B0119D25F000449FEDBEDB54
:10CBD0009FEDBFEB84423EDBA4F140511098A1F1E0
:10CBE0007F6108430FD0BC48844202DC28D11098F2
:10CBF00030B39DED100B02B0BDEC0E8B02B0BDE862
:10CC0000704001F0C5BA9DED100B53EC1D2B51EC9B
:10CC1000100BF9F713FD9DED100B41EC180B53ECC5
:10CC20001E2B51EC100BF9F709FD53EC182BF9F7FB
:10CC30005EFC41EC100B02B0BDEC0E8B02B070BD7F
:10CC4000012001F021FB02B0BDEC0E8B02B0BDE86B
:10CC5000704001F0B1BAA1489FEDA18B844256DA31
:10CC60009DED100BB4F1795F0ADA51EC100BFFF770
:10CC700015FF042808BF01F0AFFA9DED100BDAE7AD
:10CC800053EC102B51EC100BF9F7D8FC41EC190BBD
:10CC900095480621B0EE490AF0EE690A784401F0A1
:10CCA00063F953EC192B51EC100BF9F7C7FC41EC6D
:10CCB0001A0B8E48B0EE490AF0EE690A0421784456
:10CCC00001F052F953EC192B51EC100BF9F7B6FCAB
:10CCD00053EC182BF9F70BFC41EC100B51EC1A0B31
:10CCE00053EC102BF9F71CFDCDE900019DED000B75
:10CCF00053EC102B9DED100B51EC100BF9F79EFC33
:10CD00009DED101B53EC112BF9F7F1FBD2E09DEDDB
:10CD1000100B51EC100B0BF049FA53EC182BF9F7F0
:10CD20008AFC9FED730BCDE9000153EC102B9DEDB8
:10CD3000000B51EC100BF9F781FC41EC190B6E481C
:10CD40000621B0EE490AF0EE690A784401F00CF9C8
:10CD500053EC192B51EC100BF9F770FC41EC1B0B49
:10CD60006648B0EE490AF0EE690A0421784401F001
:10CD7000FBF853EC192B51EC100BF9F75FFC53EC5B
:10CD8000182BF9F7B4FB41EC1C0B51EC190B19F003
:10CD9000A7F941EC180B5A489FED5BABA04222DC8F
:10CDA00053EC1C2B51EC1B0BF9F7BAFCCDE900013D
:10CDB0009DED000B51EC180B53EC102BF9F73EFCDA
:10CDC00053EC182BF9F793FB53EC1A2BF9F736FCBD
:10CDD00053EC1D2BF9F72CFC53EC1E2BF9F72BFC15
:10CDE00041EC100B5FE08DED008B002000909DED7D
:10CDF000000B51EC180B53EC102BF9F778FB9DED61
:10CE0000000B41EC1E0B53EC102B51EC100BF9F7FF
:10CE100015FC53EC192BF9F70EFC53EC1E2BF9F70C
:10CE20007FFC41EC190B53EC1C2B51EC1B0BF9F75D
:10CE300077FC41EC1B0B53EC1A2B51EC190BF9F757
:10CE4000FDFB53EC1D2BF9F7F6FB41EC190B53ECF2
:10CE50001A2B51EC180BF9F7F1FB53EC1B2BF9F7DC
:10CE6000EDFB53EC192BF9F7E3FB9DED000B41ECC7
:10CE7000180B53EC1A2B51EC100BF9F7DFFB9FED5D
:10CE8000249B53EC192BF9F7D6FB41EC100B51EC1A
:10CE9000180B53EC102BF9F7CBFB53EC192BF9F7CC
:10CEA000CAFB41EC100B002D3FF7C5AE51EC100B47
:10CEB00081F0004141EC100BBDE6000000000000D5
:10CEC0000000F03F00000000075C143326A6913CF0
:10CED000182D4454FB21F93F0000F07F0000E03F93
:10CEE000000000000000F03F08A1010016A10100B1
:10CEF000000000000000E03F5AA0010068A001000F
:10CF00003333EF3F0000000000000000000000404D
:10CF1000182D4454FB21E93F10B54FF00E402DED84
:10CF2000028BB0EE408A18EE104A00EB4400B0F1DC
:10CF3000506F4AD84FF0FC40B0EB440F22D2B0EE15
:10CF4000C80AF7EE000A30EEC00AF6EE000A60EEFC
:10CF5000208A18EE900A19F0FAF801EE100A14F07F
:10CF6000004F1DBFDFED2D0A9FED2D0AB1EE411AD6
:10CF7000DFED2C0A08BF9FED2C0AF8EE001A21EE17
:10CF8000218A05E0DFED290A68EE088AB0EE600A22
:10CF90009FED271ADFED271A30EE080A48EE811AB6
:10CFA0009FED251A08EEA11ADFED241A48EE811A2A
:10CFB0009FED231A08EEA11A68EE281ABDEC028B29
:10CFC00001EE810A30EE200A10BD4FF0E440B0EBD4
:10CFD000440F0CD918EE100AFFF778FD042808BF9B
:10CFE00001F018F9B0EE480ABDEC028B10BD4FF00D
:10CFF0007F40B0EB440F07D2B0EE480ABDEC028B85
:10D00000BDE8104001F0F8B8012001F03DF9BDEC99
:10D01000028BBDE8104001F0F5B800000000C9BF68
:10D0200022AAFDB90000C93F22AAFD390000000074
:10D0300024FE1C3DC78AD83C1E67383D1B93993D92
:10D04000AFAA2A3E0000000070B59B482DED020BF0
:10D050002DED068B079D25F00044A04218DC974873
:10D06000844202DC0AD1069840B19DED060BBDEC6E
:10D07000068B02B0BDE8704001F08AB8002DCCBF2D
:10D080009FED8F0B9FED900BBDEC068B02B070BD3A
:10D090008F48A04215DD8F48A042D8BF4FF0FF3423
:10D0A00058DD9DED060B51EC100BFFF7F7FC042843
:10D0B00008BF01F091F89DED060BBDEC068B02B0A8
:10D0C00070BD9DED060B51EC100B0BF06FF8CDE928
:10D0D000060181489FED828BA0423CDD8248A04240
:10D0E0001FDD00249FED82AB9DED060B53EC1A2B48
:10D0F00051EC100BF9F7FBF99DED060B41EC190B08
:10D1000053EC1A2B51EC100BF9F798FA53EC182B3F
:10D11000F9F78EFA53EC192BF9F702FBCDE906016A
:10D1200049E09DED060B012453EC182B51EC100B3C
:10D13000F9F7DDF99DED060B41EC190B53EC182BBB
:10D1400051EC100BF9F774FA53EC192BF9F7E8FAD4
:10D15000CDE906012FE06848A0421FDD02249FEDC3
:10D16000689B9DED060B53EC192B51EC100BF9F756
:10D1700065FA53EC182BF9F7BAF99DED060B41EC63
:10D18000180B53EC192B51EC100BF9F751FA53EC27
:10D19000182BF9F7C5FACDE906010CE09DED060B59
:10D1A000032453EC102B9FED580B51EC100BF9F7A7
:10D1B000B7FACDE906019DED060B53EC102B51ECAF
:10D1C000100BF9F73BFA41EC180B53EC182BF9F75D
:10D1D00035FA41EC190B4E480621B0EE490AF0EE43
:10D1E000690A784400F0C0FE53EC182B51EC100B88
:10D1F000F9F724FA41EC180B4648B0EE490AF0EE74
:10D20000690A0521784400F0AFFE53EC192B51EC6C
:10D21000100BF9F713FA41EC100B51EC180B53EC0F
:10D22000102B002C0EDAF9F762F99DED061B53EC7A
:10D23000112BF9F703FA9DED061B53EC112BF9F7AF
:10D24000FAF935E0F9F753F99DED061B53EC112B74
:10D25000F9F7F4F941EC100B2F48784400EBC400C7
:10D2600090ED001B51EC100B53EC112BF9F7E0F98A
:10D270009DED061B53EC112BF9F7DAF941EC100B7D
:10D280002648784400EBC40090ED001B51EC100BD5
:10D2900053EC112BF9F7CFF941EC100B002DA2BF85
:10D2A000BDEC068B02B070BD51EC100B81F000415B
:10D2B00041EC100B01E70000000010440000F07F7B
:10D2C000182D4454FB21F93F182D4454FB21F9BF7C
:10D2D0000000DC3F0000203E0000F33F00000000A3
:10D2E000000000000000F03F0000E63F00000000EA
:10D2F000000000000000004000800340000000002B
:10D30000000000000000F83F000000000000F0BF37
:10D310007A9C0100309C0100BA9B0100729B0100C5
:10D3200070B56B4E2DED040B2DED028B82B0DDF848
:10D330001CC0DDE905235C422CF000411C4341EA9E
:10D34000D474049D22F00040B44205D86C422C43B2
:10D3500040EAD474B4420BD99DED061B9DED040B3D
:10D3600002B0BDEC028B04B0BDE8704000F01ABF03
:10D37000ACF14054A4F17F641C430BD0022404EAB6
:10D38000AC7444EAD27405439FED538B9FED542B4C
:10D3900007D015E09DED040B51EC100B04F065F97E
:10D3A00042E0002C11BF012C9DED040B02B0BDEC3E
:10D3B000028B04BF04B070BD022C38D0032C3BD0CC
:10D3C0000B439FED491B9FED4A0B0AD0B14218D188
:10D3D000B04209D121F0804120F0804007910590B2
:10D3E0000FE0002A15DA10E0434B7B44002C08BF05
:10D3F00093ED000B0DD0012C10D0022C17D0032C74
:10D400001AD0B0421DD1002A03DAB0EE410AF0EE84
:10D41000610A02B0BDEC028B04B070BD93ED000B4D
:10D4200051EC100B81F0004141EC100BF1E7B0EE34
:10D43000480AF0EE680AECE7B0EE420AF0EE620A43
:10D44000E7E7401A00153C28C8BF8DED000B19DC3A
:10D45000BCF1000FBEBF10F13C0F9FED290B8DED0D
:10D46000000B0FDB9DED060B53EC102B9DED040B19
:10D4700051EC100BF9F754F90AF098FE04F0F5F8A6
:10D48000CDE90001002C08BF9DED000BC1D0012C9F
:10D4900010D0022C9FED1C0B53EC102B9DED000BBC
:10D4A00051EC100B0DD0F9F7C3F853EC182BF9F72A
:10D4B000BFF8B9E7019880F0004001909DED000BA6
:10D4C000A7E7F9F7B5F853EC182BF9F7B4F8ABE781
:10D4D0000000F07F00000000182D4454FB2109409B
:10D4E000182D4454FB2109C0182D4454FB21F9BFC9
:10D4F000182D4454FB21F93FD29A0100000000008E
:10D500000000000000000000075C143326A6A13CC8
:10D5100010EE100A10B510EE901A4FF0684202EBB0
:10D5200040032DED028BB3F1654F3CBF02EB41028E
:10D53000B2F1654F7CD200BFC0F3C753C1F3C752ED
:10D540009A1A1B2A09DD10F0004F14BF9FED6E0AD6
:10D550009FED6E0ABDEC028B10BD12F11A0F1BDAA3
:10D5600011F0004F09D010F0004F0CBF9FED680A7A
:10D570009FED680ABDEC028B10BD80EE208A18EE8C
:10D58000100AFFF7A3FA042808BF00F043FEB0EE2C
:10D59000480ABDEC028B10BD4200B2EB410F37D9F7
:10D5A00010F0004F19BFDFED5C1A9FED5C1ADFED44
:10D5B0005C1A9FED5C1AB0EE602A0A46F1EE400A52
:10D5C00080F00041B0EE420A10460A1A5200B2F151
:10D5D000807F34D2484010F0004FDFED532A9FED9A
:10D5E000533A1DBFBEEE002A71EEE21A31EE431A25
:10D5F000B6EE002A04BF71EEA21A31EE031AF0EE65
:10D60000402A42EE602A40EE020A82EEA02A18E08A
:10D6100011F0004F04BF9FED461AF0EE411AD4D02E
:10D6200010F0004F1CBFDFED431A9FED431A00E0DE
:10D6300026E004BFDFED411A9FED411AC5E780EEF9
:10D64000202A22EE020ADFED3F0ADFED3F2ABDEC81
:10D65000028B40EE202ADFED3D0A40EE220ADFED8C
:10D660003C2A40EE202ADFED3B0A40EE220A22EE61
:10D67000000A00EE201A31EE020A30EE210A10BD37
:10D680004FF07F42B2EB400F28BFB2EB410F05D203
:10D69000BDEC028BBDE8104000F0B1BD40EA0103D3
:10D6A0005B0008BF41F0FF410BD0B2EB400F08BF59
:10D6B000B2EB410F08D120F0804000EE100A21F0BB
:10D6C000804100EE901A37E7B2EB400F12BF5FEADD
:10D6D000410240F0FF4001F000413FF42DAF4A000D
:10D6E00092EA40033FF528AF002AACBF9FED1A1A1B
:10D6F0009FED1A1A20EE010A60EE810A10EE100A60
:10D7000010EE901A18E70000DB0FC9BFDB0FC93F0E
:10D71000DB0F4940DB0F49C00000C9BF22AAFDB999
:10D720000000C93F22AAFD390060ED3EC30ACE3792
:10D7300000000000000049C022AA7DBA0000494054
:10D7400022AA7D3A2DAD65BD8FB8D53D0FB511BE6E
:10D7500061C84C3EA8AAAABE0000804F0000802FDE
:10D7600010B52F499FED2C1B2DED020B84B00598B1
:10D7700020F000408842D8BF9DED040B2DDD2949E3
:10D78000884209D1049840B94FF0010000F07CFDB7
:10D7900000F012FD06B010BD05DB9DED040B00F09E
:10D7A000F7FC06B010BD68469DED040B00F008F9CB
:10D7B00010F0030004BF9DED021B9DED000B0CD08B
:10D7C00001280ED09DED021B9DED000B022817D005
:10D7D000012000F045FC06B010BD00F00DFB06B0C6
:10D7E00010BD9DED021B9DED000B012000F038FCEB
:10D7F00051EC100B81F0004106B041EC100B10BD54
:10D8000000F0FAFA51EC100B81F0004106B041EC47
:10D81000100B10BD00000000000000000000000020
:10D82000FB21E93F0000F07F2DED020B019820F075
:10D83000004001909DED000B02B070470000000019
:10D8400010B52F499FED2C1B2DED020B84B00598D0
:10D8500020F000408842DCBF00209DED040B32DD4B
:10D860002849884209D1049840B94FF0010000F0DE
:10D870000BFD00F0A1FC06B010BD05DB9DED040B17
:10D8800000F086FC06B010BD68469DED040B00F06C
:10D8900097F810F0030011D0012818D09DED021B5D
:10D8A0009DED000B02281AD000F0A6FA51EC100BE7
:10D8B00081F0004106B041EC100B10BD9DED021B44
:10D8C0009DED000B012000F0CBFB06B010BD9DEDDF
:10D8D000021B9DED000B00F08FFA06B010BD012079
:10D8E00000F0BEFB51EC100B81F0004106B041ECA2
:10D8F000100B10BD00000000000000000000000040
:10D90000FB21E93F0000F07F00B52DED048BB0EE68
:10D91000409AF0EE609A83B051EC190BF9F7FFF8DA
:10D9200041EC180B18EE100A18EE901A8DED008BD2
:10D93000002818BF0120084320F00040C0F17F609C
:10D9400000F1E040C00F14D019EE101A19EE900A41
:10D950008DED009B002918BF0121084320F00040F5
:10D96000C0F17F6000F1E040C00F04BF012000F073
:10D970008BFCB0EE480A03B0F0EE680ABDEC048BF5
:10D9800000BD10B52DED028BB1EEC08A18EE100A65
:10D9900020F00040C0F1FF40C00F0AD010EE100A86
:10D9A00020F00040C0F1FF40C00F04BF012000F094
:10D9B0006BFCB0EE480ABDEC028B10BD000000000D
:10D9C0002DE9F14F04462DED020B2DED088B8AB0A9
:10D9D0009FEDE70B80ED020B139EE74826F0004514
:10D9E00085420ADC9DED120B002084ED000B0AB08D
:10D9F000BDEC088B03B0BDE8F08FE0489FEDE0ABD5
:10DA00009FEDE1BBA84247DDE14F9FEDE39B9FED1A
:10DA1000E48B9DED120B53EC1A2B51EC100B002EE6
:10DA20001CDDF8F705FE41EC100BBD4208D053ECAD
:10DA30001B2B51EC100BF8F7FBFDC4E900010BE0C8
:10DA400053EC192B51EC100BF8F7F2FD53EC182B9B
:10DA5000F8F7EEFDC4E900010120C8E7F8F747FD3B
:10DA600041EC100BBD4208D053EC1B2B51EC100BBA
:10DA7000F8F73DFDC4E900010BE053EC192B51EC24
:10DA8000100BF8F734FD53EC182BF8F730FDC4E910
:10DA900000014FF0FF30AAE7C348A84279DB9DEDB3
:10DAA000120B51EC100B0AF081FB41EC180B9FEDAF
:10DAB000C00B53EC102BF8F7C1FD9FEDBF1B53ECCF
:10DAC000112BF8F714FDF8F7B8FE0746F8F797FEA4
:10DAD00041EC190B53EC1A2BF8F7B0FD53EC182B53
:10DAE000F8F7A9FD41EC180B53EC1B2B51EC190B6B
:10DAF000F8F7A4FDDFF8C8A241EC100B4FEA155867
:10DB00000125FA4453EC102B51EC180BF8F790FD5B
:10DB1000032DC4E900013DD0C1F30A5005EB4511C6
:10DB2000A8EB00001139814234DA0AEB051BB0EE94
:10DB300048AA9BED000BF0EE68AA53EC102B51ECB9
:10DB4000190BF8F77BFD41EC1B0B51EC1A0B53EC56
:10DB50001B2BF8F76DFD41EC180B51EC1A0B53EC35
:10DB6000182BF8F765FD53EC1B2BF8F761FD9BEDC7
:10DB7000020B41EC1A0B53EC102B51EC190BF8F77C
:10DB80005DFD53EC1A2BF8F753FD41EC100B6D1CA7
:10DB9000B8E70EE0002EA8BF3846BFF628AF94EDD8
:10DBA000000B51EC100B81F00041C4E900017842F8
:10DBB0001DE7C6F3130040F4801EC6F30A50A0F21E
:10DBC000F530471100F01F05C5F12000DDF848B021
:10DBD00008900020069007900520EC467949002D1A
:10DBE00007EB0002794408BF51F8221009D051F820
:10DBF000223001EB8201AB404A68089922FA01F118
:10DC00001943A1FB0E26A1FB0B131A449A4234BF01
:10DC10000123002303EB06080CEB8003D3E901A6E4
:10DC20000E448E4234BF0121002192448A4411B136
:10DC3000924502D903E0924501D2012100E0002182
:10DC4000C3E901A641444CF82010011EA0F10100D7
:10DC5000C4DC029800F10050850F0298DDE90367EB
:10DC60008000DDF81480F8F7CAFD41EC1A0B30464D
:10DC7000F8F7D6FD9FED541B53EC112BF8F7DEFCA3
:10DC800041EC1B0B3846F8F7CBFD9FED511B53ECD5
:10DC9000112BF8F7D3FC41EC180B4046F8F7C0FD08
:10DCA0009FED4D1B53EC112BF8F7C8FC41EC190B01
:10DCB00051EC180B53EC192BF8F719FC53EC1B2BF8
:10DCC000F8F715FC53EC1A2BF8F711FCCDE9080115
:10DCD000002008909DED080B53EC1A2B51EC100B13
:10DCE000F8F7A6FC53EC1B2BF8F7A2FC53EC182B0F
:10DCF000F8F79EFC53EC192BF8F79DFC9FED381BB1
:10DD000053EC112BF8F79AFC9FED370B41EC180BF5
:10DD100053EC102B9DED080B51EC100BF8F78EFC1B
:10DD200053EC182BF8F7E3FB9FED310B41EC180B8C
:10DD300053EC102B9DED080B51EC100BF8F77EFC0B
:10DD400053EC182BF8F7D3FB41EC100B139810F0A1
:10DD5000004F06D06D4251EC100B81F0004141ECB8
:10DD6000100B284684ED000B41E600000000000087
:10DD70000000000000000000FB21E93F7CD90240C8
:10DD800000004054FB21F93F3163621A61B4D03D79
:10DD9000FB21F93F000000000000601A61B4D03D93
:10DDA0007370032E8A19A33BFB2139410000000048
:10DDB00083C8C96D305FE43F000000000000E03F11
:10DDC000C293010010930100000000000000103E0B
:10DDD000000000000000103C000000000000103AAD
:10DDE000182D4454FB21F93D3326A611460B113C56
:10DDF00000000054FB21F93D10B52DED040B2DED75
:10DE0000088B82B0B0EE419AF0EE619A0B9820F048
:10DE100000449FED4BABB4F1795F11DA9DED0A0B35
:10DE200051EC100BF8F709FD002801BFB0EE4A0ACB
:10DE3000F0EE6A0A02B0BDEC088B04BF04B010BD5E
:10DE40009DED0A0B53EC102B51EC100BF8F7F6FB81
:10DE500041EC180B3C480621B0EE480AF0EE680A87
:10DE6000784400F081F853EC182B51EC100BF8F7C4
:10DE7000E5FB9DED0A0B41EC1B0B53EC192B51EC10
:10DE8000100BF8F7DBFB41EC190B53EC1B2B51EC9F
:10DE9000180BF8F7D3FB53EC192BF8F7C9FB9FEDE0
:10DEA0002C0B41EC190B53EC102B51EC180BF8F721
:10DEB000C5FB41EC100B2848844210DA53EC192BB7
:10DEC00051EC100BF8F7B4FB53EC1A2BF8F7B3FB3B
:10DED00041EC100B02B0BDEC088B04B010BD1F4824
:10DEE000A042BCBF9FED1E1B8DED001B06DBA4F501
:10DEF00000100190002000909DED001B51EC100BD4
:10DF000053EC112BF8F794FB9DED000B41EC180B33
:10DF100053EC102B51EC1A0BF8F78AFB41EC1A0B5F
:10DF200053EC192B51EC180BF8F782FB53EC1A2B1E
:10DF3000F8F781FB41EC100BCCE70000000000007B
:10DF4000000000000000F03F2C90010000000000E5
:10DF5000000000000000E03F3333D33F0000E93F02
:10DF6000000000000000D23F70B504462DED028B8A
:10DF70004D1E00EBC500B0EE408AF0EE608A90EDD9
:10DF8000000B35F0060017D053EC182B51EC100B9A
:10DF9000F8F754FB41EC100B6D1E04EBC50090ED3F
:10DFA000001B51EC100B53EC112BF8F7A0FA41ECCD
:10DFB000100B35F00600E7D1022D36D0042D1CD011
:10DFC000062D1CBFBDEC028B70BD53EC182B51EC21
:10DFD000100BF8F733FB94ED0A1B53EC112BF8F7F9
:10DFE00086FA53EC182BF8F729FB94ED081B53EC39
:10DFF000112BF8F77CFA41EC100B53EC182B51EC79
:10E00000100BF8F71BFB94ED061B53EC112BF8F7E4
:10E010006EFA53EC182BF8F711FB94ED040B53EC4C
:10E02000102BF8F764FA41EC100B53EC182B51EC61
:10E03000100BF8F703FB94ED021B53EC112BF8F7D0
:10E0400056FA53EC182BF8F7F9FA94ED001B53EC41
:10E05000112BF8F74CFABDEC028B41EC100B70BDA4
:10E0600031B504462DED040B2DED0A8BB0EE41BA0F
:10E07000F0EE61BA0B989DED0A0B20F00040B0F174
:10E08000795F0DDA51EC100BFEF708FD042808BF8C
:10E0900000F0A2F89DED0A0BBDEC0A8B05B030BD77
:10E0A00053EC102B51EC100BF8F7C8FA41EC180B9D
:10E0B0009DED0A0B53EC182B51EC100BF8F7BEFA40
:10E0C00041EC190B2C48B0EE480AF0EE680A052125
:10E0D0007844FFF749FF9FED2ACBB0EE40AAF0EE5F
:10E0E00060AA9CB353EC1C2B51EC190BF8F7A6FA61
:10E0F00041EC1C0B53EC1A2B51EC190BF8F79EFA60
:10E100009FED210B41EC190B53EC102B51EC1B0B29
:10E11000F8F794FA53EC192BF8F78AFA53EC182B0A
:10E12000F8F78CFA53EC1B2BF8F782FA53EC1C2B04
:10E13000F8F77EFA9DED0A1B53EC112BF8F77BFAEA
:10E14000BDEC0A8B05B041EC100B30BDFFE753EC82
:10E150001A2B51EC180BF8F771FA53EC1C2BF8F74B
:10E16000C6F953EC192BF8F769FA9DED0A1B53EC2D
:10E17000112BF8F7BCF9E3E7BC8E010000000000AA
:10E18000495555555555C5BF000000000000E03FFA
:10E1900010B553EC102B51EC100BF8F7A8F941EC2B
:10E1A000100B10BD10B553EC112B51EC100BF8F700
:10E1B0009EF941EC100B10BD9FED050B10B553EC13
:10E1C000102B51EC100BF8F7ABFA41EC100B10BD13
:10E1D00000000000000000009FED050B10B553EC9F
:10E1E000102B51EC100BF8F729FA41EC100B10BD75
:10E1F000000000000000001030EE000A704730EE12
:10E20000200A7047DFED020A80EEA00A7047000086
:10E21000000000009FED020A20EE000A7047000097
:10E220000000001002E008C8121F08C1002AFAD13D
:10E2300070477047002001E001C1121F002AFBD186
:10E24000704700000146202908DA012088400A4A68
:10E25000104008B1012070470020FCE7402909DA8E
:10E26000A1F12000012202FA00F008B10120F2E73A
:10E270000020F0E70120EEE7FC06FFBD00BFEFF352
:10E280001081084672B67047014908607047000067
:10E29000104B00202DE9FF5F82B00021DDE9043042
:10E2A000020DDDF840B0034318D044F61050A2F23E
:10E2B000FF3242431514119801281FD0A5EB0B0023
:10E2C000401C5FEA000A4FF000064E4FDFF838911D
:10E2D000B046504615D5CAF1000413E01198012448
:10E2E0004AA3012801D16FEA0B010298119AC0E9F3
:10E2F0000031C0E9024206B0BDE8F09FCBF100005A
:10E30000DFE704460021404A491842EB0450CDE9BA
:10E31000001012E0E00707D032463B46404649462F
:10E32000F8F78CF98046894632463B461046194636
:10E33000F8F784F906460F466410002CEAD1DDE9AF
:10E340000401DDE90023BAF1000F06DAF8F776F9E7
:10E3500042464B46F8F772F905E0F8F7E1F9424614
:10E360004B46F8F7DDF904460E460022284BF8F735
:10E37000C7FA03D84FF0FF30014607E00022254BD3
:10E3800020463146F8F7B3F8F8F71AFC102409E0F4
:10E39000002C0ADB0A220023F8F732F8039B303204
:10E3A0001A55641E50EA0102F2D1641C039AC4F1AA
:10E3B00011031444119A012A03D0012208430DD1FC
:10E3C0000AE0084304D000204FF0110B119072E7CF
:10E3D000A3EB0B056D1E0DE05B4504DD4FF0000265
:10E3E00005F1010504E003DA4FF00002A5F1010593
:10E3F000002AECD002981199C0E90231C0E9004529
:10E4000079E70000000014400000F03F30000000F9
:10E410000000F0430000E03F2DE9FF4F95B09B4620
:10E420008946064600250FE2252877D10024274695
:10E43000F84A0121059400E0044316F8013F203B0F
:10E4400001FA03F01042F7D130782A2811D06FF08A
:10E450002F033078A0F13002092A16D8059A44F02B
:10E46000020402EB820203EB42021044761C059088
:10E47000EFE759F8042B0592002A03DA504244F4DE
:10E480000054059044F00204761C30782E2816D1F2
:10E4900016F8010F44F004042A280DD06FF02F0263
:10E4A0003078A0F13003092B09D807EB870302EB82
:10E4B0004303C718761CF3E759F8047B761C3078C1
:10E4C0006C280FD006DC4C2817D068280DD06A289D
:10E4D00014D104E0742810D07A280FD10DE044F450
:10E4E00000140AE044F4801401E044F4401472780B
:10E4F000824202D104F58014761C761C307866289E
:10E500000BD013DC582877D009DC002875D04528BB
:10E51000F6D04628F4D047281AD19DE118E06328A8
:10E5200035D0642879D0652812D195E1702873D050
:10E5300008DC6728F1D069286FD06E280DD06F28CD
:10E5400006D1B5E073282CD0752875D0782874D002
:10E550005A46179990476D1C75E1C4F30250022882
:10E5600009D003280DD0D9F8001004280DD00D6073
:10E5700009F1040967E1D9F80010EA17C1E900526E
:10E58000F6E7D9F800100D80F2E70D70F0E719F802
:10E59000041B8DF8001000208DF80100EA460120D0
:10E5A00003E059F804AB4FF0FF3061074FF0000172
:10E5B00002D40DE008F101018846B9420FDA804526
:10E5C000F8DB1AF808100029F4D108E008F101017D
:10E5D00088468142FADB1AF808100029F6D105981E
:10E5E0005B46A0EB080721463846179A00F094FADC
:10E5F000284400EB080507E04DE029E10DE01AF89A
:10E60000010B5A4617999047B8F10108F7D25B46BB
:10E6100021463846179A13E142E00A220092C4F3D9
:10E6200002524FF0000A022A08D059F804CB032AFC
:10E630004FEAEC710AD00DE029E02AE009F1070168
:10E6400021F00702F2E802C1914609E00FFA8CFCC2
:10E650004FEAEC71042A03D14FFA8CFC4FEAEC71BB
:10E66000002907DA0A460021DCF1000C61EB020107
:10E670002D2202E0220504D52B228DF80420012250
:10E6800003E0E20701D02022F7E7904659E00A2193
:10E6900002E010220DE010214FF0000A00910BE083
:10E6A00010224FF0000A44F004040827009203E00F
:10E6B00008224FF0000A0092C4F30252022A05D049
:10E6C00059F804CB0021032A08D009E009F1070119
:10E6D00021F00702F2E802C1914605E01FFA8CFC26
:10E6E000042A01D10CF0FF0C4FF00008220728D5B6
:10E6F000702806D0009B83F0100353EA0A0305D06C
:10E700000EE040228DF80420012208E05CEA0102BC
:10E7100006D030228DF804208DF8050002229046A4
:10E72000009B83F0080353EA0A030AD15CEA010262
:10E7300001D1620705D530228DF804204FF0010881
:10E740007F1E582804D034A003900EA802900DE03C
:10E7500036A0F9E753466046009AF7F751FE844623
:10E760000398825C0298401E029002705CEA0100ED
:10E77000F0D1029806A9081A00F1200A600702D514
:10E7800024F4803400E00127574502DDA7EB0A009E
:10E7900000E0002000EB0A01009005984144401A77
:10E7A0000590E00306D45B462146179A059800F0D1
:10E7B000B3F90544002706E001A85A46C05D179941
:10E7C00090476D1C7F1C4745F6DBE0030CD55B468C
:10E7D0002146179A059800F09FF9054404E030207F
:10E7E0005A46179990476D1C0099481E00900029C1
:10E7F000F5DC08E0029802995A460078491C02911B
:10E80000179990476D1CBAF10001AAF1010AF1DCD9
:10E8100065E10000092801003031323334353637E4
:10E82000383961626364656600000000303132335C
:10E8300034353637383941424344454600000000FC
:10E8400000F058F90544761C307800287FF4ECADD0
:10E8500019B02846BDE8F08F620700D4062709F1F9
:10E86000070222F0070CFCE80223E14603F000480F
:10E870005FEA080C02D00FF2702C0DE05FEA045C36
:10E8800002D50FF2682C07E05FEAC47C02D00FF2D9
:10E89000602C01E0AFF2700C4FF0FF3823F0004322
:10E8A000CDF850C065280CD006DC452809D0462894
:10E8B0001DD047283DD13DE0662818D067287ED17D
:10E8C00038E00021112F01DB112000E0781CCDE998
:10E8D000000106A90EA8FFF7DDFCDDE90F010E9A85
:10E8E00003910021009207F1010A04914DE04FF0DD
:10E8F00000400097CDE9011006A90EA8FFF7CAFC59
:10E90000DDE90F0203920E9B11990022DDF80CA0A5
:10E910000093049211B9791C00EB010AB7EB0A00CD
:10E9200004D4C0F1FF3007F1010A0490AAEB0700FC
:10E93000019044E0012F00DA01270021112F01DDB1
:10E94000112000E03846CDE9000106A90EA8FFF726
:10E95000A1FCDDE90F010E9A0391002104910092C0
:10E96000BA4621070CD40399514500DA8A46BAF118
:10E97000010F05DD009AAAF10101515C302908D090
:10E98000B84202DA10F1040F06DA0121CDE90110D4
:10E9900015E0AAF10101E9E7002805DC049901442A
:10E9A0000491AAEB000102E0411C514500DD8A46BA
:10E9B0000499401A401C01904FF00040029020073B
:10E9C00004D40198504501DBCDF8048000208DF877
:10E9D0004F0002980DF14F07B0F1004F25D02B20CA
:10E9E0000E9002984FF0020800280CDA4042029084
:10E9F0002D200E9007E00A210298F7F7B5FF30317D
:10EA0000029007F8011DB8F10001A8F10108F2DC3D
:10EA100002980028EFD1791E0E980870307800F027
:10EA2000200040F0450007F8020D12A8C01B00F1BD
:10EA300007081498007800B1012000EB0A01019842
:10EA400001EBE07105984144401A401E0590E00337
:10EA500006D45B462146179A059800F05DF80544F8
:10EA60001498007818B15A46179990476D1CE00326
:10EA700024D55B462146179A059800F04DF80544C9
:10EA80001CE00498002807DBDDE90301884203DD70
:10EA90000098405C179901E0179930205A4690473A
:10EAA000049805F10105401C04900198401E019056
:10EAB00004D12E205A46179990476D1CBAF10001D7
:10EAC000AAF1010ADDDC05E017F8010B5A46179997
:10EAD00090476D1CB8F10001A8F10108F4DC5B4619
:10EAE0002146179A0598ABE62D0000002B00000088
:10EAF000200000002DE9F041044600251E4617467F
:10EB0000880404D405E039462020B0476D1C641EFB
:10EB1000F9D52846BDE8F0812DE9F04104460025ED
:10EB20001E469046C80301D5302700E02027880400
:10EB300004D505E041463846B0476D1C641EF9D542
:10EB40002846BDE8F0810A68531C0B6010707047BE
:10EB50002DE9FC4105461CA103C9CDE900010027B0
:10EB6000287800282DD11A4A128891B2686811F0CD
:10EB70007FFE06462EBB00240BE004EBC4001549C3
:10EB80000844C07920B1E0B20DF80700781CC7B284
:10EB9000641C082CF1DB002408E00F4830F8140056
:10EBA0001DF804100D4A22F81100641C0848006882
:10EBB0008442F2D30A48006818B108480849096835
:10EBC0008847BDE8FC810000FFFFFFFFFFFFFFFF5C
:10EBD00060410020AC790020F4790020047A002004
:10EBE0006441002038B504460020009069460720A3
:10EBF00009F062FCBDF800104FF4167211FB02F030
:10EC0000C11700EB1151091301EB4101490001EB60
:10EC10008101032291FBF2F109B20091BDF90000DC
:10EC20000EF0B4FB00B20849A1F850006946052077
:10EC300009F042FCBDF90000502804DD0248C06C18
:10EC4000401C0149C86438BD3C50002002460021E8
:10EC500004E0505C08B101207047491C0629F8D334
:10EC60000020F9E770B504460D4604F22740FFF78F
:10EC7000EDFF0646012D06D0022D0DD0032D11D03B
:10EC8000042D19D113E0A07928B194F8240010B90B
:10EC90000EB1012070BD00BFE07910B10EB10220AD
:10ECA000F8E700BF207A08B10320F3E700BF607ADD
:10ECB00008B10420EEE700BF0020EBE70146481C46
:10ECC000052290FBF2F302FB1300C0B270472DE95E
:10ECD000F04704460D462F4695F82080B4F81C9066
:10ECE00000260BE007EB46124946A06902F011FF2F
:10ECF00010B10120BDE8F087701CC6B24645F1DBBB
:10ED00000020F7E7014691F82420012A01D1EE20E6
:10ED100000E01F2070470000014671B1002009E0AB
:10ED2000064A52F820201AB9044A42F8201003E09B
:10ED3000421CD0B20228F3DB00BF704740480020DD
:10ED4000014600200BE0084A52F820208A4204D1F4
:10ED50000022054B43F8202003E0421CD0B20228D9
:10ED6000F1DB00BF704700004048002030B5B1B073
:10ED700004200590AC2106A8F7F78CFB02208DF843
:10ED8000180000208DF81A0004908DF81000012062
:10ED90008DF8110004208DF8120001208DF8130069
:10EDA0002220ADF8040004A903910420ADF8080066
:10EDB00001A91E9105208DF81B0005A807900121CF
:10EDC000ADF8641011491A9101218DF894104FF497
:10EDD000A071289144F2506129910D482F9006A905
:10EDE0000C4802F002FF044600BF254635B100BFC3
:10EDF00009A28C212846F7F70DFA00BF00BF0121B8
:10EE0000044802F0EFFE31B030BD0000C0410020E8
:10EE1000FD110400647B00202E2E5C2E2E5C2E2E15
:10EE20005C626C655F6366675C736C6176652E63BC
:10EE30000000000070B50321084802F078FF044686
:10EE4000082C0AD000BF254635B100BF04A2AD2171
:10EE50002846F7F7DFF900BF00BF70BD647B0020D4
:10EE60002E2E5C2E2E5C2E2E5C626C655F636667B8
:10EE70005C736C6176652E630000000070B5094913
:10EE800091F8540074DF0446082C0AD000BF2546D0
:10EE900035B100BF04A2B6212846F7F7BBF900BF81
:10EEA00000BF70BD647B00202E2E5C2E2E5C2E2EAB
:10EEB0005C626C655F6366675C736C6176652E632C
:10EEC000000000001CB5FAF78EFCFCF761FA002187
:10EED0000F480DF038FE01A90D480DF023FE9DF8F6
:10EEE000040010B14FF0FF301CBD002108480DF0A8
:10EEF00061FE02200090694605480DF03DFE9DF838
:10EF0000000010B14FF0FF30EEE70020ECE700000A
:10EF1000987A002010B5054A05A16420FBF738FD5A
:10EF20000649B020F8F764F910BD000041EF020077
:10EF30006170705F417574686F6E00003940030046
:10EF400010B51C480079C8B10BF0CAFD78B11A4859
:10EF500000781E2812DA18480078401C16490870FC
:10EF60000123164AB0210020F8F7F4FB06E012480E
:10EF70000078002802DD00200F49087016F010FD0F
:10EF800080B10F480078002813DD0D480078401C40
:10EF9000C0B20B49087096280BDD9620087016F059
:10EFA000C7FC06E006480078012802D00120044989
:10EFB000087010BD74530020314000203240002002
:10EFC0003040002010B50E480079B8B101F056FA73
:10EFD000A0B10C4801790079401C0A4A107105293A
:10EFE0000CDB00201146C870074803F085FE0123A2
:10EFF000044AD21CA2210020F8F7ACFB10BD00008F
:10F0000074530020343F0020F067040010B51C202A
:10F0100000BF4FF0A042114600BFD1F81025C240FA
:10F0200002F00102144654B906480068A04206D016
:10F030000820FAF7A7FA00210348FBF783FC0148F0
:10F04000046010BDF43F00200DF0020030B587B021
:10F05000182101A8F7F71EFA0BF0F0FC08B907B069
:10F0600030BD0024002003F08FFE04B2002C7DDDB3
:10F07000611E01AA002003F07DFEBDF9082065484D
:10F0800003886549654816F095FD624800880528A3
:10F0900026DDBDF908006049B1F90010401AFF28CB
:10F0A0001BDC5E48B0F90000BDF90810401AFF28CB
:10F0B00013DC5A48B0F900005749B1F90010401A62
:10F0C000FF280ADCBDF9040010F5167F05DA544864
:10F0D0000088401C5249088002E000205049088006
:10F0E0004C480088401C4B490880BDF8040010FBC8
:10F0F00000F0BDF8061011FB0100BDF8081011FB6F
:10F100000105A5F58000002801DB014600E0414231
:10F11000444A91420ADABDF90810B1F5C06F05DD25
:10F1200041480088401C4049088002E000203E49D8
:10F1300008803D480088052803DA394800880428FB
:10F1400002DD06203949087038480078002804DDBF
:10F1500036480078401E3549087034480078002849
:10F1600039DD3348007800BB642000E04FE03049CF
:10F170000870F9F75BFB142804DD2E490420FAF728
:10F18000E1F903E02C490420FAF7DCF90121AFF2A0
:10F190004310FBF7D7FB2948007990B10123284A97
:10F1A000B0212848F8F7FAF80BE021480078022847
:10F1B00007D10420FAF7E6F90021AFF26F10FBF750
:10F1C000C1FB1B480078012820DD19480078401E4B
:10F1D000174908701AE01648007850B10020144909
:10F1E00008700420FAF7CEF90021AFF29F10FBF768
:10F1F000A9FB1548007848B901201349087004207C
:10F20000FAF7C0F900211148FBF79CFB00BF00BFD3
:10F2100025E700005C3E00207C3E0020643E00208C
:10F220005E3E0020A0860500603E0020623E002079
:10F23000633E0020009F00FF00103FFF745300203A
:10F24000313E0020343E0020303E002051F20200CA
:10F2500030B587B0182101A8F7F71CF90BF0EEFBC9
:10F2600008B107B030BD0025002003F08DFD05B2C8
:10F27000002D7DDD691E01AA002003F07BFDBDF895
:10F28000040010FB00F0BDF8061011FB0100BDF8F2
:10F29000081011FB0104A4F58000002801DB0146E1
:10F2A00000E041425D4A914208DABDF90810B1F52B
:10F2B000C06F03DD03205A49087008E05848007801
:10F2C000002804DD56480078401E55490870A4F512
:10F2D0008000002801DB014600E041424F4A914294
:10F2E00008DABDF9041011F5617F03DA03204D49F6
:10F2F000087008E04B480078002804DD4948007891
:10F30000401E48490870A4F58000002801DB014632
:10F3100000E04142414A914207DABDF9081011F577
:10F32000806F02DA00203E490870A4F580010029B0
:10F3300001DB0A4600E04A42384B9A420CDABDF93A
:10F340000400002801DB024600E04242B2F5C87F1B
:10F3500002DA00203349087031480078002803DCC5
:10F3600030480078002839DD2F48007800BB00E0E5
:10F3700052E00A202C490870F9F758FA142804DDE5
:10F380002A490420FAF7DEF803E029490420FAF7B5
:10F39000D9F80121AFF24710FBF7D4FA25480079DC
:10F3A00090B10123244AB0212448F7F7F7FF0BE07E
:10F3B0001D480078022807D10420FAF7E3F800215D
:10F3C000AFF27310FBF7BEFA17480078012822DD70
:10F3D00015480078401E144908701CE01248007857
:10F3E00050B10020104908700420FAF7CBF8002132
:10F3F000AFF2A310FBF7A6FA1148007801280AD152
:10F4000000200F4908700420FAF7BCF80021AFF281
:10F41000BF10FBF797FA00BF00BF22E7A0860500E8
:10F42000583E0020593E00205A3E0020009F00FF19
:10F4300000103FFF74530020313E0020343E002076
:10F44000303E0020014800797047000074530020CE
:10F4500010B58AB000246846F9F70CFA00980290BB
:10F46000BDF80400ADF80C00A41D00222146641C68
:10F4700002A8425401222146641C4254042221461F
:10F48000641C425401222146641C4254002220463E
:10F49000611CCCB202A90A5422222046611CCCB2C3
:10F4A00002A90A540AF078FF022803D00AF074FF78
:10F4B000032806D101222046611CCCB202A90A54BD
:10F4C00005E000222046611CCCB202A90A5409487A
:10F4D000007930B1234602AAB1210020F7F75EFF80
:10F4E00005E0234602AAB1210020F8F733F90AB05B
:10F4F00010BD00007453002010B5034A03A164201E
:10F50000FBF746FA10BD000019F502006170705F4C
:10F51000636861726765000010B50AF03DFF04463C
:10F5200014480078844224D0012C04D0022C0AD044
:10F53000032C1AD110E00520FAF724F800210E4818
:10F54000FBF700FA12E001210B48FBF7FBF90B492E
:10F550000520F9F7F7FF09E001210748FBF7F2F969
:10F5600007490520F9F7EEFF00E000BF00BF0148A2
:10F57000047010BDF83F002019F5020000103FFF95
:10F58000009F00FF30B589B00024202101A8F6F7C4
:10F5900081FF68464CDF00988010009001222146D0
:10F5A000641C01A84254F9F741F901462246641C43
:10F5B00001A881540098C2B22146641C01A842549B
:10F5C000241D3B484069020E2146641C01A8425498
:10F5D00037484069C0F307422146641C01A84254E1
:10F5E0003348808AC0F307222146641C01A8425494
:10F5F0002F48027D2146601CC4B201A8425401F08C
:10F6000003F92146621CD4B201AA505401F0F0F86B
:10F610002146621CD4B201AA5054201DC4B2244811
:10F620008069020E2046611CCCB201A90A54204810
:10F630008069C0F307422046611CCCB201A90A547C
:10F640001B48008BC0F307222046611CCCB201A9E5
:10F650000A541748027E2046611CCCB201A90A5404
:10F660000AF0D6FC0546C5F307222046611CCCB241
:10F6700001A90A542046611CCCB201A90D5401F025
:10F68000BDF8C0F307222046611CCCB201A90A5480
:10F6900001F0B4F8C2B22046611CCCB201A90A54F0
:10F6A000234601AAA1210020F7F778FE09B030BD5A
:10F6B0007453002070B50546002400BF06E0601CAE
:10F6C0006968095C0A480155601CC4B2082CF6DB65
:10F6D0006968487A01F06EF905480C38406A28B12B
:10F6E000002103480C38416208F0A4FE70BD000000
:10F6F0008053002010B50649A120F7F779FD00F0EE
:10F7000037FA044A04A14FF4FA60FBF741F910BD3F
:10F710006943030025F702006170705F636C6965DF
:10F720006E74000010B50E48007900B110BD16F0DF
:10F7300037F990B100F0A2FE68B10A48017800786C
:10F74000401C084A1070042907DB0020114608708D
:10F75000FFF718FF01E0FFF715FF00BFE6E7000025
:10F76000745300207E3F002070B5044660688078A6
:10F770006168497840EA01251648406AA0B11548F9
:10F78000406A401E2821B0FBF1F0401C124908805D
:10F790001048406A401E2821B0FBF1F201FB120024
:10F7A000401C0E49088004E000200B4908800B49EA
:10F7B000088055B901200A490870002009490880CD
:10F7C0000846008800F010F802E0284600F0D8F85B
:10F7D00070BD000074530020983E00209A3E002027
:10F7E000953E0020963E00202DE9F041054600247C
:10F7F00008F01DFE691EA02202FB0107022221461D
:10F80000641C56484254002007E055490B5C2146D1
:10F81000621CD4B2514A5354401C0828F5DB5148AD
:10F82000008802122046611CCCB24C490A544D4853
:10F8300002782046611CCCB248490A542A1220465C
:10F84000611CCCB245490A542046611CCCB24349E4
:10F850000D54002D34D101F0B1FC804601F0B4FC10
:10F8600008EB0006320E2046611CCCB23B490A541C
:10F87000C6F307422046611CCCB238490A54C6F38D
:10F8800007222046611CCCB234490A542046611C30
:10F89000CCB232490E54E01E085CFF280FD1A01EE6
:10F8A000085CFF280BD1601E085CFF2807D10846C2
:10F8B000005DFF2803D12CA10B20F8F75FFA44E08C
:10F8C00028480088854222D12B480088820023489E
:10F8D0000119384608F096FD2748007804EB8000AF
:10F8E000C4B2201F1D49085CFF282ED1E01E085C11
:10F8F000FF282AD1A01E085CFF2826D1601E085CC4
:10F90000FF2822D118A10B20F8F738FA1DE0134880
:10F910000119A022384608F075FD04F1A000C4B218
:10F92000201F0E49085CFF280FD1E01E085CFF284D
:10F930000BD1A01E085CFF2807D1601E085CFF28C1
:10F9400003D109A10B20F8F719FA2346034AA12194
:10F950000A48F7F723FDBDE8F08100006051002060
:10F9600080530020983E002073746570206F766588
:10F9700072666C6F770000009A3E00209C3E00206B
:10F9800070B5C0B00546002408F051FD691EA022E4
:10F9900002FB010602222146641C01A842540020F9
:10F9A00007E023490B5C2146621CD4B201AA5354E0
:10F9B000401C0828F5DB1F48008802122046611C05
:10F9C000CCB201A90A541B4802782046611CCCB273
:10F9D00001A90A542A122046611CCCB201A90A547A
:10F9E0002046611CCCB201A90D5412480088854202
:10F9F0000DD111480088820001A80119304608F095
:10FA000001FD0D48007804EB8000C4B208E001A8B5
:10FA10000119A022304608F0F5FC04F1A000C4B2A0
:10FA2000234601AAA1210020F7F7B8FC40B070BD21
:10FA300080530020983E00209A3E002030B5A1B0AF
:10FA400041240025802101A8F6F724FD00208DF82F
:10FA5000040000BF05E03FA0415D01AA681C1154ED
:10FA60006D1C092DF7D301A90819F8F703FFA01D94
:10FA7000C4B200222046611CCCB201A90A54012262
:10FA80002046611CCCB201A90A5404222046611C04
:10FA9000CCB201A90A5401222046611CCCB201A9B2
:10FAA0000A5400222046611CCCB201A90A54222229
:10FAB0002046611CCCB201A90A54002507E0284861
:10FAC000425D2046611CCCB201A90A546D1C062D72
:10FAD000F5DB23483338C06A020E2046611CCCB2E5
:10FAE00001A90A541E483338C06AC0F307422046B1
:10FAF000611CCCB201A90A5419483338808DC0F377
:10FB000007222046611CCCB201A90A54144833389C
:10FB100090F82C202046611CCCB201A90A54104850
:10FB20003338008E02122046611CCCB201A90A545F
:10FB30000B48333890F830202046611CCCB201A924
:10FB40000A54234601AAA1210020F7F727FC21B07F
:10FB500030BD000046554E2053484F450000000080
:10FB6000A75300200148007870470000943E002011
:10FB700010B5074A07A14FF47A70FAF709FF094850
:10FB80004169C069814202D206484169C16110BD24
:10FB9000A9FB02006170705F636C69656E745F73CE
:10FBA000746570007453002010B51C48007820B1B3
:10FBB00001280DD0022829D11BE01948007801281E
:10FBC00005D116490870FCF7B7FC1649086023E018
:10FBD000FCF7B2FC13490968401A42F210718842DE
:10FBE00003D302200D49087002E0012000F0DAFD85
:10FBF00012E0F8F76BFD18B10BA10B20F8F7BEF877
:10FC00000020074908700549087005E000200349F5
:10FC100008700349087000BF00BF10BDC03E00203F
:10FC2000943E0020C43E00207361766520737465A5
:10FC300070206661696C00000120014908707047FE
:10FC4000943E002010B53248007810B1012853D1FD
:10FC500009E015F0A5FE28B101202D49087000200B
:10FC60002C49087051E00AF03BFF80B12948007828
:10FC7000B8B901202749087000F0E2F92649087058
:10FC800001230A46A3212548F7F764FD09E021482E
:10FC90000078002805DD00201E4908701F48F7F78E
:10FCA00001FD1F48008898B1FCF746FC1D49096812
:10FCB000401A1B49098888420AD300201849088045
:10FCC0000420F9F75FFC0021AFF28700FAF73AFE53
:10FCD00015F066FE78B900200D49087010490880BB
:10FCE0000021AFF29F00FAF72DFE0420F9F74AFC3D
:10FCF0000A48F7F7D7FC08E00020054908700849D2
:10FD000008800420F9F73EFC00BF00BF10BD0000D2
:10FD1000AD3F0020AC3F0020AE3F0020803F0020E0
:10FD2000A43F0020A83F002010B583480079A0B967
:10FD30008248007801280FD100208049087080494E
:10FD40000870804908608049088080490870002157
:10FD5000AFF22B00FAF7F6FD10BD784800780128C5
:10FD600002D00120754908707548007820B101283B
:10FD70002BD0022873D173E0FFF7F4FE30B915F0F1
:10FD80000FFE18B90AF008FB012812D000F090FF0E
:10FD900078B901F0C5F860B90121AFF27300FAF744
:10FDA000D1FD14F07BF80020664908600120644909
:10FDB00008706148007938B115F0F2FD20B90AF0F9
:10FDC0008FFE08B10AF044FEB3E0FFF7CBFEA8B9FE
:10FDD00015F0E6FD90B90AF0DFFA01280ED15CA11A
:10FDE0000E20F7F7CBFF0FF08EF90021AFF2C7001E
:10FDF000FAF7A8FD00205249087012E00AF070FEE0
:10FE000078B10021AFF2DF00FAF79CFD4A48007993
:10FE100020B100204C4908804C4908700220484914
:10FE2000087048480068401C46490860642815D39B
:10FE3000FFF798FE40B9404890F82800432803D1C6
:10FE40004AA10F20F7F79AFF0FF05DF90021AFF2FA
:10FE50002710FAF777FD00203949087069E064E05F
:10FE600000F00CFB18B339480078022842D036481D
:10FE700000883C283EDCF1EE0E0AB1EE0E0AF7F7E0
:10FE8000E1FC30B902203149087000202E49088079
:10FE900030E02D4800883C2803D13BA10F20F7F724
:10FEA0006DFF29480088401C2749088022E0274828
:10FEB000007801281ED0244800883C281ADCDFED99
:10FEC0003B0A9FED3A0AF7F7BDFC30B901201F4904
:10FED000087000201C4908800CE01B4800883C2862
:10FEE00003D133A10F20F7F749FF17480088401CC2
:10FEF00015490880FFF736FE58B915F051FD40B995
:10FF00000AF04AFA012804D10AF0EAFD08B10AF021
:10FF10009FFD0AF0E5FD38B90021AFF2F310FAF7C2
:10FF200011FD00200649087003E000200449087014
:10FF300000BF00BF00BF0FE774530020B73F002091
:10FF4000AF3F0020B03F0020B43F0020B63F00206C
:10FF500061647620646973636F6E6E746564206F8C
:10FF60007665722074696D65000000007363616ED0
:10FF70002072696768742073686F6573206F766597
:10FF8000722074696D65000075706461746520424B
:10FF90006C6520636F6E6E20696E74657276616C3D
:10FFA00020372E356D73206661696C000000C842F1
:10FFB00075706461746520426C6520636F6E6E209D
:10FFC000696E74657276616C203130306D732066B5
:10FFD00061696C0010B50E4A0EA16420FAF7D8FCD6
:10FFE0000E48F7F70BFC0E48F7F7E4FB0D4A0EA19D
:10FFF0006420FAF7CDFC0F49A320F7F7F9F80E4972
:020000040003F7
:10000000A320F7F7C9FA0D49AC20F7F7F1F810BDB6
:1000100029FD0200636F6E6E656374003149030051
:100020001149030045FC0200636F6E6E6563745FE7
:100030006C6564003546030099470300D93F03000F
:1000400010B50024064890F82800432801D0022467
:1000500003E00AF045FD00B10124204610BD000078
:100060007453002010B5054A05A10020FAF790FC52
:100070000748F7F7BBFA002010BD00009500030009
:10008000646174615F7472616E7366657200000012
:100090003501030010B500F0F1F918B901F00CFAC0
:1000A000002832D01E48007830B901201C49087061
:1000B00001211C48FAF746FCFCF73EFA1A49096888
:1000C000401AB0F5FA7F12D3FCF736FA16490860E9
:1000D00015F066FC18B9FEF7D1FEFEF7ABFE13482B
:1000E000007920B10AF0FCFC08B913F0D7FEFCF748
:1000F00023FA0F490968401A032810D3FCF71CFAA9
:100100000B490860F8F7AEFE09E00548007830B109
:1001100000200349087000210248FAF713FC10BDC3
:10012000EC3F002095000300E43F002074530020C2
:10013000E83F002070B504460D46E078042803D15E
:1001400029462046F8F74AFF00F0F8FA70BD000093
:1001500010B588B0002004900590069007904A489A
:1001600090F82800432868D10AF0BAFC08B10AF0D8
:100170006FFC15F015FC08B115F0DAFBFEF77EFEFA
:10018000FBF72AFAFFF75EF9002830D03E4890F8D6
:10019000381090F8372090F836003B4B1B7ACDE9A9
:1001A0000030CDE902213848C379827937A104A80B
:1001B000FCF760FC04A8F6F778F90446214604A889
:1001C0000AF094FC002004900590069007902E48B9
:1001D0008379C27934A104A8FCF74CFC04A8F6F793
:1001E00064F90446214604A815F0E0FB21E0264806
:1001F00090F8381090F8372090F83600224B1B7A90
:10020000CDE90030CDE902211F48C37982791FA1D1
:1002100004A8FCF72FFC04A8F6F747F9044621468A
:1002200004A815F0C3FB162123A00AF05FFCFBF71E
:10023000D3F915F075FBFEF7FDFD134840796628EC
:100240001DD09FED210A2148F9F7FAFB9FED1E0A08
:100250001F48F9F7F5FB02200AF0F8F91D4802F0F3
:1002600023FD1D4A1DA16420FAF792FB1F490120BE
:1002700003F02EF801211848FAF764FB02E0012090
:100280001B49087008B010BD745300202530325847
:1002900025303258253032582530325825303258E2
:1002A000253032580000000046554E5F2530325848
:1002B00025303258000000002A2A2A2A2A2A2A2A0F
:1002C0002A2A2A2A2A2A00000000D0422454002088
:1002D0007854002090690400F50203006170705F9B
:1002E0006465746563745F4C52000000757A0200A7
:1002F000FA3F002070B50949002002F0FDFE0446D7
:100300000649012002F0F8FE0546012C01D1012D1D
:1003100002D0024802F0C8FC70BD000090690400E1
:1003200010B5054802F0E8FC0448FAF79BFB0020F2
:100330000AF08CF910BD000090690400F50203007A
:10034000B4B006460F461446224639463046F8F702
:1003500033F901202D4981F854000846806C40F0A3
:10036000040088641C2129482C30F6F793F8012EEC
:100370000CD06FF48050304478B1B0F5405F23D09A
:100380006FF440510844002830D10DE01C2220A118
:100390001E482C30F6F765F834E01C2222A11B48D9
:1003A0002C30F6F75EF82DE02546D5E9003000F157
:1003B0000D0224A102A8FCF75DFB1C2202A9134830
:1003C0002C30F6F74EF81DE0254628680090686846
:1003D00000F10D031EA102A8AA68FCF74BFB1C222A
:1003E00002A90A482C30F6F73CF80BE03A461DA16A
:1003F00002A8FCF73FFB1C2202A904482C30F6F7A8
:1004000030F800BF00BFFCF775FB0000A0FF002024
:1004100053443A20415353455254494F4E2046418C
:10042000494C45440D0A000053443A20494E564178
:100430004C4944204D454D4F52592041434345536B
:10044000530D0A00663A25732C6C3A25750D0A0087
:10045000653A25752C663A25732C6C3A25750D0A7C
:1004600000000000554E4B4E4F574E204641554C14
:1004700054203078253038580A000000014840796F
:1004800070470000343F002010B50A4A0AA16420DA
:10049000FAF77EFA0B49A220F6F7AAFE0A4A0BA148
:1004A0004EF66020FAF774FA0B49012002F010FFB3
:1004B00010BD0000DD0403006170705F67616D6551
:1004C000000000008D410300C5EF02004175746F0C
:1004D0004F757467616D6500859A030070B50024DF
:1004E00000256B480078002804DD69480078401E2C
:1004F000674908706748007810B101287CD144E052
:100500006348C078002835D06349002002F0F4FD2C
:1005100004466149012002F0EFFD054634B92DB9CA
:1005200001205C4908705A4948711DE0012C01D135
:10053000012D19D0584802F0B7FB58480078401CEC
:10054000C0B256490870C8280EDB00200870504918
:10055000C870514802F0D0FB51A10920F7F70EFCFA
:1005600000215648FAF7EEF94948007910B1002009
:100570004749087146480078002805DD5048007951
:1005800010B1002000F0E4F880E04D48007920B37D
:100590000AF0A6FA10B33E48007888B9012000F0AE
:1005A000D7F83E480078401CC0B23C490870642827
:1005B0000DDB0020087043A10920F7F7DFFB06E000
:1005C00036480078002802DD0020344908703048A1
:1005D000407810B100202E49487004E02C48407843
:1005E000401C2B49487015F0DBF930B92848807859
:1005F000401C2749887006E03DE02548807810B10E
:100600000020234988702248C07838B1204880787B
:10061000322803DC1E48407864282BDD1C48807893
:10062000322803DD2DA10920F7F7A8FB18484078F0
:10063000642803DD34A10920F7F7A0FB0020174947
:100640000870144908701249C87088704870487161
:10065000114802F051FB1A48007910B1002000F057
:1006600077F800203449087015F098F800211348F5
:10067000FAF768F90AE00020064908700449C870D2
:10068000887000210D48FAF75DF900BF00BF70BD0A
:10069000343F00204D3F0020F06704004C3F002015
:1006A00073686F657320696E746F2067616D652074
:1006B0006D6F6465206661696C000000DD040300F5
:1006C000745300206E6F20676574207269676874C8
:1006D0002073686F6573206461746100496E2067E0
:1006E000616D65206D6F64652C636C69656E742047
:1006F000646973636F6E6E746564206C6F6E6720DF
:1007000074696D6500000000496E2067616D6520A9
:100710006D6F64652C72696768742073686F6573A8
:1007200020646973636F6E6E746564206C6F6E67AE
:100730002074696D65000000413F00200348007887
:100740001E2802D01E20014908707047343F002047
:1007500038B50446009401236A46A2210020F6F72A
:10076000F9FF38BD70B50446002500260C4900206D
:1007700002F0C2FC05460A49012002F0BDFC064613
:100780005DB956B9002002F0FFFA20602068012808
:1007900001DB012070BD0020FCE70020FAE700002B
:1007A0009069040010B504460123094AA1210020E4
:1007B000F6F7D0FF0748007840B9022C06DB054861
:1007C00004700123024AA121F6F7C4FF10BD000006
:1007D000153F0020F03E002010B50123024AA12160
:1007E0000248F6F7B7FF10BD143F0020CC3E0020B2
:1007F0000148007870470000C93E00200148B0F968
:1008000000007047CA3E0020014800787047000091
:10081000C83E002010B50249A120F6F7BDFE10BD6C
:10082000BD44030010B513480078002820DD1149AD
:10083000087800EBD0714910A0EB410121B10E49BD
:100840000720F8F76FFE04E04FF07F410720F8F72C
:1008500069FE08480078142805DB00200549087067
:100860000720F8F78FFE03480078401C0149087004
:1008700010BD000035400020AF0000FF10B5034A56
:1008800003A14FF47A70FAF783F810BDA59802001F
:100890004C6F73735061636B0000000030B58BB018
:1008A0000025182101A8F5F7F5FD0AF0C7F8002882
:1008B0003BD01F480078012837D0FFF7DFFD78BB19
:1008C000002002F061FA05B200242BE001AA2146C3
:1008D000002002F04FFABDF81000ADF81C00BDF882
:1008E0001200ADF81E00BDF81400ADF82000BDF8F0
:1008F0000400ADF82400BDF80600ADF82600BDF8F0
:100900000800ADF82800BDF9281007A804F0C6FFBC
:10091000012806D107484069401C0649486103E0A8
:1009200003E0641CAC42D1DB00BF0BB030BD000063
:10093000183F00207453002070B500251248046849
:1009400012480068844201D204F180740F480068A4
:10095000201A0F49096808440D49086008460068D4
:10096000C50BB4F1807F04D9A4F1807007490860F9
:1009700001E006480460B5F5616F04D30020044926
:100980000860FFF759F970BD04B50040BC3F002076
:10099000B83F002010B5034A03A14FF47A70F9F76D
:1009A000F7FF10BD390903006D6174685F486F750A
:1009B00072000000C0EB00114904014A1160704749
:1009C000B83F002010B50A4A0AA10020F9F7E0FF5D
:1009D0000949A620F6F70CFC0849A620F6F7DCFD2D
:1009E000074A08A14FF4FA70F9F7D2FF10BD0000D2
:1009F000110A03006F7461002541030039440300AC
:100A0000FD0B03006F74615F666C6173680000002A
:100A100010B58CB0002007906348007820B1012801
:100A200061D0022877D17AE060480079002815DD8E
:100A30005F480078012855D15B4908700AF008F832
:100A40000EF061FB42F210715A48FAF72FF80123B9
:100A500007AAA6210020F6F7A1FC43E0564800684B
:100A600001283FD15548007801283BD10020524948
:100A700008605249087014F093FF10B114F058FF49
:100A800001E0FEF7FBF905A8F7F7F4FE0020089057
:100A900009900A900B909DF819009DF818109DF888
:100AA00017209DF81630CDE90032CDE902109DF8EF
:100AB00015309DF8142042A108A8FBF7DBFF08A819
:100AC000F5F7F3FC0446214608A814F06FFF14F074
:100AD00027FF0120344908704FF4FA613548F9F7CF
:100AE000E5FF00BF5CE031480079002805DD00200B
:100AF0002F4908702C49087010E014F051FF58B9C4
:100B0000FEF798F942F210712A48F9F7CFFF022058
:100B10002549087002E03BE014F00AFF40E014F0C1
:100B20003FFF10B100202049087000212148F9F74B
:100B3000BDFFFEF7A3F90020089009900A900B90E2
:100B40001A4890F8381090F8372090F83600174B74
:100B50001B7ACDE90030CDE902211448C3798279AE
:100B600018A108A8FBF786FF08A8F5F79EFC044625
:100B7000214608A814F01AFF19A10E20F7F7FEF875
:100B800014F0CEFEFEF756F900200749087007E082
:100B900000200549087000210648F9F787FF00BFCB
:100BA00000BF0CB010BD00007C3F0020745300203B
:100BB000543F0020110A0300503F0020563F002000
:100BC00046554E5F25303258253032582530325840
:100BD0002530325825303258253032580000000078
:100BE00061647620646973636F6E6E746564206FF0
:100BF0007665722074696D650000000010B51748B5
:100C00000078012822D1F8F7E9FBF7F75FFD18B16A
:100C100013A10E20F7F7B2F8242216491648F5F76B
:100C200020FC002015494876F7F796FC18B114A16E
:100C30000E20F7F7A3F8F7F767FC18B117A10E20FD
:100C4000F7F79CF802200549087006E00348007891
:100C5000022802D104200EF055FF10BD553F0020A0
:100C60006F746120736176652073746570206661AE
:100C7000696C000018500020E45300200854002044
:100C80006F7461207361766520696E666F726D6145
:100C900074696F6E206661696C0000006F7461207A
:100CA00073617665206261636B206661696C000028
:100CB0000148007870470000543F002010B5064AF4
:100CC00006A16420F9F764FE074A08A14FF47A7080
:100CD000F9F75EFE10BD00004DF002004261744461
:100CE000697370616C79000051F2020042617444D2
:100CF000697370616C795F4E0000000010B50C4A9A
:100D00000CA16420F9F744FE104A11A16420F9F700
:100D10003FFE134A13A14FF4FA70F9F739FE144954
:100D2000B120F6F765FA1349B120F6F735FC10BD8E
:100D30003D0E03006170705F706169725F52696798
:100D400068745F50726F636573730000790D030000
:100D50006170705F706169725F4C6566740000005D
:100D600025080300426C696E6B5F666C616700006A
:100D7000A1460300B147030030B589B009F044F83B
:100D800008B909B030BD2348007900B9F9E709F086
:100D900003FB04462048007800282DDD09F0A0FE62
:100DA00010B109F055FE27E000F0C0F800200590D2
:100DB000069007900890174890F8381090F8372060
:100DC00090F83600134B1B7ACDE90030CDE90221B3
:100DD0001048C379827911A105A8FBF74BFE05A83D
:100DE000F5F763FB0546294605A809F07FFE10B913
:100DF00000200949087000BF0F480078002807DD6F
:100E0000012C05D100200C4908700720F8F7BAFB27
:100E100000BFB6E77453002034400020253032581C
:100E20002530325825303258253032582530325846
:100E300025303258000000003540002070B508F021
:100E4000E3FF00B970BD2E48007900B1FAE709F060
:100E5000A3FA04462B48007810B101284CD115E0C4
:100E6000022C01D0032C10D12748FDF755FFFAF7CB
:100E7000B3FB0C2125A009F039FEFAF789FB01200C
:100E80002049087000202449087035E0022C0ED05B
:100E9000032C0CD0FAF7A0FB00201A490870072099
:100EA000F8F770FB09F01CFE08B109F0D1FD1A48F3
:100EB000007800281ADD0020174908700120114928
:100EC00008701148FDF73CFF09F00AFE08B109F06F
:100ED000BFFD8BDF05461148F5F7E7FA06463146B8
:100EE0000E4809F003FEFAF753FB00BF09F0F8FDC6
:100EF00008B1FEF7ADFA00BF00BF00BFA2E70000D7
:100F0000745300203640002065A402002A2A2A2AB1
:100F10002A2A2A2A2A2A2A003340002000550020A3
:100F200001480078704700003440002010B543208D
:100F30001D4981F828000846C06A1C4908611A4802
:100F4000008E8882184890F82800887500200DE0EF
:100F50001549891D0A5C1549091D0A541249333186
:100F60000A5C12490A310A54411CC8B20628EFDB58
:100F7000F7F7CAFA18B10EA10C20F6F7FFFEF7F743
:100F8000CAF818B110A10C20F6F7F8FE1C2106488B
:100F90000C30F5F77FFAF7F7DFFA18B110A10C2043
:100FA000F6F7ECFE10BD000074530020085400203A
:100FB000706169722073617665206261636B757020
:100FC000206661696C0000007061697220636C6565
:100FD00061722073746570206661696C00000000A6
:100FE000466C6173685F53617665496E666F6D61CB
:100FF00074696F6E206661696C00000010B5174857
:10100000407E401C15494876154A16A14FF47A7067
:10101000F9F7BEFC1649AE20F6F7EAF8154A16A114
:101020006420F9F7B5FC1A4890F83200012814D171
:1010300018490820F8F786FA01210E48F9F782FCD2
:10104000222113484185002180F83210F7F784FAF5
:1010500018B111A10D20F6F791FE10BD0854002023
:10106000B51003006170705F736166650000000079
:10107000A14503000DF002006170705F424C455FB6
:101080004C45444F4E5F505552504C4500000000B7
:10109000745300209F009FFF707772207361766504
:1010A00020696E666F726D6174696F6E206661692A
:1010B0006C00000000B58BB01E48007E002812DDD9
:1010C0001D480078401C1C490870084600783C28E0
:1010D00009DB002017490876F7F716FA18B117A1AF
:1010E0000D20F6F74BFE1348407E012820DD282115
:1010F00001A8F5F7CFF9282101A8F5F7CBF9154894
:10110000007930B10B48427E13A101A8FBF7B2FC75
:1011100005E00848427E16A101A8FBF7ABFC01A937
:101120000D20F6F72BFE10B900200249487600BFCB
:101130000BB000BD08540020F03F002073617665BD
:10114000204572725374617274436E7420666169D3
:101150006C000000745300206C6566742073686F27
:10116000657320726573746172743A2564000000BF
:1011700072696768742073686F6573207265737431
:101180006172743A25640000014602290FD10A48B1
:10119000007810B1012807D104E00120064A107040
:1011A000002070470020FCE700BF00BF01E00120E5
:1011B000F7E700BF0120F4E7553F002001484069F0
:1011C0007047000074530020014880697047000098
:1011D0007453002010B50E4A0EA16420F9F7D8FB15
:1011E0001049A520F6F704F80F4A10A16420F9F77A
:1011F000CFFB1349A520F6F7CFF91249012002F0E1
:1012000067F8114A11A16420F9F7C2FB10BD000074
:10121000A1140300737465705F5265616C53656E51
:1012200064000000F94103005D12030073746570EF
:101230005F5265616C436F6E6E6563740000000001
:101240006D440300BD3604009D0803006D617468A1
:101250005F4461696C7953746570000038B5002093
:101260000090002400255048007820B101281CD0AF
:1012700002287DD150E04D480078012808D14A4924
:10128000087000204A4908704A4801F00DFD0BE043
:1012900049480078002807DD0020474908700123ED
:1012A000424AA521F6F756FA7CE04249002001F0B7
:1012B00023FF04463F49012001F01EFF054684B983
:1012C0007DB90220384908703C4840693C490860B3
:1012D00000203C4908603C49088001203B490870D7
:1012E00019E0012C01D1012D15D0324801F0DCFCB0
:1012F0002F480078401C2E490870084600781428B2
:1013000009DB2C4801F0F8FC002027490870274928
:1013100008702E49087045E02B480088401C2A4977
:10132000088008460088B0F5167F10DB0020088092
:10133000009001236A46A521F6F70CFA1D4801F03A
:10134000DBFC0020214908701749087015E01A4895
:101350000078002804DD18480078401E16490870FF
:101360001548007848B90120009001236A4600E042
:1013700010E0A5210020F6F7EDF90C48007840B9FF
:101380000020124908700B4801F0B6FC0020064905
:10139000087007E00020054908700C4908700249F0
:1013A000087000BF00BF38BD303F0020283F00203C
:1013B000313F0020D0670400243F002074530020F8
:1013C0001C3F0020203F0020263F0020183F002027
:1013D0001CB52F480078012858D1002000900190BA
:1013E000002401222146641C0DF80120294840698F
:1013F00029490968401A020E2146641C0DF8012093
:101400002448406924490968401AC0F3074221462C
:10141000641C0DF801201F48808A1F490988401A62
:10142000C0F307222146641C0DF801201948007DF5
:1014300019490978401AC2B22146641C0DF80120EE
:1014400016480068020E2146641C0DF8012013485E
:101450000068C0F307422146641C0DF801200F48C4
:101460000088C0F307222046611CCCB20DF8002092
:101470000A4802782046611CCCB20DF800202346B1
:101480006A46A5210020F5F789FF00BF1CBD0000BA
:10149000183F0020745300201C3F0020203F0020F4
:1014A00010B50448007900B110BDFFF791FF00BFEF
:1014B000FAE700007453002003480078012800D1A7
:1014C00070470020FCE70000183F002010B50249DB
:1014D000AB20F5F78DFE10BDA942030010B5024800
:1014E00006F03AFB10BD0000D04A002010B50346BC
:1014F0000C460AB9072010BD19684A61012C01D1B8
:10150000012000E0002008610020F4E738B513480E
:1015100000680090082358221149124800680DF015
:101520001DF904460CB1204638BD0F4A69460F48E4
:1015300006F018FB04460CB12046F5E701210B48E4
:1015400006F082FB01230A4A1946084806F0D6FA3B
:101550000120084908702046E6E70000D86C040026
:1015600048940020C86C04005F3A0400D04A002070
:10157000FFFF7F00DC4A00202DE9F04106460D46C2
:1015800017463446207F10B10020BDE8F081A761E6
:1015900008F0F8FC401941F10001C4E9020120699A
:1015A00000B125612146002014F0C6FEEDE770B5BC
:1015B00004462546002028772946012014F0BCFE69
:1015C00070BD10B50446204612F0E0FC10BD0000CE
:1015D00070B5044625460E488068B0B1ADB9FCF739
:1015E0004DFE06460A4800680A49086008484068F7
:1015F0004FF0E021C1F804010020054988601EB9C0
:1016000000BF62B600BF00BF00BF00BF70BD0000DA
:101610003094002000E100E0F8B505460C4617467E
:101620002088001DB84201D90C20F8BD684679DF3A
:10163000064600BF304600B1F7E700BF032021880F
:1016400068542088401C20801920218868542088F4
:10165000401C208020884119BDF8000014F0ADFE28
:101660002188084420800020DFE710B541EC100BF2
:10167000FBF7EAFC51EC100B10BD2DE9F0412DED0C
:10168000028B04460E4617461D46B0EE408AB0EE69
:10169000000A86ED000A95ED020A20EE080A86EDA2
:1016A000010A95ED010AF1EE480A20EE200A86EDC6
:1016B000020A95ED020AF1EE480A20EE200A86EDB4
:1016C000030AB0EE000A86ED040A95ED000A20EE4A
:1016D000080A86ED050A95ED010A20EE080A86ED56
:1016E000060A95ED000AF1EE480A20EE200A86ED82
:1016F000070AB0EE000A86ED080A394630460AF0BD
:101700007FF924213046F4F7C5FE94ED010A20EE5E
:10171000080AD5ED020A20EE200AD4ED000AB0EE48
:10172000001A01EE200AD4ED020A60EE880A95ED57
:10173000011A00EEC10A86ED000A94ED010AF0EEEE
:10174000000A20EE200AD4ED000A60EE880A95ED2A
:10175000021A00EEC10AD4ED020A60EE880A95ED85
:10176000001A00EE810A86ED010A94ED000A20EECF
:10177000080AD5ED010A20EE200AD4ED020AB0EEE7
:10178000001A01EE200AD4ED010A60EE880A95EDF8
:10179000001A00EEC10A86ED020A94ED040A20EE5A
:1017A000080AD5ED020A20EE200AD4ED030AB0EEB5
:1017B000001A01EE200AD4ED050A60EE880A95EDC4
:1017C000011A00EEC10A86ED030A94ED040AF0EE58
:1017D000000A20EE200AD4ED030A60EE880A95ED97
:1017E000021A00EEC10AD4ED050A60EE880A95EDF2
:1017F000001A00EE810A86ED040A94ED030A20EE39
:10180000080AD5ED010A20EE200AD4ED050AB0EE53
:10181000001A01EE200AD4ED040A60EE880A95ED64
:10182000001A00EEC10A86ED050A94ED070A20EEC3
:10183000080AD5ED020A20EE200AD4ED060AB0EE21
:10184000001A01EE200AD4ED080A60EE880A95ED30
:10185000011A00EEC10A86ED060A94ED070AF0EEC1
:10186000000A20EE200AD4ED060A60EE880A95ED03
:10187000021A00EEC10AD4ED080A60EE880A95ED5E
:10188000001A00EE810A86ED070A94ED060A20EEA2
:10189000080AD5ED010A20EE200AD4ED080AB0EEC0
:1018A000001A01EE200AD4ED070A60EE880A95EDD1
:1018B000001A00EEC10A86ED080A22463946304673
:1018C0000CF06DFCBDEC028BBDE8F0812DE9F04120
:1018D0000446501E34F9105034F9106031F910707C
:1018E00031F910C0132018E034F91080A84501DD4B
:1018F00034F9105034F91080B04501DA34F9106031
:1019000031F91080B84501DD31F9107031F91080DE
:10191000E04501DA31F910C0401EC2F114088045DB
:10192000E2DDF018A84203DB0CEB0300B84202DA58
:101930000120BDE8F0810020FBE72DE9F0410446DD
:101940000F46154615B90E20BDE8F081002028602D
:1019500000BF0CB90E20F7E700BF00BF206808B930
:101960000E20F1E700BF00BFE088C11700EB9171C6
:101970008910A0EB810109B10720E5E700BF3846D7
:1019800000F0DEFAC6B2142E01D10520DCE7207982
:10199000B04201DC0420D7E7E188206806FB0100A3
:1019A00028600020D0E72DE9FC4105468846164610
:1019B000002437880020308095F82D0058B13A4631
:1019C0003146404600F08AFB044600BF204608B17D
:1019D000BDE8FC8100BFA87850B13A463146404688
:1019E000FFF71AFE044600BF204600B1F0E700BF33
:1019F000E87860B1E97848B23B463246414606F0A5
:101A0000D0FC044600BF204600B1E1E700BF686893
:101A100068B1696891F900003B463246414614F0CE
:101A2000ABFC044600BF204600B1D1E700BF2889C7
:101A300000280EDD43460622022105F10800CDE90B
:101A4000006714F02DFD044600BF204600B1BFE73B
:101A500000BF288A00280EDD43460722032105F136
:101A60001000CDE9006714F01BFD044600BF2046BE
:101A700000B1ADE700BF288B00280EDD43461522DC
:101A8000142105F11800CDE9006714F009FD0446A2
:101A900000BF204600B19BE700BF286A58B13B4613
:101AA00032464146286A03F0D4FA044600BF204675
:101AB00000B18DE700BF686A58B13B4632464146E7
:101AC000686A0BF06BFA044600BF204600B17FE75E
:101AD00000BF95F82C0000280BDD3B4632464146FE
:101AE000284613F055FC044600BF204600B16FE7BE
:101AF00000BF287858B13B463246414628460CF094
:101B000003FC044600BF204600B161E700BF204649
:101B10005EE72DE9F843064688461546002000900A
:101B20000DB9BDE8F88309236A464146304600F006
:101B30002BF80446BDF800003718BDF8000068B166
:101B400064B12846F4F7B1FCA04207D122463946D9
:101B50002846F4F7BFFC08B90120E2E70020E0E7DF
:101B6000F8B504460E461546002000902B466A46FE
:101B70003146204600F008F807460FB90020F8BDAE
:101B8000BDF800002044FAE7F0B504460D461E46B5
:101B900004B10AB90020F0BD002103E0605C401CE4
:101BA000084481B2481CA84206DA10888842F5DC55
:101BB000481C205CB042F1D1A94201DB0020EAE7D9
:101BC000881C87B2605C10B1605C401E00E00020A1
:101BD00083B213B1F818A84201DD0020DBE71780BB
:101BE0001846D8E780F83010704770B504460D46A7
:101BF00005B10CB90E2070BD05F1780003F041F974
:101C000008B90720F7E70020A0702C2205F1780121
:101C1000201DF4F726FC002084F83000D5F8A4003D
:101C20006063D5F8A800A0634FF6FF70A4F8240401
:101C300004F58260C4F82004002140F22C40C4F86E
:101C40002614A4F82A140155207810B9FF2084F82E
:101C5000540004F15500C4F810042046FDF752F872
:101C600040F21441085304F2144204F1550128468D
:101C7000FFF799FE064600BF304600B1BBE700BF44
:101C800004F231204FF4836108512046FDF73AF801
:101C9000A4F81C044FF48360015904F21C4205F1BE
:101CA0003C00FFF780FE064600BF304600B1A2E7C9
:101CB00000BF012151200155208B81B248200153E2
:101CC000012084F83C000021216450200155616905
:101CD000616404F13C02002104F1540072DF064605
:101CE00000BF304600B186E700BF012020703046BB
:101CF00081E770B504460D462E462088102804D092
:101D0000112807D026280FD109E0214630460FF0D0
:101D100017FE0AE0214630460FF08DFF05E0214610
:101D2000304610F06BF900E000BF00BF70BD70B529
:101D300004460E46207808B9082070BDA670002120
:101D400040F22C40C4F82614A4F82A140155A079B6
:101D500010B1A078012809D0E07910B1A07801284D
:101D600004D0E07970B1A07802280BD1606B30B15B
:101D7000012084F82D040820616B884702E00020D0
:101D800084F82D0431462046FCF76CFFA070606B90
:101D9000A0B1A078032802D0A07804280ED16079E1
:101DA00060B194F82E0448B9002084F83004012072
:101DB00084F82F040720616B884702E0002084F834
:101DC0002F04182104F13C00F4F764FB012084F88F
:101DD0003C0004F12C0010F023FC20B194F82C10EE
:101DE0005120015502E001215120015594F82400B1
:101DF00060B104F1280010F013FC20B194F8281011
:101E00005220015502E001215220015500215020AD
:101E10000155A078052824D2DFE800F01F030A113D
:101E2000180004F13C01204613F0B0FB054619E010
:101E300004F13C01204613F091FB054612E004F149
:101E40003C01204613F0B4FB05460BE004F13C01D5
:101E5000204613F0DBFB054604E0002084F8310047
:101E600000E000BF00BFA07898B104F13C0204F18B
:101E70005400D4F8201472DF05460DB128465CE703
:101E800094F8301094F8540073DF05460DB12846DD
:101E900053E7606B18B194F83100616B88470020FC
:101EA0004BE700002DE9F041044600BF14B90E20B5
:101EB000BDE8F08100BF1C2221461C48F4F7D1FA8E
:101EC0001B481A490860206860B120687ADF05461F
:101ED0000DB12846ECE7164821680A680260496897
:101EE000416005E012487BDF05460DB12846DFE77B
:101EF000002617E006EB86000E4901EB800700BFC5
:101F00004FF6FF70388000BF0B4800EB461078603A
:101F10000A4A0021381DFFF7E9FA05460DB10320F2
:101F2000C6E7761C002EE5D00020C1E74C930020C8
:101F30009A4A00203893002018930020C9630400B7
:101F400010B50446204600F01BF808B1204610BD2D
:101F50001420FCE770B504460025204600F010F878
:101F600050B1214605480CF054FC06460EB1022043
:101F700000E00120054600BF284670BDA492002065
:101F800010B50446142C01DB002010BD2146024888
:101F90000CF03FFCF9E700009C92002010B50446CD
:101FA00000BF0CB90E2010BD00BF00BF064800786E
:101FB000012801D00820F6E700BF04480168204648
:101FC00011F066FCEFE70000984A00208C4A0020E0
:101FD0000146002200BF09B90E20704700BF00BFB4
:101FE000086808B90E20F8E700BF00BF486808B9C4
:101FF0000E20F2E700BF0020064B18600120064BC0
:102000001870064B08681860054B48681860104641
:10201000E3E70000944A0020984A00208C4A002000
:10202000904A002070B504460D4600BF04B970BD4B
:1020300000BF00BF05B9FAE700BF00BF1448007831
:10204000012800D0F3E700BF2E462088112815D0C4
:10205000302804D0322807D0332814D109E0211DBC
:1020600030460FF0D7FE0FE0211D30460FF00CFB7D
:102070000AE0211D30460FF01DFD05E0211D304610
:102080000FF0CCFD00E000BF00BF00BFCFE70000B5
:10209000984A002070B504460D4600BF0CB90E20CA
:1020A00070BD00BF00BF0B480078012801D0082098
:1020B000F6E700BF0848006808B90820F0E794F880
:1020C000C80208B11120EBE72946204603F0C0FF03
:1020D000E6E70000984A0020944A00202DE9FC41E0
:1020E00005460C46174620880930B84202D90C2014
:1020F000BDE8FC8168466DDF064600BF304600B192
:10210000F6E700BF0820218868542088401C208002
:102110001B20218868542088401C20802088284467
:10212000DDF801100160BDF8051081802088801D58
:1021300020809DF80000400818B9002021886854CC
:1021400002E00120218868542088401C2080002063
:10215000CEE7000070B50DF02DF8044600BF204614
:1021600000B170BD00BF00BF084D28464FF0030C02
:1021700000DF00BF044600BF204600B1F1E700BF0A
:102180000DF032F804462046EBE70000CC94002026
:10219000014600BF09B90E20704700BF0148016029
:1021A0000020F9E7044B002010B54FF0FF3100206C
:1021B0003DDF044600BF204600B110BD00BFB12185
:1021C00000203CDF044600BF204600B1F5E700BF19
:1021D000044841690120884702200DF093FC00204B
:1021E000EBE70000B094002010B505480068416995
:1021F00000208847FFF7D8FF0446204610BD0000A6
:10220000044B002010B588B0044620216846F4F73E
:1022100041F90320ADF8000020788DF802009DF808
:102220000D0020F0200020308DF80D009DF80D00ED
:1022300020F0080008308DF80D0001208DF8100006
:102240008DF80C001720ADF8040001208DF8130064
:102250008DF812008DF811006088A21D694602F009
:1022600027FC08B010BD000030B585B00546244BF2
:102270000FCB8DE80F0000BF15B90E2005B030BDA3
:1022800000BF4FF6FF701F49888028684861002012
:1022900008760846406908B91B4848611948FFF7A5
:1022A00077FF044600BF204600B1E7E700BF00BF4C
:1022B00001208DF812004FF65960ADF8100000BFF4
:1022C000104A921C04A90120A8DF044600BF204642
:1022D00000B1D3E700BF0B49684662DF044600BF88
:1022E000204600B1CAE700BF0648FFF78BFF04464F
:1022F00000BF204600B1C1E700BF0020BEE70000DC
:10230000946D0400B0940020B17F030070B50446C2
:102310000D4600BF04B970BD00BF2088102806D04C
:10232000112808D051280AD0532810D10BE020469C
:102330000FF0FCFA0CE020460FF062FC08E02046AB
:102340000FF0AAFD04E020460FF000FD00E000BF02
:1023500000BF00BFDFE7000070B505460426287BFC
:10236000012804D0022818D003282ED10AE0012029
:1023700005F020FE04460CB9012602E0112C00D124
:10238000062624E0032005F015FE04460CB90126BC
:1023900002E0112C00D1062619E0687B142801DC2C
:1023A000687B08B905260FE06A7B05F10E0112482B
:1023B000F4F757F8687B1049091F8861084613F045
:1023C00053F9044604B9012601E0022600BF00BF0C
:1023D000012E0FD0287B314600F058F8044624B176
:1023E000064800684169032088470448006841693D
:1023F0000220884770BD0000DC940020044B0020C0
:1024000070B505460E4600BF1E48006820B11D4845
:10241000406808B1012000E0002000B970BD00BF95
:10242000184800F10801426828469047044600BF5A
:10243000082C24D07CB90020134909684876012172
:10244000022000F023F80446CCB10F48006841692F
:102450000320884713E000200B49096848760621CD
:10246000022000F013F8044624B1074800684169CF
:10247000032088470448006841690220884700BF5C
:10248000CCE70000CC940020044B0020F0B587B0CE
:1024900004460D460327002001900290039004900B
:1024A0000320069020208DF814008DF815408DF83B
:1024B00016500E48C088ADF8040002208DF80600C2
:1024C0000020ADF8080006A8039005A8049007496D
:1024D000888801A9AEDF064626B9BDF81800032892
:1024E00000D00C26304607B0F0BD0000B0940020AC
:1024F00030B1012805D0022804D0032807D102E01A
:1025000006E005E004E000BF002100BF00E000BFDE
:1025100000BF70472DE9F04104460F46A6883046BB
:10252000FFF718FD0546012D03D0204600F0ACF85A
:1025300018B120460EF080FF08E0022D02D020885E
:102540001D2803D1002120460EF082FEBDE8F08157
:102550002DE9F04104460F46A6882088102806D0B1
:10256000112819D019283FD01A284AD118E011F0A3
:1025700041F9304611F01AF930B900BF22A2F0211A
:102580000420F3F747FE06E0E07B022803D1314642
:102590002C480CF04DF934E0304611F04FF930E0A2
:1025A000207A0509042D01DB012000E0002002460D
:1025B000314624480C3005F0E5FE032D01DB0120F7
:1025C00000E00020024631461E48083005F0DAFEE1
:1025D000022D01DB012000E00020024631461948AF
:1025E000001D05F0CFFE0CE0207A48B9607AC0F3F8
:1025F000C0052A46314613480C3005F0C3FE00BF23
:1026000000BF00BFBDE8F0812E2E5C2E2E5C2E2E6A
:102610005C2E2E5C2E2E5C2E2E5C636F6D706F6EAA
:10262000656E74735C626C655C636F6D6D6F6E5C20
:10263000626C655F636F6E6E5F73746174652E6349
:1026400000000000A492002070B504460D462088CA
:10265000102806D0112808D012280ED0502810D1EA
:1026600007E020460FF0F0F80CE020460FF0AFFA3C
:1026700008E020460FF0F4FC04E020460FF0CCF810
:1026800000E000BF00BF70BD01460888262801D1C8
:10269000012070470020FCE710B5002408E007483F
:1026A00050F8240018B1054951F824008047641CF3
:1026B000034800788442F2DB10BD0000488200200D
:1026C0003C48002010B5002408E0074850F82400DA
:1026D00018B1054951F824008047641C034800786C
:1026E0008442F2DB10BD0000548200203D480020EF
:1026F0002DE9F04107460C46207820B1012824D06E
:10270000022829D127E0618804F10E02384600F042
:1027100035F8054600BF2E4636B100BF10A287210E
:102720003046F3F777FD00BF00BF384600F02EF9C2
:10273000054600BF2E4636B100BF09A28A213046A9
:10274000F3F768FD00BF00BF06E0A1890A4AA06850
:102750001268904700E000BF00BFBDE8F0810000B4
:102760002E2E5C2E2E5C2E2E5C626C655F6366677F
:102770005C686F73742E63003042002070B50446AD
:102780000E46154600BF0CB90E2070BD00BF268155
:102790002DB16988A18128886081A988E1813146AD
:1027A000A0690CF071F9F0E770B586B004460D46EB
:1027B0001A4B0FCB01AE0FC600BF14B90E2006B0E6
:1027C00070BD00BF00BF0DB90E20F8E700BF00BF0D
:1027D000A86808B90E20F2E700BFE11D01A862DF7A
:1027E000064600BF304600B1E9E700BFE0798DF84A
:1027F00016000120ADF814004FF6FF702081286804
:10280000206168686061002060810021E181A86822
:10281000A06105A8FFF7C2FBD1E70000886B0400A8
:1028200070B586B005460E46344604B10DB906B003
:1028300070BD20894FF6FF71884203D02089A98896
:10284000884200D0F3E72888112806D0392816D10D
:10285000294620460FF090FA12E0A8882189884284
:102860000CD1206950B102208DF804004FF6FF70A2
:10287000208101A920462269904700BF00E000BFE7
:1028800000BF00BFD3E770B586B005460C461421E3
:1028900001A8F3F7FFFD04F10E06207800283AD1D5
:1028A000A088012837D1A079E979884233D1002066
:1028B00022E000EBC00136F81110022902D00329F2
:1028C00017D107E000EBC00106EB41010A89ADF822
:1028D00016200FE000EBC00106EB41010989ADF8BD
:1028E000121000EBC00106EB41014A89ADF814203B
:1028F00000E000BF00BF401C217A8142D9D828697E
:1029000048B16088ADF8060000208DF8040001A9E8
:1029100028462A69904706B070BD000070B588B09F
:1029200004460E46154600BF14B90E2008B070BD0F
:1029300000BF20216846F3F7ADFDB62D01DD07206D
:10294000F4E720894FF6FF71884201D10820EDE7B6
:1029500001208DF800000C4802900394E189ADF845
:102960001210ADF816500021ADF814100696022092
:102970008DF8100001218DF8111022896946A06997
:102980000CF0ACF8D2E70000CD9C030010B5044673
:1029900000BF0CB90E2010BD00BF20894FF6FF719B
:1029A000884201D0A08908B90820F4E70121204617
:1029B00002F04EF8EFE72DE9F04186B00446884674
:1029C00017461D4600BF1CB90E2006B0BDE8F081B9
:1029D00000BF01AA29466069FEF7AFFF064600BFA7
:1029E000304600B1F1E700BF4FF6FF70854201D0DD
:1029F000019808B90520E8E70198007808B908208F
:102A0000E3E73888B62801DD0720DEE700200290E2
:102A1000039004900590A088ADF80800CDF81480CC
:102A2000049701208DF80A0002A92846AEDFCCE702
:102A300070B58EB004460E463E4B0FCB09AD0FC5A8
:102A400000BF14B90E200EB070BD00BF00BF0EB99C
:102A50000E20F8E700BF3068A061214609A862DFB8
:102A6000054600BF284600B1EDE700BF20788DF88D
:102A700036000120ADF83400A21C0DA9A8DF0546E0
:102A800000BF284600B1DEE700BF202101A8F3F710
:102A900001FD0220ADF8040020788DF80600B62074
:102AA000ADF808000120ADF80A008DF810009DF87F
:102AB000110020F0080008308DF811009DF8110079
:102AC00020F00400001D8DF8110001208DF8150084
:102AD0008DF81600608804F10C0201A901F0E8FFEE
:102AE00005460DB12846AEE7202101A8F3F7D2FC38
:102AF0000320ADF8040020788DF80600B620ADF86C
:102B000008000120ADF80A008DF810009DF81100B2
:102B100020F0100010308DF8110001208DF8150004
:102B20008DF816008DF817006088221D01A901F0AC
:102B3000BFFF88E7986B040070B504460D4605B1E9
:102B400004B970BD2E462088102804D0502807D024
:102B500057280FD109E0214630460EF0ADFE0AE0BD
:102B6000214630460FF0A8FA05E0214630460FF026
:102B70001FF900E000BF00BF00BFE2E710B500246E
:102B800008E0074850F8240018B1054951F824001E
:102B90008047641C034800788442F2DB10BD0000CB
:102BA000B07F00200242002010B5002408E0074852
:102BB00050F8240018B1054951F824008047641CDE
:102BC000034800788442F2DB10BD0000F07F002053
:102BD0000342002070B50446204613F0E8FB05468A
:102BE000C5F3400070BD70B50446204613F0DFFB0E
:102BF000054605F0010070BD38B50DF00BFA04462E
:102C000000BF25463DB100BF15A240F2CD112846B8
:102C1000F3F700FB00BF00BF0020009069460120D1
:102C20000DF02CF9044600BF25463DB100BF0CA2B3
:102C300040F2D3112846F3F7EDFA00BF00BF684613
:102C40000DF07AF9044600BF25463DB100BF04A24D
:102C500040F2D7112846F3F7DDFA00BF00BF38BDB8
:102C60002E2E5C2E2E5C2E2E5C626C655F6366677A
:102C70005C686F73742E630010B5002405F0C8FC07
:102C8000401C00B9641E70210648F3F703FC0020C5
:102C9000044981F86E00601C10B94FF0FF3010BD80
:102CA0000020FCE7AC72002070B504460CB900208F
:102CB00070BD002509E00F4850F82500A04203D15F
:102CC00000F056FB2046F3E76D1C0C2DF3DB0025CE
:102CD0000BE0084850F8250030B9064840F8254078
:102CE00000F046FB2046E3E76D1C0C2DF1DB0020D5
:102CF000DEE70000AC72002070B5054615B94FF054
:102D0000FF3070BD00240DE0094850F82400A842AF
:102D100007D10020064941F8240000F029FB0020DB
:102D2000EFE7641C0C2CEFDB6FF00100E9E700001B
:102D3000AC72002010B5002005F04AFD0446601C6E
:102D400010B94FF0FF3010BD012005F041FD0446E1
:102D5000601C10B94FF0FF30F5E770210448F3F71D
:102D600099FB0020024981F86E0000BFEBE70000EC
:102D7000AC72002070B504460D4616463246294610
:102D8000204605F093FD70BD10B50446204605F0C1
:102D9000ABFD10BD10B5024602B111B94FF0FF30C6
:102DA00010BD002067E100EB400303EBC0031344B8
:102DB0001B7A00EB400404EBC0040C44247AA342C9
:102DC00006DD00EB400303EBC00313441B7A05E070
:102DD00000EB400303EBC0030B441B7A00EB400401
:102DE00004EBC0041444237200EB400303EBC00364
:102DF00013445B7900EB400404EBC0040C44647999
:102E0000A34206DD00EB400303EBC00313445B79F0
:102E100005E000EB400303EBC0030B445B7900EBE0
:102E2000400404EBC0041444637100EB400303EB63
:102E3000C003D35C00EB400404EBC0040C5DA34270
:102E400005DD00EB400303EBC003D35C04E000EBC3
:102E5000400303EBC003CB5C00EB400404EBC00475
:102E6000135500EB400303EBC00313449B7800EBC6
:102E7000400404EBC0040C44A478A34206DD00EB3C
:102E8000400303EBC00313449B7805E000EB4003D1
:102E900003EBC0030B449B7800EB400404EBC0043D
:102EA0001444A37000EB400303EBC00313445B7AAC
:102EB00000EB400404EBC0040C44647AA34206DD3A
:102EC00000EB400303EBC00313445B7A05E000EB27
:102ED000400303EBC0030B445B7A00EB400404EBBC
:102EE000C0041444637200EB400303EBC0031344BB
:102EF0009B7900EB400404EBC0040C44A479A3428A
:102F000006DD00EB400303EBC00313449B7905E0AF
:102F100000EB400303EBC0030B449B7900EB400440
:102F200004EBC0041444A37100EB400303EBC003A3
:102F300013445B7800EB400404EBC0040C44647859
:102F4000A34206DD00EB400303EBC00313445B78B0
:102F500005E000EB400303EBC0030B445B7800EBA0
:102F6000400404EBC0041444637000EB400303EB23
:102F7000C00313449B7A00EB400404EBC0040C44F0
:102F8000A47AA34206DD00EB400303EBC003134425
:102F90009B7A05E000EB400303EBC0030B449B7AF4
:102FA00000EB400404EBC0041444A37200EB4003A4
:102FB00003EBC0031344DB7900EB400404EBC004D3
:102FC0000C44E479A34206DD00EB400303EBC003AD
:102FD0001344DB7905E000EB400303EBC0030B4433
:102FE000DB7900EB400404EBC0041444E37100EB14
:102FF000400303EBC0031344DB7800EB400404EB15
:10300000C0040C44E478A34206DD00EB400303EB6C
:10301000C0031344DB7805E000EB400303EBC0037F
:103020000B44DB7800EB400404EBC0041444E37071
:1030300000EB400303EBC00313441B7900EB400497
:1030400004EBC0040C442479A34206DD00EB4003EA
:1030500003EBC00313441B7905E000EB400303EBD3
:10306000C0030B441B7900EB400404EBC004144480
:103070002371431CD8B20228FFF695AE00208FE6DC
:1030800010B502460020137A0C7AA34200D0401CEF
:1030900053794C79A34200D0401C13780C78A3429A
:1030A00000D0401C93788C78A34200D0401C537A07
:1030B0004C7AA34200D0401C93798C79A34200D073
:1030C000401C53784C78A34200D0401C937A8C7AF1
:1030D000A34200D0401CD379CC79A34200D0401C3D
:1030E000D378CC78A34200D0401C13790C79A3424A
:1030F00000D0401C10BD0000F0B506460D460DB1D5
:10310000022E01DB0220F0BD29686A68554B03F1ED
:103110000B0416B1012E71D14DE00F7A93F808C05F
:10312000674501DD0220EEE74F7993F805C067455A
:1031300001DD0220E7E70F7893F800C0674501DD65
:103140000220E0E78F7893F802C0674501DD022096
:10315000D9E74F7A93F809C0674501DD0220D2E72D
:103160008F7993F806C0674501DD0220CBE74F78E1
:1031700093F801C0674501DD0220C4E78F7A93F818
:103180000AC0674501DD0220BDE7CF7993F807C08B
:10319000674501DD0220B6E7CF7893F803C06745A5
:1031A00001DD0220AFE70F7993F804C0674501DD28
:1031B0000220A8E74FE0177A94F808C0674501DDC0
:1031C0000220A0E7577994F805C0674501DD022089
:1031D00099E7177894F800C0674501DD022092E76F
:1031E000977894F802C0674501DD02208BE7577A93
:1031F00094F809C0674502DD022084E72AE0977948
:1032000094F806C0674501DD02207CE7577894F802
:1032100001C0674501DD022075E7977A94F80AC07E
:10322000674501DD02206EE7D77994F807C067454E
:1032300001DD022067E7D77894F803C0674501DD18
:10324000022060E7177994F804C0674501DD022089
:1032500059E700E000BF00BF024F583F97F86E00EB
:1032600000BF50E704730020411C21B90021174A18
:1032700082F86E1028E0042804D10521134A82F850
:103280006E1021E0052804D10321104A82F86E1047
:103290001AE0062804D104210C4A82F86E1013E0CB
:1032A000102804D10721094A82F86E100CE01A2870
:1032B00006D3411C21B10821044A82F86E1003E0B4
:1032C0000621024A82F86E1070470000AC7200209E
:1032D00002460B460BB1022A02DB4FF0FF3070476B
:1032E00000210BE0114800EBC1004068984204D176
:1032F0000E4800F831200020F1E7491C0529F1DBD8
:1033000000210EE0094800EBC100406840B90748C1
:1033100000EBC1004360054800F831200020DEE7E3
:10332000491C0529EEDB4FF0FF30D8E7DC720020A6
:1033300070B50646012515E0002410E00B4810F892
:103340003400A8420AD1094800EBC400406828B103
:10335000064800EBC400416830468847641C052CD1
:10336000ECDB6D1E002DE7DA70BD0000DC72002082
:10337000FEB5FF25002400BF0CE004EB440000EB89
:10338000C401374808440021016041600181817215
:10339000601CC4B2022CF0DB002414E03048583822
:1033A00050F8240068B12E48583850F824000168BD
:1033B0002B48FFF7EFFC0546681C10B94FF0FF30B3
:1033C000FEBD601CC4B20C2CE8DB6946002005F091
:1033D00053FA23496846FFF753FE07466946012022
:1033E00005F04AFA1E490B316846FFF749FE0646CA
:1033F0001FB916B94FF0FF30E2E71949002005F078
:1034000021FA0546681C10B94FF0FF30D8E714497F
:103410000B31012005F016FA0546681C10B94FF073
:10342000FF30CDE70F4805F083FF0546681C10B953
:103430004FF0FF30C4E70C4805F086FF0546681CD6
:1034400010B94FF0FF30BBE705F08AFF054625B9FC
:1034500001200349583981F86E000020B0E70000D0
:1034600004730020693203003133030070B5042572
:1034700025480078012845D1002023490870002103
:103480002248F7F75FFAF4F746FEFF22942120481E
:10349000F2F7F9FFFF221C211E48F2F7F4FF1E4845
:1034A0001B49086022211A484185012180F8321009
:1034B000F5F72AF818B119A10D20F4F75FFCF5F71C
:1034C0004BF818B11BA10D20F4F758FC012004F0B3
:1034D00071FD04460CB9012502E0112C00D106252E
:1034E000012D0FD029460120FEF7D0FF044624B15C
:1034F00017480068416903208847154800684169FA
:103500000220884770BD0000084B00206D34030086
:103510007453002008540020AA5555AA70777220D1
:1035200073617665206261636B7570206661696C9A
:1035300000000000707772207361766520696E6606
:103540006F726D6174696F6E206661696C00000056
:10355000044B002010B5034A03A16420F7F718FAC2
:1035600010BD00006D3403006273705F626C655FB4
:103570006466755F70726F636573730010B504A144
:103580001720F4F7FBFB10B90748F7F76BFA10BDEB
:103590006273705F70776D5F696E69745F65727278
:1035A0006F720D0A000000007D35030010B504A104
:1035B0001920F4F7E3FB10B90748F7F753FA10BDE9
:1035C0006273705F7274635F636F6E6669675F6575
:1035D00072726F720D0A0000AD35030010B504A1C0
:1035E0001920F4F7CBFB10B90748F7F73BFA10BDE9
:1035F0006273705F7274635F696E69745F65727223
:103600006F720D0A00000000DD35030010B504A143
:103610001320F4F7B3FB10B90748F7F723FA10BDEE
:103620006273705F737069305F696E69745F657231
:10363000726F720D0A0000000D36030010B504A170
:103640001820F4F79BFB10B90748F7F70BFA10BDE9
:103650006273705F7764745F696E69745F657272BC
:103660006F720D0A000000003D36030030B50346BE
:103670000C4600201FE09FED110A02EB800181ED56
:10368000000A002114E002EB800595ED000A01EB31
:10369000800503EB8505D5ED000A04EB810595ED6A
:1036A000001A00EE810A02EB800585ED000A491C34
:1036B0000429E8DB401C0928DDDB30BD00000000E8
:1036C00030B5A1B005460C4694ED140A8DED010A03
:1036D00094ED180A8DED020A94ED190A8DED030A96
:1036E00094ED1A0A8DED040A94ED380A8DED050A61
:1036F00094ED3C0A8DED060A94ED3D0A8DED070A26
:1037000094ED3E0A8DED080A94ED410A8DED090A0B
:1037100094ED450A8DED0A0A94ED460A8DED0B0AEB
:1037200094ED470A8DED0C0A94ED4A0A8DED0D0AD1
:1037300094ED4E0A8DED0E0A94ED4F0A8DED0F0AB1
:1037400094ED500A8DED100A002012E001A901EB62
:10375000001101EB800191ED000ADFEDFE0A30EE71
:10376000200A01A901EB001101EB800181ED000AA3
:10377000401C0428EADB11A901A809F04BFC94EDD8
:10378000020ADDED110A20EE200AD4ED060A9DEDB5
:10379000151A00EE810AD4ED070A9DED191A00EE04
:1037A000810AD4ED080A9DED1D1A00EE810A85ED0F
:1037B000000A94ED020ADDED120A20EE200AD4ED93
:1037C000060A9DED161A00EE810AD4ED070A9DED5A
:1037D0001A1A00EE810AD4ED080A9DED1E1A00EEB9
:1037E000810A85ED010A94ED020ADDED130A20EE4F
:1037F000200AD4ED060A9DED171A00EE810AD4EDD9
:10380000070A9DED1B1A00EE810AD4ED080A9DED12
:103810001F1A00EE810A85ED020A94ED020ADDED21
:10382000140A20EE200AD4ED060A9DED181A00EEC7
:10383000810AD4ED070A9DED1C1A00EE810AD4ED31
:10384000080A9DED201A00EE810A85ED030A94ED29
:103850000B0ADDED110A20EE200AD4ED0F0A9DEDD2
:10386000151A00EE810AD4ED100A9DED191A00EE2A
:10387000810AD4ED110A9DED1D1A00EE810A85ED35
:10388000040A94ED0B0ADDED120A20EE200AD4EDB5
:103890000F0A9DED161A00EE810AD4ED100A9DED77
:1038A0001A1A00EE810AD4ED110A9DED1E1A00EEDF
:1038B000810A85ED050A94ED0B0ADDED130A20EE71
:1038C000200AD4ED0F0A9DED171A00EE810AD4EDFF
:1038D000100A9DED1B1A00EE810AD4ED110A9DED30
:1038E0001F1A00EE810A85ED060A94ED0B0ADDED44
:1038F000140A20EE200AD4ED0F0A9DED181A00EEEE
:10390000810AD4ED100A9DED1C1A00EE810AD4ED57
:10391000110A9DED201A00EE810A85ED070A94ED4B
:10392000140ADDED110A20EE200AD4ED180A9DEDEF
:10393000151A00EE810AD4ED190A9DED191A00EE50
:10394000810AD4ED1A0A9DED1D1A00EE810A85ED5B
:10395000080A94ED140ADDED120A20EE200AD4EDD7
:10396000180A9DED161A00EE810AD4ED190A9DED94
:103970001A1A00EE810AD4ED1A0A9DED1E1A00EE05
:10398000810A85ED090A94ED140ADDED130A20EE93
:10399000200AD4ED180A9DED171A00EE810AD4ED25
:1039A000190A9DED1B1A00EE810AD4ED1A0A9DED4D
:1039B0001F1A00EE810A85ED0A0A94ED140ADDED66
:1039C000140A20EE200AD4ED180A9DED181A00EE14
:1039D000810AD4ED190A9DED1C1A00EE810AD4ED7E
:1039E0001A0A9DED201A00EE810A85ED0B0A94ED6E
:1039F0001D0ADDED110A20EE200AD4ED210A9DED0D
:103A0000151A00EE810AD4ED220A9DED191A00EE76
:103A1000810AD4ED230A9DED1D1A00EE810A85ED81
:103A20000C0A94ED1D0ADDED120A20EE200AD4EDF9
:103A3000210A9DED161A00EE810AD4ED220A9DEDB1
:103A40001A1A00EE810AD4ED230A9DED1E1A00EE2B
:103A5000810A85ED0D0A94ED1D0ADDED130A20EEB5
:103A6000200AD4ED210A9DED171A00EE810AD4ED4B
:103A7000220A9DED1B1A00EE810AD4ED230A9DED6A
:103A80001F1A00EE810A85ED0E0A94ED1D0ADDED88
:103A9000140A20EE200AD4ED210A9DED181A00EE3A
:103AA000810AD4ED220A9DED1C1A00EE810AD4EDA4
:103AB000230A9DED201A00EE810A85ED0F0A94ED90
:103AC000260ADDED110A20EE200AD4ED2A0A9DED2A
:103AD000151A00EE810AD4ED2B0A9DED191A00EE9D
:103AE000810AD4ED2C0A9DED1D1A00EE810A85EDA8
:103AF000100A94ED260ADDED120A20EE200AD4ED1C
:103B00002A0A9DED161A00EE810AD4ED2B0A9DEDCE
:103B10001A1A00EE810AD4ED2C0A9DED1E1A00EE51
:103B2000810A85ED110A94ED260ADDED130A20EED7
:103B3000200AD4ED2A0A9DED171A00EE810AD4ED71
:103B40002B0A9DED1B1A00EE810AD4ED2C0A9DED87
:103B50001F1A01E0BE37863500EE810A85ED120A94
:103B600094ED260ADDED140A20EE200AD4ED2A0A8F
:103B70009DED181A00EE810AD4ED2B0A9DED1C1A5A
:103B800000EE810AD4ED2C0A9DED201A00EE810A88
:103B900085ED130A94ED2F0ADDED110A20EE200ABF
:103BA000D4ED330A9DED151A00EE810AD4ED340AE6
:103BB0009DED191A00EE810AD4ED350A9DED1D1A0E
:103BC00000EE810A85ED140A94ED2F0ADDED120A4C
:103BD00020EE200AD4ED330A9DED161A00EE810A7C
:103BE000D4ED340A9DED1A1A00EE810AD4ED350A9F
:103BF0009DED1E1A00EE810A85ED150A94ED2F0A3F
:103C0000DDED130A20EE200AD4ED330A9DED171ADC
:103C100000EE810AD4ED340A9DED1B1A00EE810AF4
:103C2000D4ED350A9DED1F1A00EE810A85ED160AC6
:103C300094ED2F0ADDED140A20EE200AD4ED330AAC
:103C40009DED181A00EE810AD4ED340A9DED1C1A80
:103C500000EE810AD4ED350A9DED201A00EE810AAE
:103C600085ED170A94ED380ADDED110A20EE200AE1
:103C7000D4ED3C0A9DED151A00EE810AD4ED3D0A03
:103C80009DED191A00EE810AD4ED3E0A9DED1D1A34
:103C900000EE810A85ED180A94ED380ADDED120A6E
:103CA00020EE200AD4ED3C0A9DED161A00EE810AA2
:103CB000D4ED3D0A9DED1A1A00EE810AD4ED3E0ABC
:103CC0009DED1E1A00EE810A85ED190A94ED380A61
:103CD000DDED130A20EE200AD4ED3C0A9DED171A03
:103CE00000EE810AD4ED3D0A9DED1B1A00EE810A1B
:103CF000D4ED3E0A9DED1F1A00EE810A85ED1A0AE9
:103D000094ED380ADDED140A20EE200AD4ED3C0AC9
:103D10009DED181A00EE810AD4ED3D0A9DED1C1AA6
:103D200000EE810AD4ED3E0A9DED201A00EE810AD4
:103D300085ED1B0A94ED410ADDED110A20EE200A03
:103D4000D4ED450A9DED151A00EE810AD4ED460A20
:103D50009DED191A00EE810AD4ED470A9DED1D1A5A
:103D600000EE810A85ED1C0A94ED410ADDED120A90
:103D700020EE200AD4ED450A9DED161A00EE810AC8
:103D8000D4ED460A9DED1A1A00EE810AD4ED470AD9
:103D90009DED1E1A00EE810A85ED1D0A94ED410A83
:103DA000DDED130A20EE200AD4ED450A9DED171A29
:103DB00000EE810AD4ED460A9DED1B1A00EE810A41
:103DC000D4ED470A9DED1F1A00EE810A85ED1E0A0B
:103DD00094ED410ADDED140A20EE200AD4ED450AE7
:103DE0009DED181A00EE810AD4ED460A9DED1C1ACD
:103DF00000EE810AD4ED470A9DED201A00EE810AFB
:103E000085ED1F0A94ED4A0ADDED110A20EE200A25
:103E1000D4ED4E0A9DED151A00EE810AD4ED4F0A3D
:103E20009DED191A00EE810AD4ED500A9DED1D1A80
:103E300000EE810A85ED200A94ED4A0ADDED120AB2
:103E400020EE200AD4ED4E0A9DED161A00EE810AEE
:103E5000D4ED4F0A9DED1A1A00EE810AD4ED500AF6
:103E60009DED1E1A00EE810A85ED210A94ED4A0AA5
:103E7000DDED130A20EE200AD4ED4E0A9DED171A4F
:103E800000EE810AD4ED4F0A9DED1B1A00EE810A67
:103E9000D4ED500A9DED1F1A00EE810A85ED220A2D
:103EA00094ED4A0ADDED140A20EE200AD4ED4E0A04
:103EB0009DED181A00EE810AD4ED4F0A9DED1C1AF3
:103EC00000EE810AD4ED500A9DED201A00EE810A21
:103ED00085ED230A21B030BD30B502460B460020E7
:103EE00046E0002141E003EB001494ED000A01F1EB
:103EF000120402EB8404D4ED000A20EE200A01240F
:103F000004EB800403EB8404D4ED000A01F13604D1
:103F100002EB840494ED001A00EE810A022404EB03
:103F2000800403EB8404D4ED000A01F13F0402EBAA
:103F3000840494ED001A00EE810A032404EB80044B
:103F400003EB8404D4ED000A01F1480402EB84047D
:103F500094ED001A00EE810A00EBC0040C44104DF1
:103F600005EB840484ED000A491C0929BBDB401CD5
:103F70000928B6DB00200FE002EB800191ED000A7A
:103F8000074901EB8001D1ED000A30EE600A02EB37
:103F9000800181ED000A401C5128EDDB30BD00009E
:103FA000B48E002010B502460023002003E032F852
:103FB00010402344401C8842F9DBB3FBF1F080B28F
:103FC00010BD02468A4201DC881A70474FF6FF7026
:103FD000801A401C0844F8E738B5044625460020FE
:103FE0000090686800788DF80000686840788DF867
:103FF0000100686840786968097800EB01200A4987
:10400000088002236A46AC210020F3F7A3FB0121BC
:104010000648F6F797FCF8F78FFA05490860054956
:104020000420F5F78FFA38BDA43F002045FC0200BC
:10403000A83F0020009F00FF70B505462C460020D9
:104040001C490870207A012829D16068007801286D
:1040500025D1194890F82800432801D1012000E01B
:10406000002015494979884219D0FCF759F9662092
:1040700011494871F4F770FA18B110A10820F3F74C
:104080007DFE0D4800791449C8750B484079887643
:10409000F4F73AFA18B111A10820F3F76FFE0648B9
:1040A000007928B1237AB02114486268F3F752FBF3
:1040B00070BD0000304000207453002070777220E3
:1040C0007361766520696E666F726D6174696F6E7B
:1040D000206661696C000000085400206170705F08
:1040E0006465746563745F4C522073617665206209
:1040F00061636B7570206661696C00000C40002084
:104100000121014A117070478C40002070B50446AF
:10411000254606F0B9FA2B7AA72100206A68F3F742
:1041200019FB70BD70B505462C4612480079002871
:1041300011DD6068007818B901200F49087070BD62
:1041400060680078012813D10123A621002062684D
:10415000F3F700FB0CE00123084AA6210848F3F717
:104160001DF901200749086001210748F6F7EAFB1D
:1041700000BFE4E774530020543F00207D3F00203F
:10418000583F0020503F0020110A030070B504463C
:104190002546686800781549C8700846C078B0B1EF
:1041A000002008711248FEF77FFD1048C0780128F2
:1041B00002D1F4F76DFE05E00C48C078022801D169
:1041C000F4F76CFE01210B48F6F7BCFB06E000217A
:1041D0000848F6F7B7FB0648FEF78EFD0123034AB1
:1041E000D21CA2210020F3F7B5FA70BD343F0020A5
:1041F000F0670400DD04030070B5044625466868D6
:1042000000780B49087008460078012806D1002084
:10421000084908800848FEF747FD02E00648FEF717
:104220006BFD0123024AA5210020F3F793FA70BD2C
:10423000283F0020263F0020D067040070B50546C7
:104240002C46606840786168097840EA0126154884
:104250000079D8B160688078012803D13046F5F73D
:1042600089FB1DE06068807848B93046F5F782FB2D
:10427000237AA42100206268F3F76CFA10E0237A15
:10428000A42100206268F3F765FA09E0606880788D
:10429000022802D06068807810B93046F5F76AFBD2
:1042A00070BD00007453002008B50446A146D9F83B
:1042B00004000078009001236A46AB210020F3F748
:1042C00049FA00201C494876F4F71EF918B11BA1E1
:1042D0000D20F3F753FD4FF4FA7505B90EE000BF5A
:1042E0004FF47A7606B905E0DFF87080B7013846FA
:1042F000C04700BF681E051EF2D100BF00BF00BF4F
:1043000000BF00BF00BFBFF34F8F00BF00BF00BFA3
:104310001348006800F4E06012490843001D10498A
:10432000086000BF00BF00BFBFF34F8F00BF00BFDA
:1043300000BF00BF00BFFDE708540020617070207F
:104340007265737461727420736176652062616353
:104350006B7570206661696C0000000001680400E4
:104360000CED00E00000FA0570B505462C466068CB
:10437000067836B1012E0ED0022E17D0032E26D18C
:104380001BE014480079012802D1FCF725FA01E06E
:10439000FBF754FB1CE00F480079012803D11420DF
:1043A000FCF700FA01E0FBF7EDF811E0FDF784F807
:1043B00010B92046FBF7D8F90AE0237AA1210020A2
:1043C0006268F2F7EBFF2046FBF774F900E000BFEC
:1043D00000BF70BD7453002010B504460E4800782D
:1043E00000B910BD0D4800880D490988884210DACF
:1043F0000A480088401C80B208490880084909889A
:10440000884202DB00200449087004480088FBF75A
:10441000EBF900BFE5E70000953E0020963E002046
:10442000983E002070B5044625462B7AA72100202F
:104430006A68F2F7B3FF70BD38B5044600200090FB
:10444000254668680078009001236A46A62100206E
:10445000F2F7A4FF38BD70B5044625462B7AAD218E
:1044600000206A68F2F79AFF70BD000070B505463B
:104470002C4660680078012818D10D480078012882
:1044800011D16068407800066168897840EA01408F
:104490006168C97840EA01206168097908430549E3
:1044A0000860FCF795FF03200349087070BD000009
:1044B000183F0020203F0020243F00202DE9F0413C
:1044C00006463248007908B9BDE8F0813446606894
:1044D000077817B1012F55D12AE0002007E000F13D
:1044E00041016268525C294933310A54401C062854
:1044F000F5DB47256068405D0106681C6268105C5A
:1045000041EA0041A81C105C41EA0020E91C515C12
:1045100008431E49C862681D6168095C281D6268FD
:10452000105C41EA002119480186FBF787FA2AE06E
:10453000606840781649087060688078154908708E
:104540006068C07900066168097A40EA01406168E4
:10455000497A40EA01216068807A01430B48816111
:10456000207A192808DB6068807D6168497D00EB4E
:10457000012000B208490880002008490870FBF7B4
:1045800001F800E000BF00BF00BF9DE774530020AA
:10459000C83E0020C93E0020CA3E0020F03E002058
:1045A00008B50446F3F7A1FDF3F7B5FDF3F787FD72
:1045B000A146D9F804000078009001236A46AE2194
:1045C0000020F3F7C7F84FF4FA7505B90EE000BF05
:1045D0004FF47A7606B905E0134F4FEA8618404645
:1045E000B84700BF681E051EF2D100BF00BF00BF64
:1045F00000BF00BF00BFBFF34F8F00BF00BF00BFB1
:104600000A48006800F4E06009490843001D0749B2
:10461000086000BF00BF00BFBFF34F8F00BF00BFE7
:1046200000BF00BF00BFFDE7616904000CED00E0C2
:104630000000FA0538B5044600200090FBF700FDA5
:1046400000900F48007988B19DF80000012806D13C
:1046500001236A46A3210020F3F77CF80EE0012332
:104660006A46A3210020F2F799FE07E0012000909E
:1046700001236A46A3210020F2F790FE38BD000016
:104680007453002010B5044600210348F6F75AF988
:1046900001200249087010BD110A0300563F002096
:1046A0002DE9FF4780464FF00009002400200090CC
:1046B0000190454605F070FE012801D1BDE8FF8755
:1046C000FAF7C6FE6868016800918088ADF80400BA
:1046D0006868807900066968C97940EA01406968BC
:1046E000097A40EA01206968497A40EA0106686867
:1046F000C07A6968897A40EA012701202249087056
:1047000022490720F4F71EFF00240AE02048005D3C
:104710001DF80410884202D04FF0010903E0601C2C
:10472000C4B2062CF2DB00BF19483338C06AB0426D
:1047300007D117483338008EB84202D1B9F1000FC3
:104740001FD013483338C662078602A8F4F792F8E0
:1047500000240AE01DF804100D48015502A8015D6F
:104760000B482D380155601CC4B2062CF2DB012029
:1047700008490870F6F730FF06F0B2F908B106F004
:1047800067F900BF9AE7000035400020AF0000FF46
:10479000A75300203440002038B504460120009083
:1047A00001236A46A3210020F2F7F8FD38BD00007E
:1047B0002DE9F0478CB08046454606F091F908B1E6
:1047C00006F046F96868007B10B90CB0BDE8F087C8
:1047D000F6F702FF01204449087044490720F4F726
:1047E000B1FE4FF00009002400200890099068688D
:1047F000016808918088ADF8240068688079000617
:104800006968C97940EA01406968097A40EA01208B
:104810006968497A40EA01066868C07A6968897AF5
:1048200040EA012700BF0AE03148005D08A9095DA0
:10483000884202D04FF0010903E0601CC4B2062C8C
:10484000F2DB00BF2A48801FC06AB04207D1284867
:10485000801F008EB84202D1B9F1000F42D0244827
:10486000801FC66207860AA8F4F704F800240AE04D
:104870000AA8015D1E482D30015508A8015D1C489D
:104880000155601CC4B2062CF2DBFCF74FFB002084
:1048900004900590069007901548801F90F83810F6
:1048A00090F8372090F83600114B9B1F1B7ACDE90A
:1048B0000030CDE902210E48801FC37982790DA115
:1048C00004A8F8F7D7F804A8F1F7EFFD824651469F
:1048D00004A811F06BF8FAF7D1FA11F021F8FAF701
:1048E000A9FA00BF00BF70E735400020AF0000FF0D
:1048F0007A5300202530325825303258253032582E
:10490000253032582530325825303258000000000A
:10491000704710B50446012110200AF022FFF6F777
:1049200097F910BD10B50446F6F772F910BD0000F6
:1049300010B50548007928B1F3EE0E0AB3EE0E0A61
:1049400011F04EF810BD00007453002010B504465D
:10495000F2F78BF90148F7F765FE10BD8585030076
:1049600010B50446F2F785F90748006807498861E1
:10497000002008610648F2F709FA0320034948615C
:104980000448F7F731FE10BD04B50040447900201B
:10499000ED8403008585030010B5F3F719F9254967
:1049A00008600846006890F82000032841D00320E2
:1049B000096881F820009FED200A1E48006880EDFC
:1049C000050A9FED1E0A1B48006880ED070A9FED4F
:1049D0001B0A1848006880ED060AB7EE000A154861
:1049E000006880ED030A9FED150A1248006880ED0B
:1049F000040A9FED120A0F48006880ED010A9FED3E
:104A00000F0A0C48006880ED000A00200949096877
:104A100081F821009FED090A0648006880ED020A2E
:104A200001200449096881F823000249096881F8D6
:104A3000220010BD904000200000C842000000008D
:104A4000024909680144014A11607047FC40002096
:104A500070B58AB004460D462E46202102A8F1F713
:104A600019FDF0B28DF80400300A8DF80500012020
:104A70008DF808000D4804900594A189ADF81A102E
:104A80000221ADF81E100021ADF81C1001A90891FB
:104A900001208DF8180001218DF81910228902A932
:104AA000A0690AF01BF80AB070BD0000CD9C03009D
:104AB00070B590B006460C461546A07818B901208E
:104AC0008DF80E0002E0A0788DF80E002088ADF879
:104AD0000C0000200290607C02A910F065FEA07C12
:104AE0000DF1090110F060FEE07B08B1012000E04B
:104AF00000209DF80A1060F3C3018DF80A10207C95
:104B000008B1012000E000209DF80A1060F30411B4
:104B10008DF80A10207B08B1012000E000209DF8EC
:104B20000A1060F300018DF80A10207D08B1022000
:104B300000E001209DF80A1060F342018DF80A1090
:104B40001C2109A8F1F7A6FC607BC0F3001018B97E
:104B5000607BC0F34010F8B100200090E07C0DF1C4
:104B6000010110F021FE00BF9DF8000020F00F00B1
:104B7000401C8DF800009DF8000020F0F00010307F
:104B80008DF8000000BF9DF8020020F00600801C98
:104B90008DF80200CDF838D0607B8DF82400A07B22
:104BA0008DF82500142104A8F1F774FC03A80490E3
:104BB00002A80590A088ADF81C00A06820B1E0888C
:104BC000ADF81800A0680890A069002849D000201E
:104BD0000190A0690088ADF82C00A0694088ADF86C
:104BE0002E00A06940680A9001A80D90A169087B79
:104BF00001A910F0D9FDA169487B0DF1050110F064
:104C0000D3FDA069807A08B1012000E000209DF862
:104C1000061060F3C3018DF80610A069C07A08B1D0
:104C2000012000E000209DF8061060F304118DF8CB
:104C30000610A069007A08B1012000E000209DF86C
:104C4000061060F300018DF80610A069807B08B1A2
:104C5000022000E001209DF8061060F342018DF86B
:104C60000610E06908B1E0690C902B4604AA09A976
:104C70003046AADF10B070BD70B58AB004460E464B
:104C8000202101A8F1F706FC0020099094F8C60243
:104C900000EB8001C1EB801004EB400594F8C502E5
:104CA000B8B194F8C522521ED1B294F8C62202EBD4
:104CB0008203C3EB821204EB420501EBC10305F151
:104CC0000A0202EB43000289521C92B2ADF8242082
:104CD00002E0E888ADF824002889ADF8260003201A
:104CE0008DF8040009980590049405480390324615
:104CF00001A90448006809F0F1FE0AB070BD000087
:104D000029600300904A002010B52DED048BB0EE11
:104D1000408A9FED270AB0EE409A9FED250AF0EEFB
:104D2000408A2448006890F8220060B1B2EE040A7C
:104D3000C8EE000A1F480068C0ED010A00201D49A6
:104D4000096881F82200B2EE040AC8EE000AF0EE0B
:104D5000609A18480068001DDFED170AB0EE690A76
:104D600003F0C2FAF0EE408A9FED140AF4EEC08A16
:104D7000F1EE10FA04D29FED0E0AB0EE409A11E067
:104D80009FED0F0AF4EEC08AF1EE10FA04DD9FEDFC
:104D90000D0AB0EE409A05E0B0EE680A06F0D8FCC5
:104DA000B0EE409AB0EE490ABDEC048B10BD000095
:104DB0000000000090400020CDCC4C3D0000AF43EF
:104DC0000080CF430000C84210B51C200AF033FC1D
:104DD00008B1012010BD0020FCE710B501460022FB
:104DE0000B46002004E00C1D245C1444E2B2401C7D
:104DF000DC788442F7DC9878904201D1012010BD24
:104E00000020FCE770B505460DB9094C01E0084CDF
:104E1000083409E0204607F0B1F9064606B904E077
:104E200028467168884700BFF4E700BF70BD0000E6
:104E30007093002010B504462CB901200649487033
:104E40000020FFF7DFFF012C04D101200249887008
:104E5000FFF7D8FF10BD0000689300202DE9F04750
:104E6000024613468C46D3E90245DCE90267B6EBFD
:104E7000040877EB050002D30120BDE8F08700208D
:104E8000FBE701468878012805D191F82000012828
:104E900001D100207047886A042802D0486A04289B
:104EA00001D10020F6E70120F4E72DE9FF4F03468A
:104EB0000C46002047E0225CFF2A3ED0C2F3C01916
:104EC00022F080014DF82010B9F1000F0DD05DF8EF
:104ED000201000BF4FF0A0452E46012707FA01F52C
:104EE000C6F8085500BF00BF0DE05DF8201000BFF8
:104EF0004FF0A0452E46012707FA01F5C6F80C55DC
:104F000000BF00BF00BF5DF8201001252E4600271E
:104F1000BC46B84600BF4FF0A04BDA4645EA460B08
:104F20004BEA870B4BEA0C2B4BEA084E0AF5E06B79
:104F30004BF821E000BF00BF03E04FF0FF314DF818
:104F40002010411CC8B20428B5DB6D461A68002148
:104F500007E055F8217002F5AC6646F821704E1C4A
:104F6000F1B20429F5DB00BFBDE8FF8F0246002047
:104F700007E0536833F810308B4200D17047431C70
:104F800098B213888342F4DC00BFF7E733B58BB0E7
:104F90000546002000900C9878B100240BE02146D3
:104FA0000CA809F036FC28B1009A501C009001A80A
:104FB00020F81240641C142CF1D32C226946284698
:104FC000F1F74FFA0DB030BD10B502460B46002187
:104FD0000DE0506830F811004FF6FF74A04204D184
:104FE000506820F81130002010BD481C81B2108894
:104FF0008842EEDC0420F7E701460888062808DB33
:105000000888B0F5486F06DD08884FF6FF729042B9
:1050100001D0072070474888062808DB4888B0F58B
:10502000486F06DD48884FF6FF72904201D0072096
:10503000F0E708884FF6FF72904208D04888904207
:1050400005D008884A88904201DD0720E2E7002069
:10505000E0E72DE9F04107460D46144698462088C2
:10506000801D404502D90C20BDE8F0813846FFF78D
:10507000C3FF064600BF304600B1F5E700BF05207C
:10508000218868542088401C208012202188685480
:105090002088401C208022885119388811F08DF911
:1050A00021880844208022885119788811F085F9D8
:1050B0002188084420800020D6E7000010B504466F
:1050C00000BF03A292212046F1F7A4F800BF10BD53
:1050D0002E2E5C2E2E5C2E2E5C626C655F636667E6
:1050E0005C736C6176652E630000000030B587B09C
:1050F0001C216846F1F7CEF9002000904FF4804063
:1051000001904FF4A030029001208DF80C004FF672
:10511000FF70ADF80E0001208DF810000020059002
:10512000094806906846FCF7BDFE044600BF2546C8
:1051300035B100BF05A2A5212846F1F76BF800BFE5
:1051400000BF07B030BD0000BD5003002E2E5C2E06
:105150002E5C2E2E5C626C655F6366675C736C61AF
:1051600076652E6300000000F8B505460C46607AAF
:1051700088B9207A10B91048476801E00E4887685E
:105180002A4639466068FCF7F7F9064616B13046FC
:1051900010F0D2F80EE0002020720748406948B1B4
:1051A00001208DF80000ADF80250034841696846BF
:1051B000884700BFF8BD00004C9300200246002045
:1051C00003E0064B1B5C1354401C054B1B789842B4
:1051D000F7DB03480078087070470000D082002099
:1051E0004E4800200246002003E0064B1B5C13548F
:1051F000401C054B1B789842F7DB03480078087089
:1052000070470000948200204D480020F0B504460D
:105210000D460020002108E014F801C00646471C96
:10522000F8B20B4F07F806C0491CA942F4DB002175
:1052300008E012F801C00646471CF8B2044F07F810
:1052400006C0491C9942F4DB02490870F0BD000019
:10525000948200204D4800202DE9F0410646DDE90A
:10526000064500200F88C7F307280746401CDFF8D3
:105270003CC10CF8078091F800800746401C0CF8F0
:1052800007804F88C7F307280746401C0CF80780A3
:1052900091F802800746401C0CF807808F88C7F3FE
:1052A00007280746401C0CF8078091F80480074641
:1052B000401C0CF807801788C7F307280746401CD6
:1052C0000CF8078092F800800746401C0CF8078015
:1052D0005788C7F307280746401C0CF8078092F848
:1052E00002800746401C0CF807809788C7F3072800
:1052F0000746401C0CF8078092F804800746401CC3
:105300000CF807801F88C7F307280746401C0CF8D5
:10531000078093F800800746401C0CF807805F88E0
:10532000C7F307280746401C0CF8078093F8028053
:105330000746401C0CF807809F88C7F307280746DC
:10534000401C0CF8078093F804800746401C0CF8BA
:1053500007802788C7F307280746401C0CF80780FA
:1053600094F800800746401C0CF807806788C7F354
:1053700007280746401C0CF8078094F8028007466F
:10538000401C0CF80780A788C7F307280746401C75
:105390000CF8078094F804800746401C0CF807803E
:1053A000DFF80CC08CF80000BDE8F081D08200204E
:1053B0004E4800207FB506460C4600200290039020
:1053C000ADF80840ADF80A40009001906A4602A985
:1053D000304690DF054605B100BF284604B070BDD9
:1053E00010B5044621460248FDF74DFA10BD0000F5
:1053F000308000207CB5002000900190094800908A
:10540000094801906846FCF7E3FD044600BF2546C5
:1054100035B100BF05A22D212846F0F7FBFE00BFE5
:1054200000BF7CBDE15303001C4800202E2E5C2EE3
:105430002E5C2E2E5C626C655F6366675C686F73C2
:10544000742E630070B52DED0A8B04460D4694ED65
:10545000060AB1EE400A10EE101A0846F1F725FAD6
:1054600041EC1B0BB0EE4B0AF0EE6B0AF7F7A4FB16
:10547000B0EE40AAF0EE60AA51EC1A0BF1F758FA20
:1054800008EE900A94ED000A10EE101A0846F1F7A3
:105490000CFA41EC1B0B94ED030A10EE101A0846AF
:1054A000F1F703FA41EC1C0BB0EE4B1AF0EE6B1A5D
:1054B000B0EE4C0AF0EE6C0AF7F732FFB0EE40AAFD
:1054C000F0EE60AA51EC1A0BF1F732FA08EE100A6E
:1054D00094ED080A10EE101A0846F1F7E6F941ECCF
:1054E0001B0B94ED070A10EE101A0846F1F7DDF9D0
:1054F00041EC1C0BB0EE4B1AF0EE6B1AB0EE4C0AFE
:10550000F0EE6C0AF7F70CFFB0EE40AAF0EE60AADE
:1055100051EC1A0BF1F70CFA09EE100A9FED100A84
:1055200028EE000ABDEEC00A10EE100A00B2288074
:105530009FED0B0A28EE800ABDEEC00A10EE100A9D
:1055400000B268809FED060A29EE000ABDEEC00A8F
:1055500010EE100A00B2A880BDEC0A8B70BD0000EE
:1055600000401C4602781206437842EA03428378E0
:1055700042EA0322C3781A433C4B1A6002791206AE
:10558000437942EA0342837942EA0322C3791A4308
:10559000364B5A60027A1206437A42EA0342837A11
:1055A00042EA0322C37A1A43304B9A60427B037B60
:1055B00042EA032212B22E4B1A80C27B837B42EA5C
:1055C000032212B22A4B5A80427C037C42EA032215
:1055D00012B2274B9A80C27C837C42EA0322254B7D
:1055E0001A80427D037D42EA0322234B1A80827D8A
:1055F000224B1A80C27D224B1A70427E037E42EA01
:10560000032212B21F4B1A80C27E837E42EA03221B
:1056100012B21D4B1A80427F037F42EA032212B26C
:10562000194B5A80C27F837F42EA032212B2164B83
:105630009A8090F8212090F8203042EA032212B29A
:10564000124B1A8090F8232090F8223042EA03226D
:1056500012B20E4B5A8090F8252090F8243042EA7E
:10566000032212B2094B9A8070470000748900200F
:1056700078490020AA490020AE4900208A4900202C
:10568000A6490020744900207E490020844900205A
:1056900002781206437842EA0342837842EA032200
:1056A000C3781A433C4B1A6002791206437942EAE6
:1056B0000342837942EA0322C3791A43364B5A6084
:1056C000027A1206437A42EA0342837A42EA0322CA
:1056D000C37A1A43304B9A60427B037B42EA03222F
:1056E00012B22E4B1A80C27B837B42EA032212B293
:1056F0002A4B5A80427C037C42EA032212B2274B97
:105700009A80C27C837C42EA0322254B1A80427D28
:10571000037D42EA0322234B1A80827D224B1A80AA
:10572000C27D224B1A70427E037E42EA032212B2ED
:105730001F4B1A80C27E837E42EA032212B21D4BA7
:105740001A80427F037F42EA032212B2194B5A8029
:10575000C27F837F42EA032212B2164B9A8090F8EE
:10576000212090F8203042EA032212B2124B1A8014
:1057700090F8232090F8223042EA032212B20E4B16
:105780005A8090F8252090F8243042EA032212B281
:10579000094B9A80704700008089002090490020C2
:1057A000A8490020AC490020A2490020A5490020BA
:1057B0008C490020964900209C4900202DE9F04F9B
:1057C00089B004460F4691464FF0000B20216846F1
:1057D000F0F760FE94F8C60200EB8001C1EB801088
:1057E00004EB400594F8C50200EBC00105F10A0086
:1057F00000EB410A94F8C502401C2979884207D180
:1058000008AB00225146204606F078FC834627E08C
:1058100094F8C5621FE02879401EB04202D14FF0D3
:10582000000806E0701C00EBC00105F10A0000EB67
:10583000410808AB42465146204606F05FFC10B1D5
:105840004FF0010B0AE0C24694F8C502401C84F8F0
:10585000C502701CC6B22879B042DCDC00BF00BFB4
:10586000BBF1000F05D101203870002009B0BDE860
:10587000F08F0020387004208DF800000898049004
:105880000394044802904A4669460348006809F0B8
:1058900025F9EBE729600300904A0020F0B50346A4
:1058A000002249488446DCE90267DCF80450DCF851
:1058B00010C0A0E8E0104548851C2E6806606D68A1
:1058C0004560B3F90400002801DB054600E04542CD
:1058D0003D4E35613D4801813D480068042841DD69
:1058E000304600693546ED68A8420DDB3046C06899
:1058F000384D2D68A84202DA3046C06801E03548CC
:105900000068344D286003E049F64040314D28607E
:105910002D4805692F48006800F5FA70854205DDBD
:105920002D480068401C2C4D286002E000202A4DC4
:10593000286029480068002800DD0122274D2D68D5
:10594000012D14D1214DB5F90850204EB6F906604D
:10595000A81B002801DB054600E04542CB2D06DAF6
:10596000012204E01A480068401C194D28600024F8
:105970001A48006850B9012A08D119480068194D21
:105980002D68401BB0F5007F00DD0124A2B914484A
:105990000068884202DD1248006800E00846104DA9
:1059A000286010480068884202DA0E48006800E06B
:1059B00008460C4D286003E0094801600948016071
:1059C000064802602046F0BD604A00207492002024
:1059D000784A0020744A0020804A00207C4A002037
:1059E000844A0020884A00202DE9FF4F8BB0824670
:1059F00014461D46BAF90400002801DB014600E008
:105A0000414209B20A910C99B1F90400002801DB66
:105A1000014600E041420FFA81FB7622FE49881ED2
:105A2000F0F71FFD7622FD49881EF0F71AFD762259
:105A3000FB49881EF0F715FD7622FA49881EF0F71B
:105A400010FD7622F849881EF0F70BFDF249891EF9
:105A50000A98A1F87600F148801EA0F876B0208858
:105A6000EF49891EA1F876006088EE49891EA1F8E9
:105A70007600A088EC49891EA1F8760008A809A93B
:105A800004233C22CDE900101421E548801E02F0D9
:105A90003EFC06A807A904233C22CDE900101421EE
:105AA000E048801E02F033FC04A805A904233C2230
:105AB000CDE900101421DC48801E02F028FCDB4BED
:105AC0004FF4FA723C21D548801E06F04EFA81460A
:105AD000B9F1010F02D15020D5490880D54B4FF4C0
:105AE000FA723C21CD48801E06F0FAF90390D048A6
:105AF000B0F90000002809DDCF4B4FF47A723C2149
:105B0000C548801E06F031FA064608E0CA4B4FF43D
:105B1000FA623C21C048801E06F027FA0646BE48BD
:105B2000801EB0F97600BC49891EB1F96E10401A8A
:105B300010F1320F0FDDB848801EB0F97600BF4972
:105B4000B1F9001088420CDAB348801EB0F8760034
:105B5000BA49088005E0B048801EB0F87600B74921
:105B60000880AD48801EB0F97600B449B1F9001044
:105B7000401AB0F57A7F00DD0126A848801EB0F9F2
:105B80007600AA49B1F90010401AB0F5FA6F00DDAD
:105B90000126AB4B4FF4FA723C219F48801E06F061
:105BA0009FF907469D48801EB0F976009F49B1F9DC
:105BB0000010401AB0F5FA7F09DD9848801EB0F950
:105BC00076009C49B1F90010081AC8281FDB9248DA
:105BD000801EB0F976009849B1F90010401AB0F56E
:105BE000FA7F09DD8C48801EB0F976009449B1F93E
:105BF0000010081AC8280ADB8748801EB0F9760012
:105C00008E49B1F90010401AB0F5FA7F04DD50203A
:105C10008C4908808C490880012F02D100208A49D4
:105C200008807E48801EB0F976008049B1F90010E6
:105C3000401AB0F57A7F0BDD7748801EB0F9760008
:105C40007D49B1F90010401AB0F57A7F00DD0126D8
:105C50007E4A39B230B20FF073FC7C48B0F90000D4
:105C6000002802DD50207A4908806F48801E6D4B65
:105C70009B1E6B4A921E2946009074480FF01EFC32
:105C80007348B0F90000002804DC6E48B0F9000049
:105C900000281CDDBDF92400BDF92010401A82281F
:105CA00015DABDF91C00BDF91810401A82280EDA69
:105CB000BDF91400BDF91010401A822807DA01203E
:105CC00028806248008810B9022060490880208836
:105CD00010FB00F0618811FB0100A18811FB01009D
:105CE00002905949B1F90010002910DD0299A1F57F
:105CF0008000002801DB014600E04142554A914204
:105D000005DA5248008810B9022050490880BDF9D0
:105D10002400BDF92010401A672816DABDF91C00CE
:105D2000BDF91810401A67280FDABDF91400BDF943
:105D30001010401A672808DA012119980180464896
:105D40000068401C4449086005E000211998018062
:105D500000204149086040480068B0F5C87F03DD75
:105D600001202880394908804FF067083648B0F98B
:105D70000000002801DD40F20648384B1B88012B4B
:105D800040D1274B9B1EB3F96E30DFF894C0ACF1C5
:105D9000020CBCF976C0A3EB0C02002A01DB13460F
:105DA00000E0534243452DDA1E4B9B1EB3F96E3083
:105DB000DFF870C0ACF1020CBCF976C0A3EB0C01AB
:105DC000002901DB0B4600E04B4243451ADA164B33
:105DD0009B1EB3F96E30DFF850C0ACF1020CBCF979
:105DE00076C0A3EB0C00002801DB034600E0434231
:105DF000434507DA012028801448008810B90220A2
:105E0000124908801248B0F9000000282ADD104825
:105E10000088401E00B223E0069000207E90002003
:105E2000F69000206E910020E6910020204A00208C
:105E3000184A0020244A00201E4A0020104A002050
:105E4000224A00201A4A00201C4A0020004A002052
:105E50000A4A0020E0930400144A0020084A002067
:105E6000214908802148B0F90000002805DD1F48BD
:105E70000088401E00B21D4908801D48B0F900008E
:105E8000002805DD1A480088401E00B21849088025
:105E90001848B0F90000002805DD16480088401EAB
:105EA00000B2144908801448B0F90000002805DD4C
:105EB00011480088401E00B20F490880288810B1A0
:105EC0005020094908800D48B0F90000002805DD80
:105ED0000A480088401E00B20849088028880849FE
:105EE00008800FB0BDE8F08F0A4A00200C4A00205D
:105EF0000E4A0020184A00201A4A00201C4A00209E
:105F0000084A002030B59FB004460D467C21684603
:105F1000F0F7C0FAADF8025003208DF800000194AC
:105F20000448006818B168460249096888471FB0EC
:105F300030BD00008C4A00202DE9F04104460D469A
:105F4000164694F8C60200EB8001C1EB801004EB0A
:105F5000400840460DF07CFC0746E7B3D4F8CC027D
:105F6000062838D204F53470D4F8CC1200EBC110F6
:105F7000468004F53471D4F8CC2201EBC211081D1F
:105F800076224146F0F76DFA45B1002104F53470F0
:105F9000D4F8CC2200EBC210017007E0022104F516
:105FA0003470D4F8CC2200EBC210017004F53470C8
:105FB000D4F8CC1200EBC110C767D4F8CC02401C57
:105FC000C4F8CC020549D4F8CC020968884202D151
:105FD00020460CF00DFBBDE8F0810000944A002043
:105FE0002DE9F041A0B004460D46164694F8C602CD
:105FF00000EB8001C1EB801004EB400840460DF03F
:1060000027FC074657B17C22064901A8F0F729FA78
:10601000ADF80660029501A8B84700BF20B0BDE802
:10602000F0810000DC6A04002DE9F04105460C46D1
:1060300016462746002087F8C802324629463846C9
:10604000FFF7CEFF31463846FFF75CFFBDE8F08131
:10605000F0B589B004460E464FF4BA612046F0F719
:1060600019FA202101A8F0F715FA31461E480068F8
:1060700008F00AFD054600BF284608B109B0F0BD8A
:1060800000BFA4F8CA620020C4F8CC0284F8C7029A
:1060900084F8C60284F8C50294F8C60200EB8001B9
:1060A000C1EB801004EB400794F8C6020F4901EBE6
:1060B00080000068386002208DF804000120ADF8EF
:1060C00014003968CDF8161004940948039032463C
:1060D00001A90548006808F001FD054615B9012031
:1060E00084F8C8022846C9E7904A00207E92002022
:1060F000296003001CB518213348F0F7CBF90021C3
:1061000031482C3880F84C1080F8491080F84D1038
:1061100080F84A1080F84E1080F84B1080F8461036
:1061200080F8481080F84710002027492C3981F862
:106130004400002124482C3880F845102348224987
:106140002C394860224808600020886203210346F9
:106150000122CDE900101146072009F056F903206D
:1061600009F0DBF9042009F0D8F9052009F0D5F988
:10617000062009F0D2F90021032009F041FB00219B
:10618000042009F03DFB0021052009F039FB002126
:10619000062009F035FB0021072009F031FB032020
:1061A0000CF049FA0121072009F02AFB03200CF02A
:1061B00042FAF5F7EDF8074A07A14FF47A70F4F7C1
:1061C000E7FB0EF027F81CBDC47A002095260400DA
:1061D000FD260400F17303006472765F6C736D5FDB
:1061E0007370695F6572726F725F7265706F7274DF
:1061F0000000000038B50446134890F84900E8B1A3
:106200006946114806F031FD9DF8000000F00100DC
:1062100088B10E4800210160818001460A4805F0DE
:10622000DDFF0A48008820800848408860800748D1
:106230008088A08005E04FF0FF3038BD4FF0FF3080
:10624000FBE70020F9E70000987A0020E87A0020B8
:106250000146054802680A6042684A6002890A816C
:10626000807A887200207047DC7A00202DE9F041A6
:10627000054600260024474890F84A0000B1B61DA4
:10628000444890F8490000B1B61D424890F84B00D0
:1062900000B1B61D3F4890F84800012800D1B61D56
:1062A00018213D48F0F7F6F8F2B23B49394806F0BC
:1062B000BEF90746781C18B94FF0FF30BDE8F081F1
:1062C000002D64D0334890F84A0098B104EB4400A4
:1062D000314931F81000E88004EB440001EB400044
:1062E0004188298104EB44002B4901EB400081885F
:1062F0006981641C274890F8490090B104EB440080
:10630000254931F81000288004EB440001EB4000DF
:106310004088688004EB440001EB40008088A8803E
:10632000641C1C4890F84B0098B104EB44001A49D7
:1063300031F81000A88104EB440001EB40004188D3
:10634000E98104EB4400144901EB40008188298273
:10635000641C104890F84800012818D104EB440050
:106360000D4901EB40004078000404EB44010A4A67
:1063700012F8111040EA012004EB440102EB410144
:10638000C978084300EBC00101EB001068610020F0
:1063900094E70000987A0020E87A00203EB50020BB
:1063A00001900025002402A9214806F090F901235C
:1063B0006A463B211E4806F02CFB9DF8000000F0C9
:1063C000E000E0280CD10021194806F0EEF81E206C
:1063D0000CF05AF90621164806F0E7F8601E3EBD9B
:1063E0009DF8080008B301A9114805F057FF1048AF
:1063F00090F8490008B1E01C84B20D4890F84A00BA
:1064000008B1E01C84B20A4890F84B0008B1E01CC7
:1064100084B2074890F84800012801D1E01C84B2FA
:10642000BDF8040090FBF4F085B22846D7E70000E1
:10643000987A002010B50649064805F023FF044865
:1064400000786A2802D04FF0FF3010BD0020FCE732
:1064500084410020987A002038B50024FF20009065
:1064600001236A46002138200DF008F90446601C1B
:1064700018B19DF80000802802D04FF0FF3400E0F2
:106480000024204638BD0520704700001CB5F4F7F5
:106490005DFF0020032103460122CDE900101146D3
:1064A000072008F0B2FF032009F037F8002103208D
:1064B00009F0A6F90021042009F0A2F90021052025
:1064C00009F09EF90021062009F09AF90021072021
:1064D00009F096F918211348EFF7DCFF0021114865
:1064E0002C3880F84C1080F8491080F84D1080F856
:1064F0004A1080F84E1080F84B1080F8461080F853
:10650000481080F84710002006492C3981F84400D3
:10651000002104482C3880F84510002001492C390E
:1065200088621CBDC47A00207CB50121072009F0D7
:1065300067F9032501240020009023460246014606
:106540000190284608F061FF00BF18211548EFF7B9
:10655000A1FF002113482C3880F84C1080F8491016
:1065600080F84D1080F84A1080F84E1080F84B10DB
:1065700080F8461080F8481080F84710002009493C
:106580002C3981F84400002106482C3880F8451049
:10659000002004492C398862F4F7D8FEF4F7F8FE9D
:1065A00000207CBDC47A002010B51A491A4805F0B5
:1065B00069FE184800786A2802D04FF0FF3010BDFD
:1065C0000121154806F046FA4FF4FA601249886234
:1065D00000BF1249104806F02CFA0F48806A401E8E
:1065E0000D4988620D48007818B10846806A002875
:1065F000EFD10948806A10B94FF0FF30DFE707217B
:10660000054806F0F7FB0221034806F045FC002090
:10661000D5E7000084410020987A002085410020C1
:1066200010B54FF4FA604B49886200BF4A494948A7
:1066300006F0F9FB4748806A401E46498862464892
:10664000007818B90846806A0028EFD14148806A6E
:1066500010B94FF0FF3010BD40493E4805F0BEFD77
:106660003F48002101604160816000203D49087081
:1066700047E04FF4FA603749886200BF3649354831
:1066800006F0D1FB3348806A401E324988623248A6
:10669000007818B90846806A0028EFD12D48806A32
:1066A00010B94FF0FF30D6E72C492A4805F096FD87
:1066B00000202D4908701BE028492B4A127831F937
:1066C000120006F06DF826482749097800EB810092
:1066D000D0ED000A30EE200A21482349097800EB6A
:1066E000810080ED000A20480078401C1E49087097
:1066F0001D4800780328DFDB1A480078401C194940
:106700000870184800780528B3DB00201549087088
:1067100016E013481349097800EB810090ED000A58
:10672000F1EE040A80EE201A0D480E49097800EBBC
:10673000810080ED001A0B480078401C0949087060
:10674000084800780328E4DB0221024806F0F4FB45
:10675000002080E7987A00208D41002086410020AB
:10676000007B00208E4100208F41002010B52DEDD0
:10677000048B4FF4FA608549886200BF84498348DE
:1067800006F051FB8148806A401E8049886280483B
:10679000007818B90846806A0028EFD17B48806AE3
:1067A00020B94FF0FF30BDEC048B10BD794977481C
:1067B00005F014FD784800210160416081600020EF
:1067C0007649087047E04FF4FA607049886200BF6C
:1067D0006F496E4806F027FB6C48806A401E6B4983
:1067E00088626B48007818B90846806A0028EFD1A3
:1067F0006648806A10B94FF0FF30D4E765496348B6
:1068000005F0ECFC0020664908701BE06149644A11
:10681000127831F9120005F0C3FF5F48604909782A
:1068200000EB8100D0ED000A30EE200A5A485C49A6
:10683000097800EB810080ED000A59480078401C7F
:1068400057490870564800780328DFDB5348007822
:10685000401C52490870514800780528B3DB0020DD
:106860004E49087016E04C484C49097800EB81000D
:1068700090ED000AF1EE040A80EE201A46484749DE
:10688000097800EB810080ED001A44480078401C34
:1068900042490870414800780328E4DB00203F4962
:1068A00008702EE03C483D4A127800EB820090EDE3
:1068B000000A3C48394A127800EB8200D0ED000A09
:1068C00030EE600A10EE101A0846EFF7EEFF41ECCA
:1068D000190BB0EE490AF0EE690AF6F7A5FFB0EE23
:1068E000408AF0EE608A51EC180BF0F721F82E493F
:1068F0002A4A127841F8220028480078401C27498B
:106900000870264800780328CCDB0120274908704E
:1069100000202249087023E023482049097800EB31
:10692000810090ED000ADFED220AB4EEE00AF1EEFC
:1069300010FA0DD31C481949097800EB810090ED3D
:10694000000ADFED1C0AB4EEE00AF1EE10FA02DDF7
:1069500000201649087011480078401C0F49087043
:106960000E4800780328D7DB0021084806F0E4FA37
:106970000021064806F03EFA0721044805F073FF9F
:106980000621024805F0C4FF00200CE7987A002099
:106990008D410020864100200C7B00208E4100208C
:1069A0008F410020007B0020187B00208C410020BC
:1069B0000000B4420080D44410B54FF4FA604B4953
:1069C000886200BF4A49494805F066FF4748806A27
:1069D000401E464988624648007818B90846806AD1
:1069E0000028EFD14148806A10B94FF0FF3010BD48
:1069F00040493E4805F01CFC3F48002101604160D1
:106A0000816000203D49087047E04FF4FA60374943
:106A1000886200BF3649354805F03EFF3348806A3A
:106A2000401E324988623248007818B90846806AA8
:106A30000028EFD12D48806A10B94FF0FF30D6E71B
:106A40002C492A4805F0F4FB00202D4908701BE072
:106A500028492B4A127831F9120005F095FE264894
:106A60002749097800EB8100D0ED000A30EE200ABA
:106A700021482349097800EB810080ED000A204875
:106A80000078401C1E4908701D4800780328DFDB91
:106A90001A480078401C19490870184800780528E1
:106AA000B3DB00201549087016E013481349097834
:106AB00000EB810090ED000AF1EE040A80EE201A4E
:106AC0000D480E49097800EB810080ED001A0B4853
:106AD0000078401C09490870084800780328E4DB66
:106AE0000121024805F063FF002080E7987A00202A
:106AF0008D41002086410020007B00208E41002037
:106B00008F41002010B52DED048B864800210160D7
:106B10004160816000208449087049E04FF4FA60C8
:106B20008249886200BF8249804805F0B5FE7F48EF
:106B3000806A401E7D4988627D48007818B9084601
:106B4000806A0028EFD17948806A20B94FF0FF3081
:106B5000BDEC048B10BD7749744805F069FB00203B
:106B6000754908701BE07349734A127831F91200B5
:106B700005F00AFE6B487049097800EB8100D0ED02
:106B8000000A30EE200A67486B49097800EB810063
:106B900080ED000A68480078401C67490870664824
:106BA00000780328DFDB60480078401C5E490870ED
:106BB0005D4800780528B1DB00205B49087016E0CD
:106BC00058485949097800EB810090ED000AF1EE30
:106BD000040A80EE201A53485349097800EB8100DB
:106BE00080ED001A50480078401C4F4908704E480C
:106BF00000780328E4DB00204B4908702EE0494868
:106C0000494A127800EB820090ED000A4B48464A50
:106C1000127800EB8200D0ED000A30EE600A10EE30
:106C2000101A0846EFF741FE41EC190BB0EE490A85
:106C3000F0EE690AF6F7F8FDB0EE408AF0EE608AF1
:106C400051EC180BEFF774FE3D49374A127841F8C2
:106C5000220035480078401C3349087032480078DB
:106C60000328CCDB00203049087023E034482E494B
:106C7000097800EB810090ED000ADFED320AB4EEF6
:106C8000E00AF1EE10FA0DD32D482749097800EB00
:106C9000810090ED000ADFED2C0AB4EEE00AF1EE7F
:106CA00010FA02DD0020294908701F480078401CB6
:106CB0001D4908701C4800780328D7DB00211B48B9
:106CC00005F075FE0021194805F0CDFD1F4800783C
:106CD000012810D10121154805F035FFFF201C497E
:106CE0000870124805F01EFF19480078012816D0D8
:106CF0004FF0FF302CE701210C4805F024FFFF2066
:106D000013490870094805F00DFF11480078012863
:106D100002D04FF0FF301BE74FF0FF3018E70020A4
:106D200016E700000C7B00208E410020987A00209E
:106D30008D410020864100208F410020007B0020F3
:106D4000187B0020007C124800E62A498C41002074
:106D500085410020F8B504460026144890F84C0000
:106D6000A04221D014B1012C04D101E0002504E09F
:106D7000012502E04FF0FF3600BF00BF16B14FF013
:106D8000FF30F8BD2946094806F086F869460748ED
:106D900006F05AF89DF80000A84202D04FF0FF30EC
:106DA000EFE7024880F84C403046EAE7987A002046
:106DB000F8B5054600261A4890F84900A8422DD09B
:106DC000082D11D2DFE805F004061010080A0C0E99
:106DD00000240CE001240AE0042408E0052406E075
:106DE000062404E0072402E04FF0FF3600BF00BF96
:106DF00016B14FF0FF30F8BD2146094805F0FAFF03
:106E00006946074805F0B5FF9DF80000A04202D092
:106E10004FF0FF30EFE7024880F849503046EAE78C
:106E2000987A0020F8B504460026144890F84400EB
:106E3000A04221D014B1012C04D101E0002504E0CE
:106E4000012502E04FF0FF3600BF00BF16B14FF042
:106E5000FF30F8BD2946094806F055F8694607484D
:106E600006F033F89DF80000A84202D04FF0FF3042
:106E7000EFE7024880F844403046EAE7987A00207D
:106E80002DE9FF4F8BB08B4600200A90019091486E
:106E900090F846100B98814274D00B98082873D252
:106EA000DFE800F0040772721C31465B0024002505
:106EB0006EE0012401254FF0060ABBF1010F00D15D
:106EC00001260D98012800D101270E9808B14FF036
:106ED00001081898012800D1814659E001240425B1
:106EE0004FF0060ABBF1040F00D101260D980428CB
:106EF00000D101270E9808B14FF001081898012819
:106F000000D1814644E0012405254FF0060ABBF17B
:106F1000050F00D101260D98052800D101270E98F4
:106F200008B14FF001081898012800D181462FE0E0
:106F3000012406254FF0060ABBF1060F00D10126F9
:106F40000D98062800D101270E9808B14FF00108CE
:106F50001898012800D181461AE0012407254FF036
:106F6000060ABBF1070F00D101260D98072800D1B2
:106F700001270E9808B14FF001081898012800D198
:106F8000814605E0A4E0FFE74FF0FF300A9000BF24
:106F900000BF0A9820B14FF0FF300FB0BDE8F08F6E
:106FA00021464C4805F02AFB09A94A4805F016FB82
:106FB0009DF82400A04202D04FF0FF30EDE7002CF6
:106FC00073D05146434805F0F0FA07A9414805F04F
:106FD000C1FA9DF81C00504502D04FF0FF30DCE7AD
:106FE000012E11D131463B4805F0B5FB06A93948C1
:106FF00005F07DFB9DF81800B04201D0B01ECCE733
:107000000198C01C80B20190012F11D1394631483E
:1070100005F087FA05A92F4805F04FFA9DF81400EE
:10702000B84201D0B81EB8E70198C01C80B20190E8
:10703000B8F1010F12D14146264805F0D8F904A94C
:10704000244805F0A0F99DF81000404502D04FF00B
:10705000FF30A2E70198C01C80B20190B9F1010F86
:1070600012D149461B4805F00FFA03A9194805F04B
:10707000D7F99DF80C00484502D04FF0FF308CE75F
:107080000198C01C80B201901248019905F0FBFAEA
:1070900002A9104805F0DAFABDF8081001988142FB
:1070A00003D04FF0FF3078E7FFE72946094805F0A5
:1070B00051F908A9074805F00EF99DF82000A842EB
:1070C00002D04FF0FF3068E702490B9881F8460084
:1070D0000A9862E7987A0020F8B50446002614481A
:1070E00090F84D00A04221D014B1062C04D101E04B
:1070F000002504E0062502E04FF0FF3600BF00BF88
:1071000016B14FF0FF30F8BD2946094805F000FCE4
:107110006946074805F0D1FB9DF80000A84202D05F
:107120004FF0FF30EFE7024880F84D403046EAE785
:10713000987A0020F8B5054600261A4890F84A00CB
:10714000A8422DD0082D11D2DFE805F0040610105A
:10715000080A0C0E00240CE001240AE0042408E0D4
:10716000052406E0062404E0072402E04FF0FF3681
:1071700000BF00BF16B14FF0FF30F8BD21460948EF
:1071800005F071FB6946074805F02FFB9DF80000EC
:10719000A04202D04FF0FF30EFE7024880F84A509B
:1071A0003046EAE7987A0020F8B5044600261448ED
:1071B00090F84500A04221D014B1012C04D101E087
:1071C000002504E0012502E04FF0FF3600BF00BFBC
:1071D00016B14FF0FF30F8BD2946094805F0CEFB47
:1071E0006946074805F0ADFB9DF80000A84202D0B3
:1071F0004FF0FF30EFE7024880F845403046EAE7BD
:10720000987A0020F8B505460F461646002E01DD97
:10721000062E02DB4FF0FF30F8BD454890F84B00DA
:10722000A84278D0062E7DD2DFE806F07C03102736
:1072300030444DB10620009001236A4629213820B0
:107240000FF078FA044600E000246BE09DB1FF20C7
:10725000009001236A46292138200CF00FFA0446D9
:10726000601C18B19DF80000062802D04FF0FF34D2
:1072700002E0002400E0002454E0009501236A4667
:107280000A2138200FF056FA04464BE0FF20009008
:1072900001236A460A2138200CF0F0F90446601CEC
:1072A00018B19DF80000A84202D04FF0FF3400E072
:1072B000002437E087B301211D4805F07BFC1D4900
:1072C0001B4805F090FC0421194805F089FBFF20BC
:1072D000009001236A460321154805F09AFB00211E
:1072E000134805F07DFB9DF80000012802D04FF007
:1072F000FF3091E700210E4805F0EFFB01210C481B
:1073000005F05AFA01210A4805F0CEFB002408488E
:1073100080F84B5005E006E0FFE70024044880F8C1
:107320004B5000BF01E0002076E7204674E70000E4
:10733000987A002078410020F8B5044600261448C9
:1073400090F84700A04221D014B1012C04D101E0F3
:10735000002504E0012502E04FF0FF3600BF00BF2A
:1073600016B14FF0FF30F8BD2946094805F0B8FCCA
:107370006946074805F096FC9DF80000A84202D037
:107380004FF0FF30EFE7024880F847403046EAE729
:10739000987A0020F8B504460026144890F8480072
:1073A000A04220D01CB1012C03D1012504E000250E
:1073B00002E04FF0FF3600BF00BF16B14FF0FF30C4
:1073C000F8BD2946094805F0A4FC6946074805F0C0
:1073D00058FC9DF80000A84202D04FF0FF30EFE7C4
:1073E000024880F848403046EAE70000987A0020DA
:1073F00000B589B0202101A8EFF74CF810480068CB
:1074000048B10F480FA1026801A8F5F733FB01A9A5
:107410001420F0F7B3FC1048006848B10E480FA1E3
:10742000026801A8F5F726FB01A91420F0F7A6FCD5
:107430000020034908600849086009B000BD000049
:107440007C4100207370695F77726974655F657253
:10745000722C25640D0A0000804100207370695F62
:10746000726561645F6572722C25640D0A0000000C
:107470001CB51F480021816081810121C17300205A
:107480001B4988731B4848601B4808600020032183
:1074900003460122CDE9001011460B2007F0DDFF65
:1074A00000210B2008F0DEF9C8200BF0D3F80121F1
:1074B0000B2008F0D7F90D2008F047F800210D2027
:1074C00008F0D0F90F2008F040F801210F2008F053
:1074D000C9F9C8200BF0BEF8F1F77EFB0EF018FBDF
:1074E0000446601C10B94FF0FF301CBD0020FCE7C3
:1074F000347B0020C5320400E932040070B5054633
:107500001848807B48B3184800210160818002F050
:1075100081FC0446601C10B94FF0FF3070BD12486A
:10752000801C02F088FC0446601C10B94FF0FF304C
:10753000F4E70D48001D02F08FFC0446601C10B9F2
:107540004FF0FF30EAE70848008828800648408866
:10755000688005488088A88002E04FF0FF30DDE7B2
:107560000020DBE7347B0020984100201CB5002080
:10757000032103460122CDE9001011460B2007F03C
:107580006CFF0D2007F0E1FF0C2007F0DEFF0E205E
:1075900007F0DBFF0F2007F0D8FF00210D2008F0D7
:1075A00061F900210C2008F05DF900210E2008F09F
:1075B00059F900210F2008F055F900210B2008F09F
:1075C00051F900201CBD00001CB50020032103461A
:1075D0000122CDE9001011460B2007F03EFF0121EA
:1075E0000B2008F03FF90D2007F0AFFF00210D2020
:1075F00008F038F90F2007F0A8FF01210F2008F04C
:1076000031F9F1F7E9FA094800218160818101210E
:10761000C1730020054988730EF07AFA0446601C95
:1076200010B94FF0FF301CBD0020FCE7347B002078
:107630003EB505466348807BA84270D025B1012D38
:107640001ED0022D1BD16BE000200EF07DF8044609
:10765000601C10B94FF0FF303EBD684602F072FC6E
:107660000446601C10B94FF0FF30F5E79DF80000AC
:1076700010B14FF0FF30EFE70020524988739EE0D1
:1076800001200EF061F80446601C10B94FF0FF3085
:10769000E2E7684602F056FC0446601C10B94FF061
:1076A000FF30D9E79DF80000012802D04FF0FF30ED
:1076B000D2E706200EF01CF80446601C10B94FF00B
:1076C000FF30C9E702A802F001FC0446601C10B9B3
:1076D0004FF0FF30C0E79DF80800062802D04FF0B9
:1076E000FF30B9E702200DF0DDFF0446601C10B941
:1076F0004FF0FF30B0E701A802F0C0FB0446601C69
:1077000010B94FF0FF30A7E79DF80400022802D01F
:107710004FF0FF30A0E701202A4988734FE04FE087
:1077200001200EF011F80446601C10B94FF0FF3034
:1077300092E7684602F006FC0446601C10B94FF060
:10774000FF3089E79DF80000012802D04FF0FF309C
:1077500082E702200DF0CCFF0446601C10B94FF008
:10776000FF3079E702A802F0B1FB0446601C10B9B3
:107770004FF0FF3070E79DF80800022802D04FF06C
:10778000FF3069E701200DF08DFF0446601C10B941
:107790004FF0FF3060E701A802F070FB0446601C68
:1077A00010B94FF0FF3057E79DF80400012802D0D0
:1077B0004FF0FF3050E702200249887300BF00BF3E
:1077C000002049E7347B00201CB50020032103463C
:1077D0000122CDE900101146122007F02AFE1320E5
:1077E00007F0A7FE142007F0A4FE0021132008F0E4
:1077F0001CF80021142008F018F80021122008F0CD
:1078000014F8052007F0BEFC0121122008F00DF845
:10781000052007F0B7FC104A10A14FF47A70F3F777
:10782000B7F8F1F778F813480021016041608160F2
:10783000C16011480F4948601048086000210D4898
:10784000C17300200B4988730BF060FD08B1002064
:107850001CBD4FF0FF30FBE74D7A0300716D635F95
:107860006969635F6572726F725F7265706F72745F
:1078700000000000247B0020CD26040031270400F6
:1078800001460248C089088000207047247B002000
:107890007CB5044601208DF80000134806236A4693
:1078A000012146683820B047054615B94FF0FF3032
:1078B0007CBDBCB19DF800009DF8011040EA01209C
:1078C00000B220809DF802009DF8031040EA0120DC
:1078D00000B260809DF804009DF8051040EA012088
:1078E00000B2A0800020E3E7247B002010B50BF05D
:1078F0000DFD08B1002010BD4FF0FF30FBE7042064
:1079000070471CB50020032103460122CDE9001079
:107910001146122007F08DFD132007F00AFE1420F7
:1079200007F007FE0021132007F07FFF002114203D
:1079300007F07BFF0021122007F077FF00201CBD1D
:1079400010B50121122007F070FFF0F7E4FF0448A2
:10795000002181608181C17300200149887310BDBD
:10796000247B0020F8B505460E464FF0FF37002E69
:1079700001DD052E02DB4FF0FF30F8BD3248807B81
:10798000A8425CD0012E06D0022E18D0032E2ED095
:10799000042E53D13BE085B1062000902A480123F4
:1079A0006A462921D0F800C03820E047044614B9BF
:1079B0004FF0FF30E1E7002700E000273EE0A5B1EF
:1079C000FF200090204801236A462921D0F804C0F6
:1079D0003820E04704461CB19DF80000062802D07C
:1079E0004FF0FF30C9E7002700E0002726E00095B0
:1079F000154801236A460A21D0F800C03820E04724
:107A0000044614B94FF0FF30B7E7002716E0FF2017
:107A100000900D4801236A460A21D0F804C038209E
:107A2000E04704461CB19DF80000A84202D04FF088
:107A3000FF30A2E700270448857300BF01E0002063
:107A40009BE7384699E70000247B002000B589B009
:107A5000202101A8EEF71EFD1048006848B10F482C
:107A60000FA1026801A8F5F705F801A91520F0F7A4
:107A700085F91048006848B10E480FA1026801A8B6
:107A8000F4F7F8FF01A91520F0F778F90020034971
:107A900008600849086009B000BD0000904100205E
:107AA0006969635F77726974655F6572722C2564BA
:107AB0000D0A0000944100206969635F726561648A
:107AC0005F6572722C25640D0A00000070B50546D2
:107AD0000C464FF4803000FA04F1284600F03EFBDB
:107AE00070BD70B505460C464FF4A07000EB8400E5
:107AF00086B23146284600F04BFB70BD2DE9F047B9
:107B000004460D4616461F464FF4803000FA05F82D
:107B10004FF4A07000EB85001FFA80F926F07F4635
:107B20004146206808F044F94146206808F031F9E0
:107B30004946206808F023F932462946206808F0B3
:107B40000EF94146206808F02AF91FB14146206825
:107B500008F034F9BDE8F08710B50446206808F055
:107B600003F910BD2DE9F04303460C46164658793B
:107B7000284941F820605879274901EBC000007975
:107B800018B108221046BDE8F08321881868C0F8B3
:107B9000081500BF93F90450A778284639460028F5
:107BA00008DB4FEA417C4FEA1C68DFF870C00CF834
:107BB00000800BE04FEA417C4FEA1C69DFF860C0AF
:107BC00000F00F08A8F104080CF8089000BF00BFEF
:107BD00093F90410084600280DDB00BF00BF00F039
:107BE0001F070125BD404709BF0007F1E027C7F87F
:107BF000005100BF00BF00BF00BF01205979064DF2
